:100000000000012085FF0000ADFF0000AFFF0000F1
:10001000B1FF0000B3FF0000B5FF000000000000CA
:10002000000000000000000000000000B7FF00001A
:10003000B9FF000000000000BBFF0000BDFF000092
:10004000BFFF0000BFFF00003D050100BFFF000033
:1000500069A90000BFFF0000BFFF0000BFFF000054
:10006000BFFF0000BFFF0000BFFF0000BFFF000098
:10007000BFFF0000BFFF0000BFFF0000BFFF000088
:10008000BFFF000001090100BFFF0000BFFF00002B
:10009000BFFF0000BFFF0000BFFF0000BFFF000068
:1000A000BFFF0000BFFF0000BFFF0000BFFF000058
:1000B000BFFF0000BFFF00000000000000000000C4
:1000C000BFFF0000BFFF0000BFFF0000BFFF000038
:1000D000BFFF0000BFFF0000BFFF000000000000E6
:1000E0000000000000000000000000000000000010
:1000F0000000000000000000000000000000000000
:1001000000000000000000000000000000000000EF
:1001100000000000000000000000000000000000DF
:1001200000000000000000000000000000000000CF
:1001300000000000000000000000000000000000BF
:1001400000000000000000000000000000000000AF
:10015000000000000000000000000000000000009F
:10016000000000000000000000000000000000008F
:10017000000000000000000000000000000000007F
:10018000000000000000000000000000000000006F
:10019000000000000000000000000000000000005F
:1001A000000000000000000000000000000000004F
:1001B000000000000000000000000000000000003F
:1001C000000000000000000000000000000000002F
:1001D000000000000000000000000000000000001F
:1001E000000000000000000000000000000000000F
:1001F00000000000000000000000000000000000FF
:1002000010B5054C237833B9044B13B10448AFF350
:1002100000800123237010BDA00200200000000018
:10022000489D010008B5034B1BB103490348AFF3D8
:10023000008008BD00000000A4020020489D0100CD
:10024000154B002B08BF134B9D46A3F5803A0021A8
:100250008B460F461348144A121A12F082FE0F4BB7
:10026000002B00D098470E4B002B00D09847002061
:10027000002104000D000D48002802D00C48AFF307
:10028000008012F0B7FD2000290010F079FB12F079
:10029000FFFB00BF0000080000000120000000007C
:1002A00000000000A00200207C09002000000000E7
:1002B000000000000020704700207047F0B50446A1
:1002C00085B00E46684611461F4609F0F7FE2368C2
:1002D0006A465D6A31463B462046A84705B0F0BDF8
:1002E000F0B5044685B00E46684611461F4609F033
:1002F000F4FD23686A465D6A31463B462046A847BE
:1003000005B0F0BD70B590B00C4615461E4605F020
:1003100041FC48B364B321464022684613F0F5FD22
:100320002F21684613F088FD28B923460322402177
:10033000684609F045FE3F223146684613F0BFFD8E
:100340000C480EF0E7FC78B10B4B93F90030062B0C
:100350000CD10A4B93F9003043B901232A46694670
:1003600004480EF034FF012010B070BD0020FBE700
:100370002046F9E7E0030020D8030020B003002066
:1003800007B5002300931A46194603480FF032FCC4
:1003900003B05DF804FB00BFBC02002007B50023DA
:1003A00000931A46194603480FF024FC03B05DF889
:1003B00004FB00BFC402002082B002AB012003E9AD
:1003C000060002B0704700207047406818B100680E
:1003D00008B1007C0009704743682BB11B681BB152
:1003E0001A7C61F307121A747047406808B508B1A7
:1003F00001F03AFF012008BD13B500220446114662
:10040000684604F08BF8606801F02EFF052807D8D5
:10041000DFE800F0110311060611012002B010BD43
:1004200061684FF40072684604F06AFC0021684677
:1004300004F036FBF2E70020F0E713B50022044693
:100440001146684604F06AF82046FF22694604F027
:10045000A2FB204602B010BD07B5002300931A4648
:10046000194603480FF0C6FB03B05DF804FB00BF5C
:10047000CC020020704700002DE9FF4102AC84E867
:10048000060006463B493C489DF828809DF82C50C4
:100490001F460FF0F7FB204604F0BCFD204604F099
:1004A000BBF950BB204604F01DFC052804D8DFE84A
:1004B00000F0152417030317054630492E480FF0A6
:1004C000E1FB0A2229462C480FF045FC2A480FF090
:1004D000E9FB204604F09EFD00200BE04FF00108F0
:1004E000CDE90085336894E80600DD6B30463B4675
:1004F000A847012004B0BDE8F081204604F03CFB91
:10050000012812D0022831D01D491B480FF0BAFB38
:10051000204604F031FB0A22014617480FF034FC54
:1005200015480FF0BFFB0125C7E70021204604F066
:1005300009FA13280ED81E21204604F073FA7168B8
:100540004FF40072204605F0B9F84FF490517068EE
:1005500002F012FD0195336801250095D3F83C8027
:1005600094E806003B463046C047C2E700230393A9
:10057000F0E700BFA479010068030020BA79010008
:10058000AD79010008B511B9B0F9080008BDB0F99E
:100590000A208A4203DC0089084400B2F6E740687A
:1005A00001F00CFFF9E7000007B5002300931A469D
:1005B000194603480FF01EFB03B05DF804FB00BFB3
:1005C000D40200200A460068022100F099BD000014
:1005D00070B503680546F3B17221FFF7F3FF286891
:1005E0000E4E03680021DB69984700242868042C1C
:1005F00003680CD0DB689847A35D984205D0286853
:1006000003685B6A9847002070BD0134EEE75B6ABF
:1006100098470120F8E71846F6E700BF147A010072
:100620002DE9F041036804461BB900263046BDE8B9
:10063000F081FFF7CDFF07460028F6D0254672214E
:100640002046FFF7BFFF55F8100B03680421DB6954
:10065000984704F11608002620680368DB6898476D
:10066000C0B205F8010B0138C0B2FD2898BF3E4664
:10067000A845F1D1206803685B6A9847D6E7F8B5CA
:10068000036804460F4613B900252846F8BDFFF756
:100690009FFF05460028F7D072212046FFF792FF02
:1006A000206803682646DB690421984756F8100B3A
:1006B000036806225B68394698473B682361BB881C
:1006C000B380206803685B6A9847DEE770B503680B
:1006D00004460D46164613B90025284670BDFFF79F
:1006E00077FF0028F8D072212046FFF76BFF2068C3
:1006F00003684021DB699847731E2A460021206861
:100700000FF0A4FD06B2206803685B6A9847002ECC
:10071000E2D00023AB55E0E738B5036804460D4648
:100720000BB9002038BDFFF753FF0028F9D0284649
:1007300013F0BDFB0F28F4D872212046FFF742FFCB
:10074000206803684021DB699847294620680FF03C
:10075000A2FA2068036800211B68984705462068B4
:1007600003685B6A9847281C18BF0120DAE738B590
:10077000036804460D460BB9002038BDFFF728FF7B
:100780000028F9D0284613F092FB0F28F4D87221E4
:100790002046FFF717FF206803685021DB69984760
:1007A000294620680FF077FA2068036800211B684B
:1007B00098470546206803685B6A9847281C18BF5D
:1007C0000120DAE770B5036804460D46164613B9F2
:1007D0000025284670BDFFF7FBFE0028F8D07221E7
:1007E0002046FFF7EFFE206803682021DB69984769
:1007F000731E2A46002120680FF028FD06B22068EB
:1008000003685B6A9847002EE2D00023AB55E0E70F
:1008100038B5036804460D460BB9002038BDFFF714
:10082000D7FE0028F9D0284613F041FB1F28F4D842
:1008300072212046FFF7C6FE206803682021DB698D
:100840009847294620680FF026FA2068036800219F
:100850001B6898470546206803685B6A9847281C10
:1008600018BF0120DAE773B5036805460E461BB9C9
:100870000024204602B070BDFFF7AAFE04460028FF
:10088000F6D072212846FFF79DFE286803681021E4
:10089000DB69984704220DEB020128680FF0C1FCC8
:1008A000019930460FF0C3F9286803685B6A9847DE
:1008B0003379002BDCD0FF2BDBD17379FF2BD8D120
:1008C000B379FF2BD5D1F479FF3C18BF0124D0E7D1
:1008D00073B5036805460E461BB90024204602B0D6
:1008E00070BDFFF775FE04460028F6D07221284639
:1008F000FFF768FE286803681C21DB69984704221B
:100900000DEB020128680FF08CFC019930460FF0C6
:100910008EF9286803685B6A98473379002BDCD02E
:10092000FF2BDBD17379FF2BD8D1B379FF2BD5D136
:10093000F479FF3C18BF0124D0E773B5036805467E
:100940000E461BB90024204602B070BDFFF740FEE2
:1009500004460028F6D072212846FFF733FE2868A7
:1009600003681421DB69984704220DEB0201286813
:100970000FF057FC019930460FF059F928680368C9
:100980005B6A98473379002BDCD0FF2BDBD173797E
:10099000FF2BD8D1B379FF2BD5D1F479FF3C18BF09
:1009A0000124D0E773B5036805460E461BB9002441
:1009B000204602B070BDFFF70BFE04460028F6D0BB
:1009C00072212846FFF7FEFD286803681821DB69BD
:1009D000984704220DEB020128680FF022FC0199D0
:1009E00030460FF024F9286803685B6A984733792A
:1009F000002BDCD0FF2BDBD17379FF2BD8D1B3795F
:100A0000FF2BD5D1F479FF3C18BF0124D0E737B5CF
:100A10004B6801930368044613B9002003B030BD4E
:100A2000FFF7D6FD0028F8D072212046FFF7CAFD57
:100A3000206803681021DB69984720680368042256
:100A40005B680DEB020198470546206803685B6A06
:100A50009847281C18BF0120E0E737B54B68019381
:100A60000368044613B9002003B030BDFFF7B0FDA2
:100A70000028F8D072212046FFF7A4FD2068036803
:100A80001C21DB6998472068036804225B680DEB32
:100A9000020198470546206803685B6A9847281C4E
:100AA00018BF0120E0E737B54B680193036804469F
:100AB00013B9002003B030BDFFF78AFD0028F8D03D
:100AC00072212046FFF77EFD206803681421DB6950
:100AD00098472068036804225B680DEB0201984781
:100AE0000546206803685B6A9847281C18BF0120E8
:100AF000E0E737B54B6801930368044613B900205B
:100B000003B030BDFFF764FD0028F8D07221204605
:100B1000FFF758FD206803681821DB6998472068B3
:100B2000036804225B680DEB0201984705462068C4
:100B300003685B6A9847281C18BF0120E0E713B5DB
:100B40007723009303680446A3B1FFF741FD88B102
:100B500072212046FFF736FD206803680C21DB690F
:100B600098470422694620680FF05BFB2068036801
:100B70005B6A9847009B0020DAB262F30700C3F378
:100B8000072262F30F20C3F3074262F317401B0EE4
:100B900063F31F6002B010BD37B5019103680446CE
:100BA00013B9002003B030BDFFF712FD0028F8D0C4
:100BB00072212046FFF706FD206803680C21DB69DF
:100BC00098472068036804225B680DEB0201984790
:100BD0000546206803685B6A9847281C18BF0120F7
:100BE000E0E707B5FFF7ABFFC043C0F3C01003B0A9
:100BF0005DF804FB37B505460C46FFF7A0FF84F00F
:100C00000104019064F3C7108DF80400019928468F
:100C100003B0BDE83040FFF7BFBF07B5FFF78FFF58
:100C2000C0F3002003B05DF804FB37B50D46044661
:100C3000FFF785FF0190C0F3072065F300008DF8F2
:100C400005000199204603B0BDE83040FFF7A4BF7E
:100C500007B5FFF774FF80F00800C0F3C00003B0D1
:100C60005DF804FB37B505460C46FFF768FF84F0D6
:100C70000104019064F3C3008DF804000199284633
:100C800003B0BDE83040FFF787BF37B50D460446D7
:100C9000FFF755FF019065F302008DF804000199FC
:100CA000204603B0BDE83040FFF776BF37B50D46AC
:100CB0000446FFF744FF019065F306108DF8040029
:100CC0000199204603B0BDE83040FFF765BF07B586
:100CD000FFF735FF00F0070003B05DF804FB07B530
:100CE000FFF72DFFC0F3021003B05DF804FB000016
:100CF00070B51E4D0C468AB0064604341C49284681
:100D00000EF0C0FF214607A80FF0DDFC07A928461A
:100D10000EF0BCFF2846174D0EF0C4FF07A80FF0D9
:100D200042FC294601A80FF083FC01A904A80FF09A
:100D3000CAFC214604A80FF006FD2946044607A870
:100D40000FF076FC07A920460FF0FDFC0146304667
:100D50000FF0B9FC07A80FF026FC04A80FF023FC45
:100D600001A80FF020FC30460AB070BD68030020D7
:100D7000197A0100247A01007FB50D46044622212C
:100D800028460FF035FD2221064628460FF04AFD81
:100D9000002E034604F1040422DB002820DD721C2F
:100DA000294601A80FF042FD01A920460FF095FC4D
:100DB00001A80FF0F8FB0D490D480EF063FF214626
:100DC00001A80FF080FC01A909480EF05FFF084858
:100DD0000EF068FF01A80FF0E6FB012004B070BD23
:100DE000294620460FF060FCE5E700BF267A0100A7
:100DF000680300207FB503680446002B39D07721B3
:100E0000FFF7E0FB206803680021DB6998470025B5
:100E1000206802690368954204D21B680021984744
:100E20000135F5E7DB69144E00219847002520685D
:100E3000715D036801351B689847042DF7D1206860
:100E400003685B6A98470D4901A80FF0F1FB01A9FF
:100E50002046FFF791FF01A80FF0A5FB07212046D0
:100E6000FFF713FF07212046FFF720FF012004B002
:100E700070BD1846FBE700BF147A0100029801001C
:100E80007FB50368044613B9002004B070BDFFF7B6
:100E90009FFB0028F8D0E3681F2BF5D82646722167
:100EA0002046FFF78FFB56F8040B03686021DB69CF
:100EB0009847314620680EF0E9FE2068036800215B
:100EC0001B6898470546206803685B6A98478DB1A0
:100ED0000A490B480EF0D6FE314601A80FF0F3FB8D
:100EE00001A907480EF0D2FE05480EF0DBFE01A86E
:100EF0000FF059FB281C18BF0120C6E73E7A0100FD
:100F00006803002030B5036885B0044613B900209B
:100F100005B030BDFFF75CFB0028F8D025467221F4
:100F20002046FFF74FFB55F8040B03686021DB698F
:100F300098470022216801A80FF0A2F901A92846CC
:100F40000FF0CBFB01A80FF02EFB206803685B6A53
:100F500098470B490B480EF095FE294601A80FF063
:100F6000B2FB01A907480EF091FE06480EF09AFE6A
:100F700001A80FF018FBE068003018BF0120C7E798
:100F8000317A01006803002007B5002300931A4658
:100F9000194603480EF02EFE03B05DF804FB00BFB7
:100FA000DC02002007B5002300931A4619460348C7
:100FB0000EF020FE03B05DF804FB00BFE402002049
:100FC00001207047C08A7047027D1AB10368FF2173
:100FD0001B68184770470369994228BF1946816109
:100FE00008467047037D10B5044633B9A0692369EC
:100FF00098422CBF0020012010BD03681B69984750
:10100000FF28F3D10020F7E7036810B504461B69F9
:101010009847A3690133A36110BD704708B5026901
:101020008369934205D2C169034819440EF031FC2B
:1010300008BD4FF0FF30FBE7EC02002010B5D0E90F
:1010400006345A1C82610A460248E1180EF023FC5D
:10105000012010BDEC02002008B590F82020772A6E
:101060000BD10368DB6A9847044905480EF00AFE75
:101070000348BDE808400EF015BE08BD637A0100C4
:1010800068030020F0B50D4685B004463F21284690
:1010900017460FF0ADFB031E0BDB0022294601A80B
:1010A0000FF0C4FB01A928460FF017FB01A80FF0B1
:1010B0007AFA114928460FF052FB064660B1002328
:1010C000A3614FF4FA43236101208423E361207577
:1010D00084F8207005B0F0BD084928460FF03FFBAA
:1010E0000028F7D08423C4E906662361267584F8B6
:1010F00020700120EEE700BF4A7A0100577A010014
:1011000001294FF0000303D002290CD01846704784
:1011100083614FF4FA4303618423C361017580F84E
:101120002020012070478421C0E906330161037546
:10113000F5E7000007B5002300931A461946044856
:101140000EF058FD034803B05DF804EB0EF09EBBB3
:10115000ED020020EC02002038B50023836083807C
:10116000036804460D46002B47D0274A1268002A20
:1011700043D0002908BF1D462B7C03F00F03062B2C
:1011800010D1224A224829460DF073FA08B143696A
:101190002371204A1E4829460DF06BFA00282DD0F5
:1011A000436963711C4A216819480DF062FA0546CB
:1011B00008BB1A491A480EF065FD0A2261791848E1
:1011C0000EF0E2FD174916480EF05CFD0A22217967
:1011D00013480EF0D9FD12480EF064FD2B460E4A5E
:1011E00021680B480DF08DFA0B4A216808480DF074
:1011F00040FA054608B11435A56038BD286811F0DD
:101200002AFC6071CEE700BF300400204097010047
:101210006C070020A87A01000E7B0100117B010001
:10122000680300208087010010B504460160114664
:10123000FFF792FF204610BD41790C4A002352F877
:101240002300884203D10A4A52F82300704752F81B
:10125000230028B942F82310054A42F823007047BA
:101260000133052BEBD10020704700BF04030020A1
:101270001803002010B50A4A4079002352F8234091
:10128000844203D1074A42F8231010BD52F823408C
:1012900014B952F82320F5E70133052BEED1F4E71A
:1012A0000403002018030020F0B52DED028B9BB045
:1012B0000446FFF7C1FF05460FF0E0FA00230146A0
:1012C00043F69822284608F00FFF002800F0E78038
:1012D00006231622617905A80EF0D2F8372105A859
:1012E0000EF0DEF80022114605A80EF0F5F90021F7
:1012F00008EE900A05A80EF087FA6B4908EE100A6E
:101300006A480EF0BFFC0A22617968480EF03CFD85
:10131000674966480EF0B6FC18EE900A10F0DAFF46
:10132000022502460B46009560480EF0E9FD614932
:101330005E480EF0A7FC18EE100A10F0CBFF0095E7
:101340000B46024659480EF0DBFD5B4957480EF04C
:1013500099FC56480EF0A6FC584A216858480DF0F2
:1013600088F9584A2168074655480DF082F9F4EE8D
:10137000688AF1EE10FA06460FD60AAD18EE901AFA
:10138000284603F0D8F80023CDE900334FF0FF31B1
:1013900095E80C00384608F0C1FEB4EE488AF1EE3C
:1013A00010FA0FD60AAD18EE101A284603F0C3F84B
:1013B0000023CDE900334FF0FF3195E80C003046B3
:1013C00008F0ACFE404A21683D480DF052F9054650
:1013D00000285ED0037C03F00F03042B59D1F5EEF7
:1013E000408AF1EE10FA54D0B5EE408AF1EE10FAD0
:1013F0004FD0F4EE688AF1EE10FA4AD1B4EE488A82
:10140000F1EE10FA45D100213C220BA80A9111F00F
:10141000A8FD696940220AA812F077FD2F210AA8C9
:1014200012F00AFD28B96B69032240210AA808F0CE
:10143000C7FD26490AA812F0F0FC02A818EE901A7F
:1014400008F04BFD22480DF065FC40B1214B93F9AB
:10145000003023B902AA0AA91D480DF0A3FE0AA86C
:1014600012F025FD1AAB1844482300F8413C18EE51
:10147000101A02A808F031FD15480DF04BFC40B1E0
:10148000144B93F9003023B902AA0AA910480DF0B1
:1014900089FE0FF0F3F901462046FFF7EBFE1BB083
:1014A000BDEC028BF0BD00BF0A7B01006803002089
:1014B000167B0100267B01002D7B01002F7B0100A4
:1014C0006C070020347B0100387B0100409701004D
:1014D000E0030020B00300202DE9F04F054600682E
:1014E00087B00F46904640B1A86830B10378FF2915
:1014F00003F0100335D11BB9012007B0BDE8F08F10
:10150000032AF9D047789C499C480EF0BBFB0A227D
:1015100069799A480EF038FC994998480EF0B2FB68
:10152000AB68964859780A2201F00F010EF02CFCA6
:101530003F09944991480EF0A5FB0A2239468F488D
:101540000EF022FC8D480EF0ADFBAB685A7802F02D
:101550000F02BA4207D11A786FF304121A700020F2
:10156000CBE7002BFBD100220DF1080911464846BC
:1015700002F0D4FFAB685B7803F00F03BB4223D0CB
:10158000B8F1030F20D080497C480EF07BFB0A2283
:1015900069797A480EF0F8FB794978480EF072FBC9
:1015A000AB68764859780A2201F00F010EF0ECFB87
:1015B000744972480EF066FB0A2239466F480EF0F5
:1015C000E3FB6E480EF06EFB29680C2F00F2AF8033
:1015D000DFE807F0073A94A1A3947394A5A784A920
:1015E000AB00AB685B7803F00F03023B082B24D8F9
:1015F000DFE803F00523239D230F23231900634A0B
:1016000063480DF036F8AB681C78064604F0010418
:101610002DE0604A5E480DF02CF8AB681C78064659
:10162000C4F3400423E05C4A59480DF022F8AB684B
:101630001C780646C4F3800419E0584A54480DF05B
:1016400018F80646002412E0554A51480DF011F8EA
:10165000AA681378D94303F0010461F300031370FF
:10166000064620B90122494604A803F034FB4D4A3E
:10167000296847480CF0FDFF4B4A296882464448D8
:101680000CF0F7FF834638B9BAF1000F04D1524687
:10169000494604A803F01FFB002E4BD1484603F037
:1016A000BBF8002846D1AB685A7867F303025A703A
:1016B0001A7866F304121A701EE73C4A34480CF09C
:1016C000D8FFA9680B7883F00202C2F34002C3F38B
:1016D0004004064662F341030B70C8E7344A2C48C5
:1016E0000CF0C7FFA9680B7883F00402C2F38002F4
:1016F000C3F38004064662F38203EDE7274A2448D9
:101700000CF0B7FF064600289CD10222494604A8E7
:1017100003F0E1FA96E7274A72E7274A70E7274A7B
:1017200078E7274A76E7274A7EE7274A7CE70024BE
:1017300026469CE7AB68B8F1030F5A780FD067F3E1
:1017400003025A701A786FF304121A70CDE900ABD5
:10175000214699E80C00304608F0E0FCCCE602F0A7
:101760000F01B9423FF4C8AE67F307125A701A78F6
:1017700042F010029FE700BFA07A0100680300203A
:101780004C7B0100AA7A0100A87A0100AE7A010020
:101790006C070020AD7A0100B47A0100BB7A010029
:1017A000C07A0100F67A0100387B0100C57A010099
:1017B000CB7A0100D17A0100D67A0100DC7A0100EF
:1017C000E27A0100E97A0100EF7A01002DE9F043A5
:1017D0005D4A95B00746884601685C480CF049FFB1
:1017E0005B4A3968814659480CF043FF0646B9F117
:1017F000000F01D100287AD0564A396853480CF0BE
:1018000038FF554A3968054650480CF032FF5349B5
:10181000044653480EF036FA0A22797950480EF001
:10182000B3FA50494E480EF02DFA0A2241464C4870
:101830000EF091FA4A480EF035FA5EB3337C03F0AD
:101840000F03042B26D14022716904A812F05DFB1E
:1018500045480DF05FFAE8B1444B93F90030CBB93D
:101860002F2104A812F0E8FA28B973690322402155
:1018700004A808F0A5FBB8F1000F41D025B12B7CDE
:1018800003F00F03042B35D0394A012304A936484D
:101890000DF09DFCB9F1000F29D099F8103003F03C
:1018A0000F03042B23D1D9F8141004A800F062FF11
:1018B00004A800F09DFEB8B1B8F1000F34D025B1F6
:1018C0002B7C03F00F03042B25D002AC0122002156
:1018D000204602F023FE01220023CDE9002304A8C4
:1018E00094E8060001F0AAFB04A800F0B3FC15B0D0
:1018F000BDE8F0836A691378002BCBD00123C5E7DC
:1019000024B1237C03F00F03042B02D00123194AD6
:10191000BCE76269EFE769690B78002BE4D000222D
:1019200004A802F0FFF9DFE724B1237C03F00F03E2
:10193000042B02D002AC0222C9E761690B78002BAC
:10194000D2D04246ECE700BFF67A01006C070020D7
:10195000387B0100C07A0100BB7A0100037B0100E3
:10196000680300202B7B0100E0030020B00300206F
:10197000EA900100F590010070B598B0054602AC00
:1019800084E8060039483A490EF07CF90A22697960
:1019900036480EF0F9F9374934480EF073F920460D
:1019A00003F038FB2968344A34480CF062FE002307
:1019B000CDE900334FF0FF3194E80C0008F0AEFBA6
:1019C00029682F4A2D480CF054FE29682D4A0646F6
:1019D0002A480CF04EFE054660B3037C03F00F036B
:1019E000042B27D14169402208A812F08EFA2F213A
:1019F00008A812F021FA28B96B690322402108A82F
:101A000008F0DEFA0023102200930DEB02014FF4E0
:101A10000073204603F0EAF91B480DF07BF948B14A
:101A20001A4B93F900302BB9012304AA08A91648D0
:101A30000DF0CDFBC6B1337C03F00F03042B13D1A3
:101A4000716908A800F096FE08A800F0D1FD40B129
:101A500001220023CDE9002308A894E8060001F044
:101A6000EDFA08A800F0F6FB18B070BD680300207E
:101A70000A7B01002B7B0100FF7A01006C0700202C
:101A8000F67A0100387B0100E0030020B00300205B
:101A900010B503788B42044604D14378402B01D122
:101AA000408810BD40232170637008460EF0DEFFB1
:101AB00080B26080F5E7000083682DE9F0410446BC
:101AC0000D46002B00F05A81AD4F3B780133DBB25D
:101AD0000A46FF213B70FFF7FFFC637926790E3B36
:101AE000072BC6F3400830D8A64A2168A6480CF058
:101AF000C0FD064648B3037C03F00F03052B24D139
:101B00006179A248FFF7C4FF0022804631469E4813
:101B10000CF0A5FD436998451FDA0026032D60D01F
:101B2000A3685A7802F00F02013A0B2A59D8DFE86D
:101B300012F01F00ED0042006A00ED007200ED009F
:101B40009100A200AA00D300E50060790FF0BEF872
:101B5000A8EB00035E425E41E0E7314601228A487D
:101B60000CF07DFD4669B045CCBF00260126D5E7C7
:101B7000B3F802800EF082FE4FF6FF7381B24FF48D
:101B80007A72404608F0B0FA58B3814A21687E481C
:101B90000CF06FFD28B12A4603212046FFF79CFC7C
:101BA0001FE07C4A216878480CF063FD0028F2D1E0
:101BB0002A460D21F1E7B3F802800EF05FFE4FF6E2
:101BC000FF734FF4967281B2404608F08DFA40B12F
:101BD0002A4604212046FFF77FFC0EF04FFEA36843
:101BE0005880A2681378C3F3C001B14200F0468167
:101BF00013F0E00F00F09C80C3F34211013961F350
:101C000047131370B6E0B3F802800EF037FE4FF6BC
:101C1000FF739622D7E7B3F802800EF02FFE4FF63F
:101C2000FF7381B24FF47A72404608F05DFA0028E3
:101C3000D7D0594A216854480CF01BFD10B12A46F0
:101C40000821AAE7554A21684F480CF012FD0028E8
:101C5000F5D1ADE7B3F802800EF010FE4FF6FF733A
:101C60004FF4967281B2404608F03EFA0028B8D090
:101C70002A460921AEE7B3F802800EF0FFFD4FF6C9
:101C8000FF739622EEE7B3F802800EF0F7FD4FF6F1
:101C9000FF7381B24FF47A72404608F025FA0028AB
:101CA0009FD03F4A216838480CF0E3FC10B12A4627
:101CB0000B2172E73B4A216833480CF0DAFC00281C
:101CC000F5D1394A216830480CF0D3FC00287FF464
:101CD0006FAF2A46062160E7B3F802800EF0CEFD12
:101CE0004FF6FF734FF4967281B2404608F0FCF94C
:101CF00000283FF476AF2A460C216BE7B3F8028048
:101D00000EF0BCFD4FF6FF739622EDE7B3F80280AC
:101D10000EF0B4FD4FF6FF7381B24FF416724046D9
:101D200008F0E2F900283FF45CAF2A46002134E7CE
:101D30000EF0A4FDA36858805B7803F00F03002E1B
:101D400051D0072B11D8DFE803F04810041010041D
:101D5000104B164A21680C480CF08BFC40B32A4605
:101D600006212046FFF7B8FB20B1A3681A7866F376
:101D7000C3021A703B78013BDBB23B70BDE8F081D7
:101D800000030020FB7A01006C0700202C030020D8
:101D9000D17A0100D67A0100DC7A0100E27A0100F2
:101DA000E97A0100EF7A0100CB7A0100C57A0100DF
:101DB000334A216833480CF05CFC0028CFD1324A0A
:101DC000216830480CF055FC0028C8D12F4A216802
:101DD0002C480CF04EFC0028C1D12A460121C0E756
:101DE0002A460A21BDE7013B0C2BBED801A252F8BE
:101DF00023F000BF291E00006B1D00002F1E0000F5
:101E00002F1E00006B1D0000351E00006B1D000022
:101E1000771E0000771E0000771E0000771E00006E
:101E2000771E00002F1E00002A46022199E72A464D
:101E3000052196E7164A216812480CF01AFC10B1E9
:101E40002A4607218DE70E4A21680E480CF011FC46
:101E50000028F5D10C4A21680A480CF00AFC002839
:101E6000EED12168094A07480CF003FC014600281E
:101E7000E6D12A4675E72A46002172E70221BEE62E
:101E8000DC7A01006C070020E27A0100AD7A0100E3
:101E9000C57A01002DE9F047032986B0804669D054
:101EA0000168624A62480CF0E4FB98F805100646A7
:101EB0006048FFF7EDFD05B2002E69D0337C03F0DA
:101EC0000F03052B64D1314659480CF0BEFB0328A3
:101ED00053D90022314656480CF0C1FB0122446917
:101EE000534831460CF0BBFB0222D0F814A05048F6
:101EF00031460CF0B4FB43694D480A2703223146B2
:101F000007FB03F90CF0ABFB43695F4321460097E5
:101F10004B46524628460EF03CFB044631464448A8
:101F20000CF093FB052830D10422314640480CF0D8
:101F300096FBB0F914A03E48BC42C4BF3C4640F2F8
:101F4000FF3531464C45BCBF4C4600250CF07DFBAF
:101F5000022826D10022314635480CF080FB436927
:101F6000AB4251DC0122314631480CF078FB436929
:101F7000AB4258DB06B0BDE8F08705EB8504640092
:101F80004FF000094FF42057C8E74FF0010AD2E79D
:101F900005EB850464004FF000094FF420574FF023
:101FA000010AD8F80830B3F902002A1A002AB8BF8B
:101FB0005242524507DC1A785109052907D80131E8
:101FC00061F3471202E01A786FF347121A701B7818
:101FD0009F2B03D94C4501D0BC42CBD1A842C9D0DC
:101FE0000022114604AE02A802F098FA224602A985
:101FF000304602F0FCFD96E806004046FFF7BCFCC8
:10200000D8F808305D80B5E70024D8F80830B3F977
:102010000230A342AED021464046FFF7D7FBD8F8A6
:1020200008305C80A6E70124EFE700BFFB7A0100DF
:102030006C0700202C03002008B583680246F3B12A
:10204000012916D00ADB032908DC0379402B0CD0C8
:1020500006D8032B02D81046FFF72EFD002010E013
:10206000422B02D0FAD3803BF3E71046FFF712FF72
:10207000F4E70379042BF1D1FFF716F9EEE74FF0FF
:10208000FF3008BD7FB5037C03F00F03062B054628
:1020900023D10146124A13480CF0EBFA90B1037CAD
:1020A00003F00F03052B0DD1C4680026ACB12946FF
:1020B00001A80194FFF750F8039B1E600EF034FC5A
:1020C0006468F3E704AC002144F80C5D2046FFF798
:1020D00043F802212046FFF7AFFF04B070BD00BFF8
:1020E000FF7A01006C07002038B583680446BBB155
:1020F000124B1B68A3B10068FFF7C4FFA36800255B
:102100001D602379032B0CD8012B94BF0221294693
:1021100060790EF0A1FDA3685A7865F303025A7046
:1021200038BD402B03D0422BFAD1294600E00221D2
:102130006079BDE838400EF08FBD00BF300400204C
:10214000002303807047000013B500242346009449
:102150002246214603480DF04DFD034B1C8002B082
:1021600010BD00BFF80200202C03002010B504466B
:1021700070B3204911F06DFE58B31F49204611F08D
:1021800068FE40B31D49204611F063FE28B31C4988
:10219000204611F05EFE10B31A49204611F059FE98
:1021A000F8B11949204611F054FEE0B11749204614
:1021B00011F04FFEC8B11649204611F04AFEB0B1E9
:1021C0001449204611F045FE002814BF00201520B8
:1021D00010BD0120FCE70220FAE70520F8E7062001
:1021E000F6E71320F4E71420F2E70E20F0E70F20C3
:1021F000EEE700BF5C7B0100657B0100807B010096
:10220000897B0100FE7B0100077C0100D17B01007E
:10221000DA7B0100107C010070B5054680B10478BE
:1022200064B1084E012404EB84013144284611F0C6
:1022300010FE18B101340E2CF5D10024204670BDDB
:102240000446FBE7347C0100406910B103681B6958
:102250001847704710B50446406910B103685B68C1
:102260009847204610BD000008B5032201680448C5
:102270000CF0F5F908B1007D08BDFF20FCE700BFB8
:102280006C07002010B503220C46016810480CF0C2
:10229000E6F9E0B1037C13F00D0F18D1022262F3CE
:1022A0000303037443690B4923F07F4323F0FF03C7
:1022B0002343436108480DF0E5FC21460A22064805
:1022C0000DF062FD0448BDE810400DF0EBBC10BD00
:1022D0006C070020DA7E01006803002010B503229D
:1022E0000C46016808480CF0BAF960B1037C03F0B1
:1022F0000F03022B01BF24F07F41406921F0FF0151
:10230000084018BF002010BD6C07002010B5032244
:102310000C46016809480CF0A2F970B1037C13F077
:102320000D0F0AD1022262F30303037424F07F41EC
:10233000436921F0FF011943416110BD6C07002082
:1023400010B50446406968B103685B69984718B1E5
:10235000606903681B69984760690368DB68984790
:1023600008B9012010BD2046FFF77EFF20B14FF4D1
:1023700080712046FFF7CAFFA368002BF1D04FF40D
:1023800000712046FFF7C2FFEBE7000010B5032203
:102390000C46016808480CF062F958B1037C13F050
:1023A0000D0F07D1E143436941F07F4141F0FF0147
:1023B0001940416110BD00BF6C07002038B50C46C4
:1023C0004168054609B9002038BD0B7C03F00F03B6
:1023D000022B03D1002CF6D14869F5E7052BF2D189
:1023E00005480CF032F98442EDDAE2B2696802483D
:1023F0000CF035F94069E7E76C07002038B50D4669
:102400004168044621B9DFED1A7A17EE900A38BD0B
:102410000B7C03F00F03052B15D116480CF015F9B2
:10242000854210DAEAB2616812480CF018F9002807
:10243000E9D0037C03F00F03022B0FD1D0ED057A16
:10244000F8EEE77AE1E7002DDDD16268137C03F056
:102450000F03022B07D1D2ED057AF1E7032BD2D17E
:10246000D0ED057AD1E7032BCDD1D2ED057ACCE7BB
:10247000000000006C07002008B5416869B10B7CC2
:1024800003F00F03022B06D0052B06D104480CF0F5
:10249000DCF800B208BD0120FCE70020FAE700BF2D
:1024A0006C07002008B5816809B9002008BD087CC8
:1024B00000F00F039A1E012A00D90BB90009F5E7B5
:1024C000052BF2D1002203480CF0C9F80028ECD00B
:1024D000007CF3E76C070020826810B5BAB1137C6A
:1024E00003F00F039C1E012C00D983B9516183684E
:1024F0001A7C022161F303021A748268137C03F0D0
:10250000F001602902BF0A2161F30713137410BDA3
:10251000826810B5BAB1137C03F00F039C1E012C26
:1025200000D983B9516183681A7C032161F30302E6
:102530001A748268137C03F0F001602902BF07213E
:1025400061F30713137410BD836853B11A7C02F052
:102550000F02901E012800D91AB91A7C61F30712E4
:102560001A74704708B5C16809B9002008BD0B7C12
:1025700003F00F03022B01D14869F7E7052BF4D1D3
:10258000002203480CF06BF80028EED04069EDE71C
:102590006C0700202DE9F041C36804460F46A3B93B
:1025A00001681248114E0CF050F80546042D0CDC61
:1025B0003046D4F800800CF08EF841460246E060C8
:1025C00030460CF065F80135F0E7E26862B1137C43
:1025D00013F00F0106D1022161F303031374E368C2
:1025E0005F6101E00229FAD0BDE8F0816C070020AC
:1025F000006828B1007C00F00F00431F584258418A
:1026000070470000F8B50446FFF7F2FF002832D00B
:1026100021683748364F0CF018F80546032D266818
:1026200009DC38460CF057F83146024638460CF0C3
:102630002FF80135F2E7002231462D480CF00FF853
:1026400002F0B3FB01222074216829480CF007F83E
:1026500002226060216826480CF001F80422A06084
:10266000216823480BF0FBFFE060207C0C282CD075
:1026700002D803280ED0F8BD102830D01228FAD185
:102680000C200EF091F91B4B44600360054606F0E8
:10269000E1FB18E010200EF087F9174B03600546A8
:1026A000446000212046FFF789FE03B2002BB6BF2D
:1026B00040422B8128816868FFF7DEFE0F4B2B60BC
:1026C00000236881AB816561D5E714200EF06CF9B9
:1026D0000B4B44600360054606F02EF8F3E70EF05E
:1026E00063F9084B44600360054606F0DFFDEAE746
:1026F0006C0700207C910100D4790100CC9101008D
:10270000A09001006C92010010B500230446016006
:10271000436103768362FFF775FF204610BD00001A
:1027200070B5056806462F21284611F00FFC0446B7
:1027300098B1002300F8013BFFF76EFD0B490546F9
:102740000B480DF09FFA0A22294609480DF003FBB9
:1027500007480DF0A7FA284670BD2846FFF75CFD34
:1027600005460028F7D03460F5E700BF3D7B010047
:10277000680300202DE9F04389B0002400F1180817
:102780000546CDF804804461047684620E46002933
:102790003BD01F4B1F68002F37D02F21304611F040
:1027A0004BFB814650B3234602AAF05C19B238B104
:1027B0002F2805D0142B02D0D0540133F5E7194649
:1027C00008AB1944002301F8183C124839460BF0B5
:1027D00050FF0F22286009F10101404611F095FBDE
:1027E00001A8FFF79DFF019BA86203B92B7628463D
:1027F000FFF708FF284609B0BDE8F08332463946A6
:1028000004480BF036FF2860F1E700232B60EEE769
:10281000D40300206C07002008B543693BB9007C55
:10282000052809D014280CBF0020FF2008BD1A6815
:102830001846926B9047F3E75020F7E708B505225A
:10284000016805480BF00BFF20B1037C13F0F0008A
:1028500018BF180908BD00BF6C0700202DE9F74319
:102860006D4685E80600016881461F4619B90020BB
:1028700003B0BDE8F0833448DFF8CC800BF0E5FE10
:102880000446052CD9F8006009DC40460BF023FF14
:102890003146024640460BF0FBFE0134F1E70522CB
:1028A000314629480BF0DBFE04460028DFD02846DD
:1028B00002F062F90F28DAD8284601F0F9FF002863
:1028C00007DD237C13F00D0F10D003F00F03072B4F
:1028D0000CD0237C1D491E486FF3071323740DF0A1
:1028E000D1F91B480DF0DEF90120C1E70DF0C6FF5C
:1028F0000646284601F0DCFF002F237C0CBF022295
:10290000072262F30303304460612374284602F017
:1029100033F9237C0F4960F3071323740C480DF03F
:10292000B1F9284601F0C4FF0A22014608480DF01B
:10293000F0F9094906480DF0A5F90A226169044831
:102940000DF0E7F9CDE700BF6C070020997C01008E
:1029500068030020A37C0100AE7C0100F0B587B0C5
:102960006F4687E80600054697E8030002AC84E856
:10297000050038461E4602F0FFF801380C2838D80A
:10298000DFE800F0424B959E8C0739373754627E62
:1029900070004EBB0722214604A802F09CF9494969
:1029A00049480DF06FF9204602F0E6F80A22014688
:1029B00045480DF0E9F9454943480DF063F92046D3
:1029C00001F076FF0A2201463F480DF0A2F93E4889
:1029D0000DF068F99DF8303094E806002846FFF7BE
:1029E0003DFF012007B0F0BD2846FFF727FF002874
:1029F000D0D10020F6E70EB10622CCE72846FFF73B
:102A00001DFF0028F8D1F4E70EB90222C3E72846DB
:102A1000FFF714FF0028F8D1EBE70EB10122BAE767
:102A20002846FFF70BFF0028F8D1E2E74FF480318A
:102A30002846FFF753FC08B10B22ACE72846FFF706
:102A4000FDFE0028F8D1D4E74FF480312846FFF787
:102A500045FC08B90A229EE72846FFF7EFFE00284A
:102A6000F8D1C6E74FF400312846FFF737FC08B924
:102A70000C2290E72846FFF7E1FE0028F8D1B8E7DE
:102A80004FF400312846FFF729FC08B10D2282E7F8
:102A90002846FFF7D3FE0028F8D1AAE70EB103229B
:102AA00079E72846FFF7CAFE0028F8D1A1E70EB95A
:102AB000052270E72846FFF7C1FE0028F8D198E705
:102AC000042268E7C87C010068030020DC7C010068
:102AD00018B1034903480DF0D5B80349FAE700BF20
:102AE000497B0100680300204E7B01002DE9F04383
:102AF0009FB04FF0000802AC84E8060006461022A2
:102B000041460AA81D46269FCDF8248010F029FAD8
:102B10002046CDE906888DF8208002F07BFAEA0590
:102B20001AD5204602F028F8172800F2CE8001239B
:102B300003FA00F0974B18420AD1974B0340002B41
:102B400040F0C78010F0240F00F0BF80934900E0F0
:102B5000934906A811F087F992480CF0DBF8002899
:102B600000F0AB80904B93F900209846002A40F08B
:102B7000A480002F44D13B46032240210EA807F039
:102B80001FFA33683F2219680EA811F098F9AB05B7
:102B900040F1AE80204601F0EFFF022800F0A8804F
:102BA000204601F0E9FF052800F0A280204601F050
:102BB000E5FF012840F090804FF001094FF40073C9
:102BC000142209A9CDF80090204602F00FF94B46D7
:102BD00009AA0EA973480CF0FAFA744974480DF06A
:102BE00051F80EA972480DF056F8724970480DF070
:102BF00049F809A96E480DF04EF86D480DF052F8ED
:102C0000204601F01AFE05F4005908B1A90503D4C5
:102C1000B9F1000F00F09D800023032240210EA88F
:102C200007F0CEF933683F2219680EA811F047F972
:102C300047B161490EA811F0F0F83F2239460EA8BD
:102C400011F03DF95C490EA811F0E7F83F22B9F107
:102C5000000F67D059490EA811F031F9204601F054
:102C60008DFF043801285FD81722214604A802F0FE
:102C700032F8002300934FF44073142209A9204630
:102C800002F0B4F849494A480CF0FCFF0EA9484844
:102C90000DF001F8474946480CF0F4FF09A94448F3
:102CA0000CF0F9FF42480CF0FDFF3E480CF032F802
:102CB00018B198F90030002B40D030462946FFF774
:102CC00025FB00201FB0BDE8F0833D4938480CF0DB
:102CD000D9FF25F480753FE7204601F04FFF022819
:102CE0003FF46AAF204601F049FF08283FF464AF83
:102CF000E80585D59DF81830002B81D0012306AA60
:102D00000EA928480CF063FA284929480CF0BAFFAC
:102D10000EA927480CF0BFFF264925480CF0B2FF4A
:102D200006A967E7274996E70023B9F1000F00934A
:102D30000CBF4FF400734FF440739EE70EA90123BC
:102D400009AA18480CF043FA4FF400713046FFF717
:102D50001DFBEA0540F18480204601F00DFF01389B
:102D6000142835D8DFE810F0D900340034003400DE
:102D70003400D9003400340034003400340034000E
:102D80003400DD00D7003400340034003000D300BC
:102D9000D50000BF42C0380001008000657B010003
:102DA0005C7B0100E0030020B0030020C27C010036
:102DB00068030020AA7A010080870100487C010096
:102DC000B47C01003E7C01005C4906A811F04BF880
:102DD0000023032240210EA807F0F2F833683F22B7
:102DE00019680EA811F06BF847B155490EA811F0FB
:102DF00014F83F2239460EA811F061F850490EA888
:102E000011F00BF83F224F490EA811F058F84E4927
:102E10004E480CF037FF0EA94C480CF03CFF4C49D3
:102E20004A480CF02FFF06A948480CF034FF4748E9
:102E30000CF038FF47480BF06DFF00283FF43DAF22
:102E400098F90030002B7FF438AF0EA9012306AAB1
:102E500040480CF0BCF94FF480713046FFF796FA09
:102E60006B0552D54FF480313046FFF737FA002812
:102E700059D0394906A810F0F6FF0023032240215B
:102E80000EA807F09DF833683F2219680EA811F0CC
:102E900016F847B12A490EA810F0BFFF3F22394665
:102EA0000EA811F00CF826490EA810F0B6FF3F222C
:102EB0002A490EA811F003F8234924480CF0E2FE39
:102EC0000EA922480CF0E7FE214920480CF0DAFE5A
:102ED00006A91E480CF0DFFE1C480CF0E3FE1D485E
:102EE0000BF018FF00283FF4E8AE98F90030002BF3
:102EF0007FF4E3AE0EA9012306AA16480CF067F989
:102F00004FF480613046FFF741FA0120DAE61449B8
:102F10005BE7144959E7144957E7337C052B7FF4E5
:102F200057AF124951E74FF400313046FFF7D6F959
:102F300008B10F499EE70F499CE700BFFE7B0100E7
:102F400080870100397C0100C27C010068030020F9
:102F5000AA7A0100E0030020B67B0100617C010039
:102F6000077C0100107C0100DA7B0100D17B0100AD
:102F7000C87B0100AD7B0100F0B5CB070C4644BF18
:102F800021F4805424F0010414F4805785B00546E0
:102F90000CD004F4E0612846FFF7B8F9144915484D
:102FA0000CF070FE4FF0FF3005B0F0BD06F08EFF64
:102FB0009528EED902F0EEFD0028EAD002AE3A469E
:102FC0003946304601F0AAFA4FF44072294630469D
:102FD00001F096FE4FF4E0612846FFF77FF9009775
:102FE00044EA000396E806002846FFF77FFDDBE78A
:102FF0007A7C01006803002010B54FF4407104464C
:10300000FFF76CF9014670B1074B93F90030062BBE
:1030100009D12046FFF7B0FF20464FF44071BDE8CC
:103020001040FFF7B3B910BDD803002043691BB1AE
:103030001A681846926B1047007C70472DE9F04FD4
:1030400093B00DF1280809939DF8703003939DF813
:1030500074300493054688E8060006F037FFB0F5A3
:10306000966F04460EDAB549B5480CF00BFE0A22FD
:103070002146B3480CF06FFEB1480CF013FE4FF040
:10308000FF3896E30DF0FAFB0790404601F02AFE68
:103090008346064602F07EFD099B06901BB11A7816
:1030A000002A40F0D6852B7E13B105F11803099351
:1030B000002E40F0E785099B002B40F0CD85D5F828
:1030C00028B0BBF1000F00F0DD85404601F00AFE9C
:1030D000002840F0D7855FFA8BF2414610A801F036
:1030E00005FE00F0CFBD2B68002BC8D0BBF1040F4C
:1030F00007D1049B98E806002846FFF7AFFB8046FF
:1031000057E398E803000CAB83E80300404601F066
:1031100033FD092800F21B82DFE810F00A001902D3
:10312000190219026701190219021902A901A9015C
:1031300000220DF138091146484601F0EFF94046EA
:1031400001F07BFB0646002800F04981BBF10C0F23
:1031500017D8DFE81BF00D001600650016001600FA
:10316000160016001600160016001101FD002D01B4
:10317000099F57B1734974480CF084FD72480CF0F4
:1031800091FD0024A1462646F3E0284600F0C0FF4A
:103190000028D4BF002101210A2204466A480CF00D
:1031A000DAFD6A4968480CF076FD404601F080FB84
:1031B0000A22014664480CF0ACFD63480CF072FD35
:1031C000002C404640F33C8501F072FB68BB0222B4
:1031D000414610A801F07FFD40F20114012706E0EE
:1031E0000122414610A801F076FD40F201144FF48F
:1031F00000722946484602F0BDFA484601F0BEFC7E
:10320000042814D1404601F0B9FC022814D14046EC
:1032100001F0B4FC0EA9024610A801F0B2FC0BE0CC
:10322000002426464FF0FF37E1E73C46D6E7484604
:1032300001F0A4FC0528E5D02B7C072B08D14046E3
:1032400001F002FB20B102220EA910A801F099FCA6
:103250002846FFF7EBFE00B200900DF138090DF1A2
:10326000280810A898E80C00494601F04DFF484690
:1032700001F0D0FE3EB1404601F080FC02284DD165
:10328000484602F0A3FA99E8030088E8030044F4F2
:1032900090544FF000094FF0FF382B7C072B40F083
:1032A0004482039B63B36B681B7C03F00F03052B05
:1032B00040F05681069B002B00F04F81284600F01D
:1032C00027FF049B099A00280AA96868D4BF4FF019
:1032D00000084FF0010800F09FFEBBF1010F4FFA0C
:1032E00088F740F03D810AA801F0A7FA039038B1B1
:1032F000049B00930CAA434606CA2846FFF72EFB00
:103300000AA801F039FC0338042800F24F81DFE8F5
:1033100010F029014D01E80171015001404601F012
:103320002DFC0128ACD0404601F028FC0A28A7D08B
:10333000404601F023FC0B28A5D1A1E7E77C010062
:1033400084030020277D0100680300204C7B0100DE
:1033500029464FF40072484602F00CFA404601F04C
:10336000C5F9C1B2484601F069F998B9B1460026DD
:1033700034464FF0FF378EE729464FF40072484637
:1033800002F0F8F9404601F0AAF90146484601F07A
:103390003BF9EAE799E80300022288E803000026E7
:1033A000414610A801F0A2FC4FF49054B146E0E76A
:1033B0004FF400722946484602F0DCF9404601F01D
:1033C00074F90146484601F04AF999E803004FF0C4
:1033D000000988E803004FF490544E46C9E781463F
:1033E00004464FF0FF38474657E7BBF1090F20D09E
:1033F000284600F08DFE00280DDD4146022210A86F
:10340000012601F068FC40F201144FF0FF384FF044
:103410000009374641E74146012210A84FF0000954
:1034200001F059FC40F201144FF0FF3801264F46DD
:1034300033E74FF480312846FEF750FF06464FF43D
:10344000803128465EB1FEF7A1FF40F201444FF003
:1034500001084FF000094E464FF0FF371DE7FEF719
:1034600055FF40F201444FF00108B146F3E798E8F8
:1034700003000EAF87E80300404601F0DEF9E0B933
:103480000524404601F078FB4FF4007209282946D4
:10349000404608BF644202F06DF90022414610A880
:1034A00001F019FCBBF10B0F49D8DFE80BF0214804
:1034B0000D484848484848482343404601F0D0F961
:1034C00004460028DCD0DCE700262846FFF7A4F9F4
:1034D00021460246404601F00BF9044690BB97E8AE
:1034E000030088E803004FF001094FF0FF38B3E70D
:1034F0000126EAE72146404601F056F950B1022282
:10350000414610A84FF0000901F0F0FB4FF4905431
:103510004E46EAE797E8030088E80300A749A84871
:103520000CF0B0FBA6480CF0BDFB00244FF00109E5
:103530002646DAE72146404601F05BF9DEE7002443
:10354000A146F5E74FF490544FF00009CDE7002471
:103550004FF0FF38A146264645E7069B0393CFE68A
:103560000023FBE72846FEF77FFE0528074602D02A
:103570004FF003081DE1934993480CF083FB0A22A6
:10358000394691480CF0E7FB8F480CF08BFB4FF469
:10359000007229460AA802F0EDF801220AA910A833
:1035A00001F099FB44F4807444F001044FF0000AE8
:1035B00043E02846FEF758FE062807460DD183490A
:1035C00081480CF05FFB0A2239467F480CF0C3FBB0
:1035D0007D480CF067FB0222E0E77D497A480CF059
:1035E00051FB0A22394678480CF0B5FB76480CF0BE
:1035F00059FBBDE74FF480312846FEF76FFE0028E7
:103600006DD1781C06D1284600F082FD0028D4BF79
:1036100000270127002F5DD14FF4007229460AA828
:1036200002F0A8F801220AA910A801F054FB44F402
:10363000807444F001044FF0060A0AA801F0F1F882
:10364000002866D10AA844F0010401F0F6F8002829
:1036500062D044F40074039B13B124F40074A4B248
:10366000224629460AA802F029F84FF00108B9F1CC
:10367000000F40F037836869002840F0D7814FF48D
:1036800000312846FEF72AFE002800F0D881514973
:103690004B480CF0F7FA4A480CF004FB630500F1C4
:1036A000C2824D4948480CF0EDFA0A22414646488C
:1036B0000CF051FB494944480CF0E4FA0DF0DEF8F7
:1036C000079B0A22C11A40480CF051FB3E480CF0FF
:1036D000E9FA6EE042493C480CF0D4FA48E7414927
:1036E000F9E7791C06D1284600F012FD0028D4BF66
:1036F000002701275FB102220AA910A844F48074B0
:1037000001F0E9FA44F001044FF0050A95E7364963
:10371000E1E744F4807495E74FF4007229460AA863
:1037200001F0EEFA002894D195E77A1C06D12846DC
:1037300000F0EEFC0028D4BF00270127002F2B4902
:10374000214818BF01260CF09DFA0A2239461E486E
:103750000CF001FB26491C480CF094FA0A22314671
:1037600019480CF0F8FA18480CF09CFA099800284F
:1037700044D0FEF7FBFC08902846FEF775FD0FFAD3
:1037800080FA089BBAF1000F01D10FFA87FA002BDB
:103790005BD09A4530D017490B480CF073FA0A22D7
:1037A000514609480CF0D7FA07480CF07BFA6FF045
:1037B0000208404613B0BDE8F08F00BF3C7D010019
:1037C00084030020487D0100680300205D7D010026
:1037D000747D0100287E01007B7E0100867E010051
:1037E000927D0100AC7D0100C17D0100DE7D010004
:1037F000EC7D0100F37D010000230993BBF1010F73
:1038000030D1039B1BB10AA801F017F803900AA856
:1038100001F0B2F9152800F2F480DFE810F0B500ED
:10382000C800A5002600B500960074005000B50041
:10383000B500EF00EF0000010001DD00DD00F20047
:10384000F200F200DD00DD00DD0068690028D5D05F
:10385000049A0368CDE900620AAA9C6A099B06CA19
:10386000A0474CE400230393D1E72846FEF7FCFC75
:10387000052806467FF47CAE8A498B480CF002FA94
:103880000A22314688480CF066FA87480CF00AFA9A
:103890004FF4007229460AA801F06CFF2B7C052B1F
:1038A0000CBF0E2201220AA910A801F014FA44F458
:1038B000807444F001044FF0000A012666E02846B7
:1038C000FEF7D2FC0628064616D1784976480CF059
:1038D000D9F931460A2274480CF03DFA72480CF0CE
:1038E000E1F90AA910A8022201F0F5F94FF400212C
:1038F0002846FEF74BFDDAE76D496B480CF0C2F93C
:103900000A2231466FE64FF480312846FEF7E6FC86
:1039100000287FF4E4AE002F7FF4DCAE4FF4007299
:1039200029460AA801F026FF01220AA910A801F0E1
:10393000D2F944F480744FF400212846FEF7E6FCE7
:1039400044F001044FF0060AB7E7002F3FF4DFAE62
:1039500002220AA910A844F4807401F0BCF944F0D2
:1039600001044FF0050AA8E70AA800F05AFF06462E
:10397000002859D02846FEF777FC05283FF4F8AD1B
:1039800044F4807444F001044FF0000A039B002BC0
:103990003FF46DAE049B00930CAA07F0010306CA26
:1039A000284624F40074FEF7D9FFA4B25FE60AA803
:1039B00000F037FF00283FF47EAF6FB13D493A4831
:1039C0000CF060F928460121FEF75CFC4FF48851A9
:1039D0002846FFF7D1FACBE50AA800F022FF0646F9
:1039E00010B30AA800F029FF28B94FF40072294645
:1039F0000AA801F0BFFE44F44074C3E744F48064B5
:103A000059E70AA800F008FF08B144F480740AA836
:103A100000F013FF064638B144F40074B4E74FF0E9
:103A2000000A4FF4806448E7B24646E703680AAAF2
:103A30001B6B06CA984700287FF421AE27E66F6902
:103A4000002F39D00AAF24B122462946384601F06A
:103A500035FE049A68690368CDE900629E6A099B95
:103A600097E80600B0478046686903689B6B9847F3
:103A7000052808BF44F0010414F4806F18BF4FF00C
:103A80000108BAF1000F03D051462846FEF7FAFBB1
:103A9000069B002B3FF405AE21462846FFF76CFA43
:103AA000FFE500BF487D0100680300205D7D010047
:103AB000747D01000F7E01002B7C052B75D0062B39
:103AC000DFD10AA800F0A8FE00286ED039462846AB
:103AD000FEF774FC074606B20AA801F04DF8049BF5
:103AE0008146002B47D024B1224629460AA801F07E
:103AF000E5FD002EC5D0BCBF7E4236B206F1FF33D5
:103B00009BB2B4BF01270027192BBAD80121304638
:103B10000DF0A2F8B9F1150F09D8012303FA09F93C
:103B2000724B19EA030F35D119F0A40F3AD170493D
:103B300070480CF0A7F80A2231466E480CF00BF9D9
:103B40006D496C480CF09EF80A22059969480CF002
:103B500002F968480CF0A6F8304606F0BFFC28B120
:103B60002846FEF76BFE08B902F0A6FD44F4807407
:103B700044F0010451E0304606F0B0FC0028B2D019
:103B80005E495F480CF07EF85D480CF08BF86FF0F2
:103B900004080EE687F001030593194630460DF040
:103BA00083F8C4E705973946F8E724B12246294649
:103BB0000AA801F083FDBBF1020F31D0BBF1030F66
:103BC00009D0BBF1010F7FF45CAF44F4807444F082
:103BD0000104D84655E72846FEF7C4FC030C064608
:103BE00005D12B6847491A6847480BF0DBFA0AA849
:103BF00000F07EFE0EF06EFB0022444B0EF0C2FB86
:103C00000EF070FE60F30F06082006F04BFC60F328
:103C10001F4631462846FEF7BDFC4FF0010830E74D
:103C200044F40074A4E7069B002B3FF43AAD294608
:103C30004FF480620AA801F041FD4FF480612CE747
:103C400000F036FE00287FF4CBAA04460746FFF7B3
:103C5000CEBABBF1000F15D11B78002B3FF42FAA71
:103C600009A8FEF75DFD8346404601F03BF828B900
:103C70005FFA8BF2414610A801F038F8BBF1000F53
:103C80003FF41DAA22491B480BF0FCFF0A222146E3
:103C900018480CF060F81F4916480BF0F3FF2B682A
:103CA000144819680BF0F7FF1B4912480BF0EAFFA4
:103CB000099910480BF0EFFF18490E480BF0E2FF8E
:103CC000404601F0A7F9099B002B3FF40CAA1B7892
:103CD000242B7FF408AA124906480BF0D3FF0548AD
:103CE0000BF0E0FF6FF0030863E500BF42C0300057
:103CF000677E0100680300202B7B01005A7E0100D3
:103D0000840300206C7E0100E00300200000594085
:103D1000FB7C0100067D01000D7D01004C7B010054
:103D2000137D01002DE9F04F8FB08046CDE90221CF
:103D3000002900F0688106F0C9F8B0F5966F0446D6
:103D400010DAB249B2480BF09DFF0A222146B04872
:103D50000CF001F8AE480BF0A5FF4FF0FF300FB0AC
:103D6000BDE8F08F029B0BB11B782BB998F8183087
:103D700013B108F118030293029BE3B9D8F8286045
:103D800016BB4021039810F057F8002839D004469C
:103D9000002304F8013B0398214606F09DFB0394A1
:103DA00081460024039D2F5D6FB3384611F0A1F8C2
:103DB00028550134F6E71B78002BDFD002A8FEF768
:103DC000AFFC06460028D9D00D2EDAD108AC00226F
:103DD0001146204600F0A2FB039A21460AA800F0F3
:103DE0006EFF324621460AA800F080FF00230193AF
:103DF00001230093029B94E806004046FFF71EF95A
:103E0000ADE78146CDE7284600F03AFB04ACC2B2EC
:103E100005463946204600F081FB052E24D0062EAB
:103E200008BF17255FFA86FA0AAF52462146384680
:103E300000F05CFF092D19DC082D80F2D480AA1C4B
:103E400003DB6B1C40F3DF80D5B103A805F095FFC1
:103E5000024618B12146384600F0B1FE0123009316
:103E6000CDF804900023C6E71825DBE7172D00F0F6
:103E70008980182DE9D100222146384600F02BFF19
:103E800006AD03A9284605F099FF52462946384653
:103E900000F02CFF284600F071FE10F1000A18BF58
:103EA0004FF0010A4FF0000B039A0FFA8BF35AB14F
:103EB000BBF1030F07D003A805F05FFF47F82B0005
:103EC0000BF1010BF0E75B460B2E0DD00C2E13D03F
:103ED0000A2E19D1284600F0EBFC81B2204600F0F2
:103EE00093FBCDF8049083E7284600F0E1FCC1B2D3
:103EF000204600F0A3FBF4E7284600F0D9FC014679
:103F0000204600F0ACFBECE753449BB2013B032B93
:103F100030D8DFE803F00207122095E8030084E8B8
:103F20000300DEE7284600F0C3FC9DF8283082B28B
:103F3000214608A800F08CFED3E7284600F0B8FC24
:103F40009DF82C2000929DF8283082B2214608A8C6
:103F500000F067FEC5E7284600F0AAFC9DF82C207B
:103F60000092214682B29DF8283008A800F059FE40
:103F70000C99C5E7274926480BF084FE24480BF02E
:103F800091FEAEE700222146384600F0A4FE00254F
:103F9000039A2BB242B1042D0AD003A805F0EDFE1E
:103FA00047F825000135F3E7032B10D0042B98D1F7
:103FB0009DF8341001919DF8301000919DF82C303F
:103FC0009DF82820214608A800F066FE89E79DF8A4
:103FD000301000919DF82C309DF82820214608A82B
:103FE00000F04AFE7DE708AC03A9204605F0E6FE96
:103FF000EAB22146384600F06EFE52462146384667
:1040000000F074FE6DE70020A9E600BF8D7E010080
:1040100084030020A57E01002DE9F04F0E468FB0ED
:1040200091469A46002856D0037C03F00F03052BD7
:1040300065D1344DC4682B78DFF8CCB0DFF8CC8084
:1040400001332B70002C57D0237C03F00F03042B7B
:1040500050D16269DBF8001040460AF00AFB0746BF
:10406000002847D0037C03F00F03052B42D1014603
:1040700003A8FEF749FB6EB103A8FEF7B9FA48B1F1
:1040800000230093CDF804A04B463168726803A862
:10409000FEF7D4FF0022394640460AF0E0FAE8B1C4
:1040A000037C03F00F03022B18D14369072B15D1B2
:1040B0000122394640460AF0D2FA53464A46314672
:1040C000FFF7AAFF9EB990B12B7803A8013B2B7094
:1040D000FEF7C0F801200FB0BDE8F08F3EB903A88D
:1040E000FEF786FA18B103A800F012F8EBE703A870
:1040F000FEF7B0F86468A5E72B78013B2B70002031
:10410000E9E700BF65030020D40300206C0700200E
:1041100073B5002205461146684600F0FFF92B688A
:10412000464819680BF0B7FD454944480BF0AAFD15
:104130002846FEF75DFA58B9424940480BF0A2FD07
:104140003E480BF0AFFD4FF0FF34204602B070BD8B
:104150002846FEF789F80646686958B10368DB6AA5
:10416000984704B2002C05DB14BF01200020FEF7A5
:10417000AFFCEAE72B7C072B13D0701C152810D856
:104180000126314C06FA00F0044004D110F0490F2A
:1041900007D02046EBE72D4928480BF073FD344645
:1041A000D3E74FF400722946684600F0A9FD2B7C46
:1041B000033B062B3AD8DFE803F0352039390435C4
:1041C00020006B681B7C03F00F03052B34D12049C2
:1041D0001A480BF057FD002319461A466868FFF786
:1041E0001BFF1C49044615480BF04CFD2046FEF70A
:1041F0006FFC12480BF056FDA7E70021684600F05F
:104200004FFC044614490D480BF03CFD21460A22A0
:104210000A480BF0A0FD09480BF044FD003418BF1C
:10422000012492E7684600F043FBEAE70B490348A4
:104230000BF028FD002488E70024E3E76803002052
:104240004C7B0100E27E010084803000497B01004C
:10425000E2820100EB7E0100F87E0100EE7E0100AB
:10426000F0B54FF4006185B00546FEF737F8002839
:1042700047D0002202AC1146204600F04FF94FF41F
:1042800040722946204600F03BFD6B69002B38D078
:104290004FF400612846FEF779F81B491B480BF0E4
:1042A000F1FC6869002301260268CDE90063976A82
:1042B00094E80600B847431C044622D02B681348F4
:1042C00019687CB90BF0E7FC114910480BF0DAFCD7
:1042D00010490E480BF0D6FC0C480BF0E3FC2046CE
:1042E00005B0F0BD0BF0D7FC094908480BF0CAFC3B
:1042F000094906480BF0C6FC04480BF0D3FC3446D1
:10430000EDE70224EBE700BF8B7C0100680300208F
:10431000B27C0100CB880100EB8101002DE9F04F58
:10432000044689B08946FFF79BFF0522216847486C
:104330000AF095F90646002872D0037C03934FEAF1
:10434000131A45690CF09AFABAF1000F68D0A5EB80
:10435000000804AD52460B21284606AF00F0DEF8F7
:1043600042462946384600F02AFCB9F1040F17D11D
:104370000023009395E806004FF400532046FEF713
:10438000B5FB0A224FF47A71314898FBF1F10BF03A
:10439000C0FC30492E480BF075FC2D480BF082FC18
:1043A000B8F1000F3CDA2C4B984539DB05F08EFD57
:1043B0004FF00008CDF8008083464FF4005395E895
:1043C00006002046FEF792FBBBF5966F10DA2349F4
:1043D00023480BF057FC0A22594621480BF0BBFC3E
:1043E0001F480BF05FFC4FF0FF3009B0BDE8F08FC5
:1043F000337C68F30713337452464146384600F065
:104400008DF8039B03F00F03DA1F534253410193CE
:104410000123009397E8060043462046FEF70EFE70
:10442000B9F1010F02D12046FEF7E6FD606908B937
:104430000020DAE703685B6998470028F8D06069D4
:1044400003680FFA89F19B689847CEE76C07002054
:1044500068030020B27E010002000080C17E0100DE
:104460008403002007B5002300931A461946034829
:104470000BF0C0FB03B05DF804FB00BF300300206D
:10448000F8B50646F0B10378E3B12D2B1ED0A3F1A9
:104490003002092A1AD9252B1AD07B2B1AD0232BAC
:1044A0001BD00F4F012404EBC4053D4428460FF0F8
:1044B000FEFC2946024630460FF015FD20B10134BE
:1044C000192CF0D14FF0FF342046F8BD0024FBE753
:1044D0000824F9E76FF00104F6E71724F4E700BFBA
:1044E000157F0100F8B5064690B1037883B10A4FF5
:1044F000002404EBC4053D4428460FF0D8FC2946AF
:10450000024630460FF0EFFC20B10134172CF0D1F9
:104510004FF0FF342046F8BDF67F010010B50023B0
:104520008370C370037143718371C37161F30713A7
:104530004370027010BD10B5002307240370837010
:10454000C37064F307134370416010BD93B2112B25
:1045500070B516469CBF134AD25C4B7888BF0022C8
:1045600062F307134B7005460C460F480F490BF0DA
:1045700089FB0A2231460C480BF0EDFB0C490A4836
:104580000BF080FB617808480A2209090BF0FCFB5C
:1045900005480BF087FB23682B6063686B60284637
:1045A00070BD00BF037F0100680300203B81010054
:1045B000468101004B781B09013B082B1AD8DFE824
:1045C00003F0160E0E19191919050C000C4B4B604F
:1045D0000B6803604B68436070470A4BF7E764233E
:1045E0008B71CB7923F00103CB7100234B71FF2337
:1045F0000B71EDE700230B714B718B71CB71E7E70A
:104600000000A0410000964243781A0903D0022A14
:1046100005D000207047022262F30713437040F276
:104620006D139942A8BF1946C379817123F0010324
:10463000C1F300211943C1710120704743781A0961
:1046400003D0022A05D000207047022262F307132C
:1046500043706429A8BF642141710120704713B5DC
:104660000446084631B9E37960F34703E37101205A
:1046700002B010BD642300934FF4FA720023992115
:104680000BF087FF63781A0908D0032A0BD820EAB9
:10469000E0706428A8BF64200130E4E7022262F3DE
:1046A00007136370F3E70020E2E707B5C27912F061
:1046B000FE0F11D043781B09013B022B0CD8500888
:1046C0004FF4FA73009364229923002101380BF010
:1046D00060FF03B05DF804FB4FF0FF30F9E7C379EA
:1046E000827903F0010342EA032070474079704762
:1046F00043781B09013B10B50A2B53D8DFE803F0C0
:104700000606525252482F2F2F10100002796423B0
:1047100091FBF3F1114481F308010171012010BDF7
:10472000632944684FF064030FDC03FB04112AB1D2
:1047300053439942A8BF194621EAE1714378416089
:10474000062262F307134370E8E791FBF3F121447B
:10475000E2B19142A8BF114621EAE17116E0436837
:1047600007EE903AFDEEE77A642417EE903A91FB5B
:10477000F4F1194422B19142A8BF114621EAE17136
:1047800007EE901AF8EEE77A17EE901A4160C5E747
:1047900043681944002AF9D0642353439942A8BFBF
:1047A0001946D9E70020BAE743781B09022B1ED12E
:1047B000C279837902F0010243EA0223642291FB69
:1047C000F2F11944B1F5B77F0FDA40F26D1331EA17
:1047D000210128BF1946C379817123F00103C1F378
:1047E00000211943C171012070470021F3E7002027
:1047F000704743781B09022B0CD14379642291FB4B
:10480000F2F1194421EAE1719142A8BF11464171C8
:1048100001207047002070470078003018BF012049
:104820007047437803F00F03012B04D80078003061
:1048300018BF0120704700207047437813F0F00F35
:1048400014BF012000207047407800F0E0002028CD
:1048500004D0A0F1400358425841704701207047EE
:1048600043781B09013B0A2B1ED8DFE803F00A0A34
:104870001D06061B0F0F0F060600436864205843F1
:1048800070470079642310FB03F0704743689FED85
:10489000077A07EE903A67EE877AFDEEE77A17EE31
:1048A000900A704740687047002070470000C84277
:1048B00043781B09013B0A2B18D8DFE803F00808EE
:1048C000170606120A0A0A060600406870470079B1
:1048D0007047406807EE900AFDEEE77A17EE900AFF
:1048E00070474068642390FBF3F0704700207047E6
:1048F00043781B09013B0A2B1ED8DFE803F0131392
:104900001D06060E191919060600436807EE903AAF
:10491000F8EEE77A17EE900A70474368642293FB3B
:10492000F2F3F3E7037907EE903AF8EE677AF1E7EE
:10493000436807EE903AEDE7DFED017AEAE700BF62
:104940000000000043781B0907B50B2B60D8DFE897
:1049500003F06216165F5F5F44245F5F06064068DF
:1049600049B1D0F1640056D46428A8BF642000B2D5
:1049700003B05DF804FB0028F6DA0846F8E7007992
:1049800031B1002100916423FF220BF002FEEEE71B
:1049900064230093FF220B46F7E7436807EE903A43
:1049A00099B19FED1F7A77EE677AF5EEC07AF1EE56
:1049B00010FA30D4F4EEC77AF1EE10FA2DDCFDEEE9
:1049C000E77A17EE903A18B2D2E7F5EEC07AF1EE38
:1049D00010FAD2D49FED127AECE7436861B142F24B
:1049E0007372934217DC13F1630F16DB6FF06300F1
:1049F00093FBF0F06430BAE713F1630FBDDB42F2D2
:104A0000737293424FF06400B2DC93FBF0F0AEE7B8
:104A10004FF0FF30ACE70020AAE76420A8E700BF12
:104A20000000C84213B50446084663781B09013BE1
:104A30000A2B32D8DFE803F00F0F313131281A3159
:104A400031060600FF2300930023642219460BF071
:104A5000A0FD606007E0FF23009300236422194655
:104A60000BF097FD2071012002B010BDFF230093D1
:104A70000023642219460BF08CFD07EE900AF8EE35
:104A8000E77A17EE900AE4E746F29C33009300239E
:104A9000642219460BF07DFD60600020E4E7000011
:104AA00043781B090B2B5FD8DFE803F06117175E13
:104AB0005E5E461E5E5E0606406841B1002839DB38
:104AC000FF28A8BFFF20C0F1FF0001B20AE00028C4
:104AD00008DBFF28A8BFFF20F7E700790029F4D002
:104AE000C0F1FF01084670474368A9B107EE103ACC
:104AF000B5EEC07AF1EE10FA1CD4DFED1E7AB4EEFA
:104B0000E77AF1EE10FA32DC77EEC77AFDEEE77A5B
:104B100017EE903A19B2E5E707EE903AF5EEC07A53
:104B2000F1EE10FADED49FED137AF4EEC77AF1EECF
:104B300010FAEBDDFF21D5E7406859B110F1630FA2
:104B4000F8DBB0F5C84F12DA6FF0630190FBF1F0BB
:104B5000FF30BAE710F1630FC4DBB0F5C84FE9DAF4
:104B6000642190FBF1F0B0E74FF0FF31BAE700218C
:104B7000B8E700BF00007F43007870474078000925
:104B800070474B7810B562F307134B700B680360E6
:104B90004B68436010BD4B7810B51C09013C012CDB
:104BA00084BF012464F3071382F30802D2B288BFE2
:104BB0004B700B680A7103604B68436010BD4B7803
:104BC0004A6030B50A2565F307134B700B68036024
:104BD0004B68436030BD4B784A6030B5072565F3BC
:104BE00007134B700B6803604B68436030BD4B7814
:104BF00030B5062565F307134B700A235A434A6004
:104C00000B6803604B68436030BD4B784A6030B539
:104C1000062565F307134B700B6803604B68436010
:104C200030BD70B54C788A71022666F307144C705B
:104C3000C2F30024CA794B7122F001029DF81030B2
:104C40000B7122430B68CA7103604B68436070BDEF
:104C500070B54C788A71032666F307144C70C2F362
:104C60000024CA794B7122F0010222430B68CA71F9
:104C700003604B68436070BD70B54D784B7104267E
:104C800066F307159DF810304D700B718A710B6833
:104C900003604B68436070BD70B54D784B7105265D
:104CA0009DF810300B7166F307159DF814304D70A8
:104CB000CB718A710B6803604B68436070BD4B78A1
:104CC0004A6030B50C2565F307134B700B68036021
:104CD0004B68436030BD10B50A700B6803604B68C9
:104CE000436010BD407800F00F0070474B7810B55E
:104CF00062F303034B700B6803604B68436010BDA5
:104D00002DE9F041044616460D4619B900273846EC
:104D1000BDE8F0810846FDF76BFC07460028F5D09A
:104D20002846FDF7BFFBF305804603D52846FDF76F
:104D30009BFA207006F40076B8F1000F09D0637872
:104D400068F307136370002EE1D0AB685B696360A2
:104D5000DDE7002EDAD0AA68137C03F00F03022BE4
:104D600003D0032B09D04746D1E7637852696260CC
:104D70000A2161F307136370C9E753696278072159
:104D800061F307126270E2E710B500230446037076
:104D900043708370C370037143718371C3714FF4A7
:104DA0000072FFF7ADFF204610BD70B50446C8B1D4
:104DB000037C03F00F03042B10D146693046FFF744
:104DC00091FB051E0EDB304609F048FD237C656132
:104DD000022262F303032374284670BD022B01D123
:104DE0004569F9E74FF0FF35F6E700002DE9F0439C
:104DF0002DED028B85B00446154699469DF8388006
:104E00000F46002948D0002A00F0E78000230B70ED
:104E1000017871B319F4807F2BD0714B01EBC10184
:104E2000194438460FF071F8637813F0F00F07D08B
:104E300019F4007F04D02A466A4938460FF03FF83B
:104E400038460FF034F82D1A3E18013D637813F000
:104E5000F00F21D019F4007F1ED01B09013B0B2B52
:104E60001AD8DFE803F0084071A6AC257B7B7B22D3
:104E70001FB43E46EAE72079B8F1000F06D064235C
:104E800000930023FF2219460BF083FB564A03468A
:104E9000294630460EF000FF384605B0BDEC028BC7
:104EA000BDE8F0836368514AF2E76368504AEFE770
:104EB000616800294FF064020EDA91FBF2F04B4278
:104EC00002FB1011494293FBF2F34A4A0091294632
:104ED00030460EF0E1FEDFE791FBF2F302FB131226
:104EE0000092454AF3E72046FFF7DFFBE279A3791A
:104EF00094F8059001B20029207902F0010202DB4A
:104F0000B8F1000F14D043EA0224B8F1000F06D024
:104F1000642300930023FF2219460BF03AFBCDE9EE
:104F200000902346354A294630460EF0B5FEB3E7D9
:104F3000CDE90101CDF8009043EA0223304A294629
:104F400030460EF0A9FEA7E7E379A27961790091D6
:104F500003F0010342EA03232A4AB8E7636808EE34
:104F6000103AB5EEC08AF1EE10FA4CBFF1EE487A75
:104F7000F0EE487AFDEEE78AB8EEE87A77EEC77A87
:104F80009FED217A67EE877A17EE900A0BF052FFB9
:104F900007EE900AB5EEC08AFDEEE77AF1EE10FA60
:104FA000CDED007A18EE903A01D5184A8FE7184AED
:104FB0008DE72279A379019262790092B2E7E279D2
:104FC000A37902922279019262790092B6E72A4689
:104FD000616830460EF099FF5EE717465CE700BF58
:104FE000157F01004C7B01005C8101005F810100A5
:104FF0006381010067810100688101007481010003
:10500000718101007781010000007A447D810100F7
:105010007E81010030B58BB0134C00232022009319
:1050200002A94FF440730546FFF7E0FE02A92046AF
:105030000AF031FE0D4920460AF024FE69780A2262
:10504000090920460AF0A0FE094920460AF01AFE86
:1050500069780A2201F00F0120460AF095FE2046E9
:105060000AF020FE0BB030BD68030020498101002A
:105070004E81010070B54B78B2EB131F86B0054628
:105080000C46164606D123682B6063686B60284681
:1050900006B070BD184919480AF0F4FD6178174848
:1050A0000A2209090AF070FE154914480AF0EAFDBF
:1050B0000A22314611480AF067FE12490F480AF0E9
:1050C000E1FD0023CDE9043366F3071322788DF860
:1050D00011304FF0FF338DF81020009302A8636861
:1050E000226804A900F010F8029B2360039B636010
:1050F0002046FFF78FFFC6E7868101006803002086
:10510000AA7A01004C7B01002DE9F04F8DB004AD6F
:1051100085E80C00BDF85830112B98BFB64A804680
:1051200028460C4694BF12F803904FF00009FFF791
:10513000BCFA011E02DB2046FFF791FA9DF8113000
:105140006278C3F3030161F3030262709DF81010EB
:105150002170C2F303120B2A38D8DFE812F0A00046
:105160000C000C00C9002F010D01A800CF00CF00DA
:10517000CF00A800A8001B090C2B77D8DFE803F0AC
:10518000265244180A073955767630306E009DF85D
:105190001720E2719DF81620A2719DF8152062710A
:1051A0009DF814202271627863F3071262700DE09B
:1051B000BDF81630C3F30802E379A27123F00103AE
:1051C00043EA1223E3719DF815306371B9F1000FC2
:1051D00000F0FC804A46214606A8FFF74BFFF5E0A9
:1051E000059B002B36DBFF2BA8BFFF23DBB223710F
:1051F000ECE7059B13F1630F2CDBB3F5C84F2BDAFB
:10520000642293FBF2F3F1E7BDF81630C3F3080212
:10521000E379A27123F0010343EA1223E3719DF8BD
:10522000153063719DF81430E1E7DDED057AF5EE98
:10523000C07AF1EE10FA0DD49FED707AF4EEC77AD1
:10524000F1EE10FA08DCFCEEE77ACDED027A9DF87B
:105250000830CCE70023CAE7FF23C8E763780C22B5
:1052600062F307136370059B6360AFE764496548A9
:105270000AF008FD9DF8111062480A2209090AF097
:1052800083FD61495F480AF0FDFC61785D480A22B0
:1052900009090AF079FD5B480AF004FD96E7627897
:1052A0001B0963F307120598627060608EE71B09A3
:1052B000032B04D00C2BD1D0059A626073E7002138
:1052C0002046FFF7EDFBBDF816302071C3F308024E
:1052D000E379A27123F0010343EA1223E3719DF8FD
:1052E000153063716378022262F3071363706DE710
:1052F00000212846FFF7D4FB2071F3E71B090C2B94
:10530000B4D801A252F823F0CD5100004753000059
:1053100075530000BF520000755300007553000024
:105320003D530000695300006953000069530000B9
:1053300055530000635300005D520000059B6360FD
:1053400006226378D0E79DF8143007EE903AF8EE25
:10535000677A03E0DDED057AF8EEE77A17EE903A2A
:1053600082E7DDED057AF2E7627863F30712627097
:10537000059B79E7627894E701271B090C2B3FF620
:1053800075AF01A252F823F0CD510000E1530000A7
:1053900035540000E1530000C1530000C153000028
:1053A000E1530000E15300006D5200006D52000017
:1053B000E1530000E15300005D5200000027DCE7EC
:1053C000059A6260627863F3071262702368C8F816
:1053D00000306368C8F8043040460DB0BDE8F08F77
:1053E000013B0A2B00F2CD80DFE803F0BACB10CBF3
:1053F000CBBFC4CBCBBDBD00037F010000007F430A
:10540000C580010068030020AA7A0100FF23BDF8CF
:1054100016208DF81430642161F30802ADF81620CF
:1054200000228DF815209DF81120022161F307124A
:105430008DF811200023FF259DF8150000956422AA
:1054400019460BF0A6F80028C0F29D8000239DF8B5
:1054500015000095642219460BF09BF8A84208DC61
:10546000002300959DF81500642219460BF091F871
:1054700005469DF81400FAF7FDFF0646002F47D0B9
:105480009DF817707F08013F3FB27B1C40F0888079
:105490007F2D4FF0FF0778DC0023C5F17F00194610
:1054A00047F68162704300970BF073F84FF4FF7377
:1054B000009300231946E0717F2228460BF069F81B
:1054C0000023194600903A4630460BF062F80097E8
:1054D0000646642328467F2200210BF05AF8BE427C
:1054E0000546A8BF3E466B496B480AF0CBFB0A2233
:1054F000294669480AF02FFC684967480AF0C2FB50
:105500000A22314664480AF026FC63480AF0CAFBC6
:1055100000231A46194606A80AF02CFABDF8160010
:105520004FF6FF7300930023194640F26D12C0F34B
:1055300008000BF02EF8F2B2E9B280B20AF030FAAD
:10554000030CA371030A63712071554952480AF094
:1055500099FB2046FFF75EFD06A80AF0A0F935E6A4
:105560009DF8143053E7059B51E7059B642293FB9C
:10557000F2F34CE7DDED057AFDEEE77A17EE903AAF
:1055800045E7002343E7002573E764232846009797
:105590003A4680210AF0FDFF00230546E371A2E7A9
:1055A0004FF01E0B64231A46CDF800B00021384698
:1055B0000AF0EFFF4FF0640A03905B463846CDF8DF
:1055C00000A0524600210AF0E4FF7F2D83464FF0F1
:1055D000FF0754DCC5F17F00002370431946314AB0
:1055E00000970BFB00F00AF0D4FF4FF4FF73E0715B
:1055F0000398009300231946E32228180AF0C9FFF4
:1056000000231946029000903A4630460AF0C1FF46
:1056100000230646009728467F2219460AF0B9FF64
:10562000BE420546A8BF3E461F491B480AF02AFB5A
:105630000A22039918480AF06CFB1C4916480AF024
:1056400021FB0A22594614480AF063FB1849124804
:105650000AF018FB0A2229460F480AF07CFB15497C
:105660000D480AF00FFB0A2231460B480AF073FB83
:10567000114909480AF006FB0A22029942E75346FB
:10568000284600973A4680210AF083FF002305460A
:10569000E371C9E7D780010068030020E4800100BE
:1056A00017810100646A3100F2800100F880010076
:1056B000FE800100068101000E810100F8B505465B
:1056C00017460C4611B900263046F8BD0846FCF7CF
:1056D0008FFF06460028F6D079050CD52B780A3BBB
:1056E000032B08D8DFE803F01F02242A4FF480318F
:1056F0002046FCF70BFEFA0507D52978A1F10A032D
:10570000032B02D92046FCF7BDFDBB051BD56B78EA
:1057100069681B09073B2046042B1FD8DFE803F00C
:1057200011111E1B1B004FF480312046FCF72EFE8A
:105730004FF400312046FCF729FEDCE74FF400313E
:10574000D6E7FCF7E5FE094909480AF09BFA284626
:10575000FFF760FCB8E7FCF7BFFEF4E7FCF7BCFE20
:10576000697820460909FCF7EFFEECE75581010056
:105770006803002073B504460D46FFF7C1FA0646DC
:10578000E8B9104910480AF07DFA2846FDF74EFCAA
:10579000214602B26846FEF7D9FE21466846FEF76A
:1057A00009FF29464FF400722046FFF787FF204685
:1057B000FFF730FC4FF490512846FDF7DDFB3046F3
:1057C00002B070BD1E8101006803002043781B09F0
:1057D000013B012B37B5054620D80023FF24007973
:1057E0000094642219460AF0D4FE002814DB00233A
:1057F00028790094642219460AF0CBFEA04207DC07
:10580000002300942879642219460AF0C2FEC4B22B
:105810002C71012003B030BD0024F9E70020F9E726
:1058200007B5002300931A46194603480AF0E2F927
:1058300003B05DF804FB00BF3803002002F07CBD1C
:1058400002F03CBD07B5002300931A4619460348F1
:105850000AF0D0F903B05DF804FB00BF400300205C
:10586000024B0F221A70C820704700BFD8030020D7
:1058700008B5044904480AF005FA04F025FC4FF481
:10588000FA7008BDE0860100B403002038B5094D68
:1058900001244FF47A700BF025F8214601340A22D6
:1058A0002846E4B20AF070FA142CF2D14FF4FA70E0
:1058B00038BD00BFB403002008B503F0C7FFC820FF
:1058C00008BD10B5044604300AF06DFE204610BD38
:1058D0000128F8B507460C46174E184D13DD4868E9
:1058E0000DF0B9F8C1B216483170FBF7CEF9022FAE
:1058F00007D0A0680DF0AFF8C1B211482970FBF7CE
:10590000D5F9C82401E04FF4C8740E490E480AF0D6
:10591000B9F90A2231780C480AF036FA0B490A48DC
:105920000AF0B0F90A22297807480AF02DFA064849
:105930000AF0B8F92046F8BD050000200600002056
:105940003C04002075880100B40300208988010010
:1059500030B587B00023044600931A460D4602A8CE
:1059600019460AF047F904A80AF03CF9042C12DDA4
:1059700004A9286904F0B2FA68B104A92548FBF724
:105980006CF804A9E86804F0A9FA50B104A9214808
:10599000FBF7AFF80BE002A91E48FBF75EF8032CFB
:1059A000EFDC02A91B48FBF7A4F8022C1CDD04A9BC
:1059B000A86804F093FAB8B104A91648FBF773F885
:1059C00004A9686804F08AFAA0B104A91148FBF799
:1059D0001EF8114911480AF055F900210D48FBF74E
:1059E00024F9C82007B030BD02A90A48FBF75BF8CC
:1059F000012CE5DC02A90748FBF709F8012CE8D1E6
:105A000002A90448FBF703F8054904480AF03AF9EB
:105A1000DFE700BF3C04002042830100B403002004
:105A20003283010008B548B149680548FAF774FEA9
:105A3000044905480AF026F9C82008BD0146F4E7E4
:105A40003C040020A4830100B403002008B548B141
:105A500049680548FAF78BFE044905480AF012F92F
:105A6000C82008BD0146F4E73C040020CA860100B6
:105A7000B403002030B5144D144C85B077220121B9
:105A80002846FBF73DFB00230193114B009311497E
:105A900002954FF0FF33204603930AF0F3F80E4BC4
:105AA0000E4819686A4608F0A9FD2846FBF7D4FAA3
:105AB0000B4920460AF0E6F820460AF0F3F80948B8
:105AC000FBF7DEF905B030BD54040020B40300201C
:105AD000E097010029860100300400206C070020B7
:105AE000438601003C040020012810B50C4622DD4D
:105AF000124960680EF073F918B901211048FBF7DC
:105B000079F8104960680EF06AF9014610B90C483E
:105B1000FBF770F80C490D480AF0B4F80848FBF799
:105B200060F80A22014609480AF015F907480AF008
:105B3000B9F8C82010BDFFF79DFFFAE7738E01008A
:105B40003C0400207C8E010053860100B403002039
:105B500010B50C48FBF74EF918B10B490B480AF089
:105B600091F80B4C722201212046FBF7C9FA237DE4
:105B70001BB1FF212046FBF761FA0548FBF76CFAE1
:105B8000C82010BD3C040020DF890100B4030020C0
:105B900054040020034B93F90000053818BF01207E
:105BA000704700BFD803002030B593B000230A46E9
:105BB0000546402101A804F003FA01A80EF077F988
:105BC00001A90446024628460EF08DF900280CBFB4
:105BD0002046002013B030BDF0B504469DB00E46FF
:105BE00001B18AB96A496B480AF04CF86A496948B8
:105BF0000AF048F8214667480AF04DF867496548B9
:105C00000AF040F8634821E000258D5404F05EF965
:105C10005F4907465F480AF035F80A2239465D4871
:105C20000AF099F85E495B480AF02CF82146594879
:105C30000AF031F85B4957480AF024F8B7F59D7F20
:105C400008DA594959480AF01DF858480AF02AF864
:105C50001DB0F0BD04215648564F03F035FF56499C
:105C60004C480AF00FF831464A480AF014F85249F5
:105C700048480AF007F847480AF014F83C22294639
:105C80000DA80C950DF06DF997F90020052A27D184
:105C900003212046FFF788FF05B26DBB474DEB6837
:105CA0001B78DB07D4D501212046FFF77DFF00B22A
:105CB0000028CDD0242120460EF048F90028C7D175
:105CC0003F49344809F0DEFF2146324809F0E3FF3E
:105CD000304809F0E7FF2146284609F004FAB7E703
:105CE00001212046FFF760FF05B2C5B90221204619
:105CF000FFF75AFF05B2C5B12544324928460EF0D8
:105D0000A8F8A0B930460EF0D2F801280FD92146E4
:105D10002A4809F0E8F9304608F0C8FD98E73F2224
:105D200021460CA80EF0F1F8E6E7274967E7204680
:105D300024210EF00BF90446002889D1294601A838
:105D4000FCF718FD01A8FCF753FCE0B122463146F0
:105D500001A8FDF7E7FF002815DD9DF8303093B16D
:105D600097F90030052B0ED018490A4809F08AFF30
:105D70000CA9084809F08FFF064809F093FF0CA909
:105D80000E4809F0B0F901A8FCF764FA60E700BF1B
:105D90000198010068030020DB820100409D0100A2
:105DA000E4820100E7820100EA820100840300200E
:105DB00034040020D8030020247A0100E0030020EE
:105DC000F7820100618E01000F8301001A83010038
:105DD0002DE9F04116491748174E184F154D09F097
:105DE00051FF0024A6F10F0816F8013F0F2B03D82E
:105DF0003946284609F04FFF052C4FF010020DD010
:105E00003178284609F085FF0D49284609F03AFF08
:105E10000134E4B2062CE7D1BDE8F08198F8151002
:105E2000284609F076FF284609F03CFFF0E700BF5E
:105E300064860100B40300204B040020C4970100D5
:105E4000B27C010010B58AB00DF11F0304930DF16F
:105E50002503039309AB0C4602930DF12303019331
:105E60000DF12203009308AA0DF121030E49606889
:105E70000DF046FF05280BDC0C490D4809F002FF28
:105E800061680B4809F007FF4FF4C8700AB010BDF5
:105E900008A90848FAF7F3FBFFF79AFF06490748F5
:105EA00009F0F0FEC820F1E7F28601000687010044
:105EB000840300203C04002018870100B403002064
:105EC00008B508B9002008BD037C03F00F03052BBB
:105ED000F8D1CAB20146064808F0C1FB0028F1D04B
:105EE000037C03F00F03042BECD14069EBE700BF08
:105EF0006C070020F7B53C4C2678002E6CD13B4B4C
:105F000093F90030012B67DD394B1968002963D004
:105F1000384A394808F0ADFB054600285CD00146F8
:105F2000354808F092FB07B2002F55D0314628467D
:105F3000FFF7C6FF012F064650D0294601222E4802
:105F400008F08DFB4569684605F0B2FA10222B492E
:105F5000684603F0E9FF2A492A4809F093FE3146D2
:105F6000284809F098FE2849264809F094FE0A229C
:105F70002946244809F0EFFE2349224809F08BFE08
:105F80001E49204809F087FE1E4809F08BFE40F2AA
:105F900002211E4805F024FDAAB231461C481D4DC1
:105FA00009F06EFD15491A4809F06EFD1A4B186884
:105FB00018B10021FFF784FF2860296889B11448CF
:105FC00009F06AFD0021124809F06EFD0123134912
:105FD0000C48237009F056FE03B0F0BD40F20225D4
:105FE000B1E70F49EBE700BF78040020D803002099
:105FF00030040020968201006C070020540300202A
:106000009D820100B4030020B27C0100C004002086
:106010009C04002080030020DC030020AC820100EF
:10602000019001002DE9F04FA7B0002396488DF8AC
:106030001330CDE90533CDE9073308F06BFE934FFC
:10604000054610B105233B70F8E0914C216841B939
:106050009049914809F016FE8F4809F023FE0F235E
:10606000F1E78E4808F0F1FA0FFA80F8B8F1010F65
:10607000EEDD294620688A4EFFF722FF002800F057
:10608000E08030608749884809F0FCFD3168864827
:1060900009F001FE844809F005FE01212068FFF7A0
:1060A0000FFFB8F1020F824600F0CE800222216875
:1060B0007A4808F0D4FAB8F1030FD0F8149000F041
:1060C000C58003212068FFF7FBFE0546102205A9C5
:1060D0007648FAF7FBFA002840F0BB80B8F1040FCD
:1060E00040F3B78004212068FFF7EAFE70490446B8
:1060F0006D4809F0C7FD6C4809F0D4FD1FFA89F21C
:106100005146614809F072F90DF1240869495E4869
:1061100009F06FF90DF1340B1022674940460DF07C
:10612000F4FE002301222021584603F049FF634971
:1061300058460DF072FE62495B4809F0A3FD5146D6
:10614000594809F0A8FD5F49574809F09BFD0A220C
:106150004946554809F0FFFD5B49534809F092FD57
:106160002946514809F097FD58494F4809F08AFDE2
:106170002B780BB91C461D46CDF80C804FF0020958
:106180004FF001082A46CDE90198CDF800B023462A
:1061900031683D484E4D08F0D3FE00285BD04D4B92
:1061A0004D49414800241C7009F06CFD31683E489F
:1061B00009F071FD3C4809F075FD484B032283F856
:1061C00000804121234615A803F0FAFE444915A892
:1061D0000DF023FE15A92C4809F0D6F823464A46AF
:1061E000412115A803F0ECFE3E4915A80DF015FE5F
:1061F00015A93D4809F066FD15A9234809F0C4F822
:1062000042462346412115A803F0DAFE354915A878
:106210000DF003FE15A9344809F054FD15A91A48DC
:1062200009F0B2F805233B700AF028FB2F492860DB
:106230001D4809F027FD1C4809F034FD27B0BDE8D2
:10624000F08F2B4B33601DE740F25B790DF11305A6
:106250003CE705AC52E727490F4809F013FD0A480F
:1062600009F0C9F80A2201460B4809F074FD2249D9
:10627000094809F007FD084809F014FD0AF0FEFA84
:106280000C232860DFE600BFE0030020D8030020D5
:10629000DC030020B88B0100840300206C07002081
:1062A00080030020EE8B0100B40300203C0400209A
:1062B000FB8B0100D95B0000A78F0100EB8F010071
:1062C0001B8C0100B27C01003B8C0100F18D0100B0
:1062D0008804002020040020428C01006603002076
:1062E000508C0100A87A010068030020568C010040
:1062F00001900100738C01007F8C010010B5114CDE
:106300001149204609F0BEFC1049204609F0C3FCA3
:106310004FF4FA700AF0E6FA012115200AF09CFC0D
:10632000002115200AF0C0FC4FF4FA700AF0DAFAE6
:10633000152001210AF0B8FC4FF4FA70BDE81040B6
:106340000AF0D0BAB40300203E8E01005E8E010038
:1063500070B592B002A809F045FC04A809F042FC0F
:1063600006A809F03FFC08A809F03CFC71497248F6
:10637000724E09F087FC704809F094FC02A970483D
:10638000FAF771FAF8B96F496B486F4C09F07AFC6B
:106390004FF47A6242F6E0616C4804F029FF00286D
:1063A00040F091806A496B4809F06CFC6A49694881
:1063B00009F068FC237801332370F6233370FFF76C
:1063C0009DFF12B070BD5E48FAF727FC18B15E4B16
:1063D0001B78022BD7D961495748614C10AD09F0A1
:1063E00051FC039B10942846119303F0C3FD04A9AC
:1063F0005348FAF7A2FA00285DD05A494E4809F0EE
:1064000041FC059B10942846119303F0B3FD06A9A7
:106410004B48FAF7C7FA002841D05349464809F0DB
:1064200031FC079B10942846119303F0A3FD08A9A3
:106430004348FAF74DFA10B34C493F4809F022FCA3
:10644000099B11932846109403F094FD039B00953B
:10645000CDE90B34059B3D480A94CDE90D34079BEB
:10646000CDE90F34099B11930CAA0EAB0AA904F0D5
:1064700049FF314809F016FC02233370A1E7039B62
:1064800032480C94CDE90D34059BCDE90F34079BC0
:1064900011930EAA2B460CA904F064FFE9E7039BB5
:1064A0002A480E94CDE90F342A46059B11930EA974
:1064B00004F080FFDDE7039B2448109429461193E4
:1064C00004F092FFD5E72A491B4809F0DBFB10A82E
:1064D00004F0EEFF119B039310A8214B109303F0DF
:1064E00049FD154809F0DEFB02A91548FAF78FFAB5
:1064F000204B13485B68119304A90593FAF7D3FA6C
:1065000010A805F019F8119B0D48079306A9FAF792
:10651000F0FA10A804F0EEFF119B0948099308A9AE
:10652000FAF79BFA01210648FAF77FFB0023237054
:10653000A2E700BF1D890100B4030020D80300209A
:106540003C0400202A890100480300204C0400205C
:106550005E89010084030020A089010036890100C2
:10656000AC9801004C890100528901005789010053
:10657000CF8901005806002007B51049104809F0DE
:1065800081FB684604F094FF684603F0F3FC0D4B72
:1065900000930D4B68465B68019303F0EBFC684683
:1065A00004F0CAFF684603F0E5FC684604F0A2FF69
:1065B000684603F0DFFC03B05DF804FBF7880100D8
:1065C000B4030020AC9801005806002018B103491C
:1065D000034809F057BB0349FAE700BF3C8E0100AE
:1065E000B4030020439D010010B5264C26492046E7
:1065F00009F048FB2549204609F044FB244B186864
:10660000003018BF0120FFF7E1FF2249204609F0C2
:1066100039FB214B1868003018BF0120FFF7D6FF67
:106620001E49204609F02EFB1D4B1868003018BF8C
:106630000120FFF7CBFF1B49204609F023FB1A4B33
:106640001868003018BF0120FFF7C0FF1749204627
:1066500009F018FB164B1878FFF7B8FF204609F031
:1066600021FB1449204609F00DFB03F02FFC0A2200
:106670000146204609F07BFB2046BDE8104009F0AA
:1066800011BB00BFB40300203E8801004B8801000D
:10669000D403002053880100D00300205C8801004F
:1066A000DC03002063880100240400206C880100C2
:1066B00078040020348201000020704710B5464C59
:1066C0004649204609F0DEFA4549204609F0DAFA43
:1066D0004449204609F0D6FA4349204609F0D2FA47
:1066E000204609F0DFFA4149204609F0CBFA40493B
:1066F000204609F0C7FA3F49204609F0C3FA3E494F
:10670000204609F0BFFA3D49204609F0BBFA3C4952
:10671000204609F0B7FA3B49204609F0B3FA3A4956
:10672000204609F0AFFA3949204609F0ABFA38495A
:10673000204609F0A7FA3749204609F0A3FA36495E
:10674000204609F09FFA3549204609F09BFA344962
:10675000204609F0A0FA3349204609F093FA32495D
:10676000204609F08FFA3149204609F08BFA30496A
:10677000204609F087FA2F49204609F083FA2E496E
:10678000204609F07FFA2D49204609F07BFA2C4972
:10679000204609F077FA2B49204609F073FA2A4976
:1067A000204609F06FFA2949204609F06BFA28497A
:1067B000204609F067FA2749204609F063FA26497E
:1067C000204609F05FFA2046244909F05BFA20468A
:1067D000BDE8104009F066BAB4030020EF8901005B
:1067E000118A0100248A0100328A01003A8A0100DC
:1067F0004A8A0100568A0100638A0100788A0100F2
:10680000878A01008F8A01009A8A0100A78A010005
:10681000B18A0100C08A0100C88A0100D48A01003F
:106820005E8E0100EA8A0100098B01001E8B0100C7
:106830002B8B0100398B0100458B01004D8B010032
:10684000588B0100658B01006D8B0100788B010076
:10685000878B0100908B01009E8B0100AC8B0100A7
:1068600008B5FFF72BFFFFF787FE0349034809F040
:1068700009FAC82008BD00BFBB830100B403002093
:1068800070B594B003F022FB064609F0F7FF054609
:106890002D4808F03FFA002854D02C4B1C7864B2E5
:1068A000002C4FD123460122402104A803F088FB8D
:1068B000274904A80DF0B1FA264904A80DF0ADFA55
:1068C000254904A80DF0A9FA3146684603F0F6FB05
:1068D00001236A4604A91C4808F079FC23460122DA
:1068E000402104A803F06CFB194904A80DF095FAA7
:1068F000184904A80DF091FA184904A80DF08DFA72
:1069000068464FF47A71B5FBF1F103F0D7FB012330
:106910006A4604A90C4808F05AFC2346012240218B
:1069200004A803F04DFB0E4904A80DF076FA0F22DF
:106930000C4968460DF0E9FA01236A4604A90248A9
:1069400008F045FC14B070BDE0030020B003002047
:10695000F28F010080870100558F01000A9001002D
:10696000EB8F0100E58F010010B50C4C2046F9F7C4
:1069700057FE78B90A490B4809F084F9DE232374DD
:10698000AD236374BE23A374EF23E374FE23237546
:10699000FF236375BDE81040FFF71ABA3C040020DE
:1069A000A3860100B403002008B5002008F03AF8DF
:1069B0001C491D4809F066F91C491D4807F0C0FF35
:1069C0001C491D4807F0BCFF1C491D4807F0B8FFD3
:1069D0001C491D4807F0B4FF1C491D4807F0B0FFD3
:1069E0001C491D4807F0ACFF1C491D4807F0A8FFD3
:1069F0001C491D4807F0A4FF1C491D4807F0A0FFD3
:106A00001C491D4807F09CFF1C491D4807F098FFD2
:106A10001C491D4807F094FF1C491D48BDE808406B
:106A200007F08EBF698601006803002061680000DE
:106A30006D860100E95A000072860100615800006D
:106A400077860100E57900006B900100455E00004B
:106A50007C8601008D58000080860100515900009D
:106A600085860100255A00008B8601004D5A0000E2
:106A700088860100515B00008F860100715800007C
:106A800095860100D158000099820100B958000094
:106A90009C8601002DE9F04F364D2B6885B00746E6
:106AA000002B63D0344C267876B2002E5ED122784B
:106AB000DFF8CC90DFF8CC80013252B2227099F826
:106AC0000020013252B289F80020D8F800A009F065
:106AD000D5FE334601460B22504603F005FB4E46D9
:106AE00000283BD02B68DFF8A0A0DD68DFF89CB061
:106AF0005DB32B7C03F00F03062B24D152462946AD
:106B0000584607F0B6FDA8B1037C03F00F03052B30
:106B100010D1D0F80C90B9F1000F14D049462A4694
:106B200001A8FAF781FB394601A8FBF785FAD9F8E5
:106B30000490F0E72946002201A8FAF775FB3946D0
:106B400001A8FBF779FA6D68D2E7032F03D009F0AB
:106B500095FEC8F800000948FBF7F2FA3378013BCC
:106B60005BB233702378013B5BB2237005B0BDE8A4
:106B7000F08F00BFD0030020CD0300202C030020A5
:106B80006503002084040020FF7A01006C070020C8
:106B90000220FFF77FBF000010B5094C23780133B6
:106BA0005BB2237009F0C0FE0320FFF773FF09F00A
:106BB000BBFE07F025FF2378013B5BB2237010BDBD
:106BC000B00300202DE9FF411E4F3B68002B35D05C
:106BD0001D4B1E7876B28EBB1C4C1D4D22780132A7
:106BE00052B22270D5F8008009F048FE33460146C3
:106BF00041F28832404603F077FA2E46D0B13B6826
:106C0000DD68A5B12B7C03F00F03062B08D12946C4
:106C1000002201A8FAF708FB012101A8FBF70CFAF2
:106C200009F082FE0220FFF735FF6D68E9E709F001
:106C300025FE30602378013B5BB2237004B0BDE8D1
:106C4000F08100BFD0030020CD03002065030020A9
:106C50009004002030B51449144885B009F012F8AA
:106C6000124809F01FF8124B1968D9B1114CCD68C0
:106C70002278013252B2227085B12B7C03F00F03CF
:106C8000062B07D10022294601A8FAF7CDFA01A860
:106C9000FBF72AFA09F048FE6D68EDE72378013B1F
:106CA0005BB2237005B030BDB2810100B403002097
:106CB000D0030020650300202DE9F04F934C23689A
:106CC0008FB0002B00F01C81914F3B78002B40F0DF
:106CD00017813B788F499048904D01335BB23B70F0
:106CE00008F0D0FF8C4808F0DDFF8D4A21688D4800
:106CF00007F0BFFC8C4A286021688A4807F0B9FC7D
:106D00008A4B8B4A18602168864807F0B2FC894B91
:106D1000894A18602168834807F0ABFC874B1860EC
:106D2000FFF7E8F8864A21687E4807F0A2FC854B09
:106D3000A946186070B1844C23785BB902F088FDD5
:106D4000002814BF01230023237003D07F49724819
:106D500008F098FF7E4A00231360D9F8003092466D
:106D6000002B00F0AF80D3F80C80DFF810B2794D23
:106D7000D9F80030002B00F0C680B8F1000F00F009
:106D80009E8098F8102002F00F02052AF2D14146A9
:106D9000644807F05AFC0128EAD9414603A8FBF7EA
:106DA000B3FC03A8FBF724FCA8B103A8FBF7C8FABF
:106DB000064680B9014603A8FBF700FB041E03A8A2
:106DC000BCBF64420126FBF74FFA9DF81C20052A40
:106DD00009D0062A44D009F0A7FD03A8D8F80480FA
:106DE000FBF738FAC4E718B9022103A8FBF74AFAFF
:106DF0004FF4807103A8FBF789FA059B23B14FF488
:106E0000007103A8FBF782FA20B203F067FB064685
:106E100060B15149514808F035FF0A2221464F48D8
:106E200008F099FF4D4808F03DFFD4E701212046C6
:106E300009F012FF3146204609F036FF5946284630
:106E400008F020FF21460A22284608F084FF444922
:106E5000284608F017FF4349284608F013FFBAE711
:106E600001900121204609F0F7FE20B203F036FB25
:106E7000019B20B10021204609F016FFABE7D6B1F7
:106E800013F1FF3618BF01263146204609F00CFFEA
:106E90003549284608F0F6FE0A222146284608F021
:106EA0005AFF3249284608F0EDFE0A2231462846AC
:106EB00008F051FFCFE7013B5E425E41E4E7DB684B
:106EC000CAF8003023482A4C08F0ECFEFFF7C2FE57
:106ED000FFF78AFB274B284801221A7004F08CFB2D
:106EE00020B1254804F04AFC0423237094F90030B3
:106EF000072B04BF042323703B78013B5BB23B703C
:106F00000FB0BDE8F08FDB68FFDE00BF300400206B
:106F10006503002049820100B4030020D40300204F
:106F2000598201006C0700206C8C0100980400203D
:106F3000607A0100D00300205F820100DC030020A2
:106F400064820100240400202804002067820100DC
:106F50002C040020680300207782010084030020B5
:106F60008F82010094820100677E01002B7B01006B
:106F7000D8030020640300209C03002087820100C6
:106F80002DE9F0433B4C23688DB0002B6ED03A4D79
:106F90002E6809F073FC002301464FF47A723046E4
:106FA00003F0A2F8074610B109F068FC2860334DE1
:106FB000DFF8D4902B7801335BB22B702368DE6846
:106FC0007BB2002B14BF4FF004084FF00208226878
:106FD000F2B1EEB1337C03F00F03052BF8D131464B
:106FE000484607F032FB0128F1D9314601A8FBF7EA
:106FF0008BFB01A8FBF7FCFA18B1414601A8FDF78D
:107000008DF909F091FC01A87668FBF723F9DEE71A
:107010002B78013B5BB22B70194B93F90030052B99
:1070200024D01FB3174F00263D463968F1B1EEB9A1
:107030000B7C03F00F03052B0CD101A8FBF764FBBD
:10704000012101A8FDF76AF9061C01A818BF012655
:10705000FBF700F92B684BB109F066FC2B685B6805
:107060002B60002BE1D12368DB682B600DB0BDE8FD
:10707000F08300BFD40300208C04002065030020AF
:10708000D80300202C0400206C070020F8B580EA0B
:10709000E074A4EBE074054620B20E4603F01EFA3D
:1070A000074668B11549164808F0ECFD0A2221464A
:1070B000134808F050FE1248BDE8F84008F0F2BD51
:1070C0000121204609F0C8FD022E09D1394620468B
:1070D00009F0EAFD0B490C4808F0D4FD0A48EBE73B
:1070E00036B9E943C90F204609F0DEFD0749F2E74A
:1070F000E90F204609F0D8FD0549ECE7C5820100FB
:1071000084030020D382010068030020E99001007D
:10711000F49001002DE9F04F2DED048B8A4B95B0D2
:107120001C6809F0ABFB0023014647F230522046B1
:1071300002F0DAFF002800F00081844B1A68002A70
:1071400000F0FB808249D4680B78DFF854929FED01
:10715000819A01335BB20B700025002C00F0BF80D8
:10716000237C03F00F03052B13D100222146484650
:1071700007F075FA4369052B0BD1214609A8FBF7E7
:10718000C3FA09A8FBF734FA804620B909A8FBF72F
:1071900061F86468E1E709A907A8FDF7F5FD09A80A
:1071A000FBF7E0F90021064609A8FBF707F90546B9
:1071B00007A8FDF79DFB08EE900A09A8FBF754F815
:1071C00033B207EE903AF8EEE77A834687EE898A83
:1071D00009A8FCF79DFF60498246604808F052FD0F
:1071E000022718EE900A0BF075F8009702460B463E
:1071F000CDE90401594808F083FE5949574808F081
:1072000041FD18EE100A0BF065F8009702460B4698
:10721000CDE90201514808F073FE52494F4808F089
:1072200031FD59460A224D4808F095FD5FEA164B9C
:1072300050D0082003F036F94FF6FF7381B240F6C4
:107240002712584602F050FFC8B12168464808F09E
:1072500022FD4649444808F015FD22684449454846
:1072600007F0A0FFB1B209A8FBF794F93946284608
:10727000FFF70CFF09A8FAF7EDFF454689E7DFEDB8
:107280003E7AB4EEE78AF1EE10FA04DD22683B495B
:10729000384807F087FFBAF1000F01D10121E6E776
:1072A0000022374BDDE904010AF0B4FEDDE90223D8
:1072B0000BF0F8FA08B10021D9E7F4EEC88AF1EE34
:1072C00010FAEBD92F49254808F0DCFC234808F0D8
:1072D000E9FCCFE72C49214808F0D4FCCAE71C4C54
:1072E0002378013B5BB2237009F0C8FA164B186093
:1072F000FFF7C6FA35B32549184808F0C3FC02F079
:10730000E5FD0A220146154808F031FD20491348E1
:1073100008F0B8FC217811480A2249B208F01BFD98
:107320001C490E4808F0AEFC1B4B0C4819680A2299
:1073300008F01DFD094808F0B5FC15B0BDEC048B44
:10734000BDE8F08F1549D7E794040020D40300204E
:10735000650300200000C842EF810100680300209F
:10736000F58101008C7D010084030020FB81010078
:107370000B820100E0030020000018421782010088
:107380000000F03F248201000182010033820100ED
:1073900039820100418201007C0400204C7B010005
:1073A0006C0700202DE9F043644E33688DB0002B4C
:1073B00000F0C280002832D101276149614D624846
:1073C00008F060FC604808F06DFC2B785F4A0133E0
:1073D0005BB22B7013689046002B61D0DC68DFF83D
:1073E000A091002C63D0237C03F00F03052B14D154
:1073F0002146484607F029F978B1216801A8FBF732
:10740000B9F901A8FBF7F4F810B101A8FAF71CFFCD
:1074100009F08AFA01A8FAF71DFF6468E1E74C4910
:1074200049484C4CDFF8748108F02CFC464808F0C1
:1074300039FC09F023FA274605462378EBB109F019
:107440001DFA0023014642F21072284602F04CFE5B
:1074500098B907F0D5FA98F80030D3B93E4B93F9B4
:107460000030052B01D0FFF78BFDFFF753FE022004
:10747000FFF710FB09F058FADFE73B78002B9BD0B1
:107480003649374808F0FEFB354808F00BFC00276A
:1074900093E7344B1B68002BE0D002F0EFFADDE7F6
:1074A0003149294808F0EEFB274808F0FBFB2F4B39
:1074B0002F49254800241C6008F0E4FB224808F00E
:1074C000F1FB642009F00EFA2A4B2B491C702B4B60
:1074D0001D481C7008F0D6FB02F0F8FC0A22014699
:1074E000194808F044FC3168254806F0D2FC254BC9
:1074F00025491C60254B14481C60254B34601C60DA
:10750000244BC8F800401C60164B1C6008F0BAFB06
:1075100002F0DCFC0A2201460B4808F028FC0A486D
:1075200008F0C0FB1C4B1C702B78013B5BB22B702E
:1075300038460DB0BDE8F0830127F9E7300400209C
:10754000F68D01008004002068030020D403002091
:10755000BE8D010065030020D8030020D38D0100FB
:1075600084030020240400200C8E01002C04002041
:107570001C8E010078040020248E0100640300208A
:107580006C070020D0030020FE7E0100980400203C
:10759000DC03002080030020660300202804002074
:1075A000F0B5454C267876B289B02746002E47D1F3
:1075B00023784249424D434801335BB2237008F0BF
:1075C00061FB404808F06EFB722201212846F9F762
:1075D00097FD2846F9F722FD7B2846D13A493B48DA
:1075E00008F050FB394808F05DFB394B04933046F6
:1075F0004FF0FF33079305960695FFF7D3FE04A9D6
:107600003448354E06F058FF30602846F9F724FD1F
:107610003568BDB93149324808F034FB304808F0CC
:1076200041FB304901A809F003F801A92E48F9F7F8
:10763000A3FB01A808F0B7FF2378013B5BB22370DE
:10764000002010E029491F4808F01CFB1D4808F0E5
:1076500029FB2378013B5BB22370FFF72DFB224807
:10766000F9F750FC012009B0F0BD2846F9F7BAFC43
:1076700098B12B7D1BB1FF212846F9F7DFFC194992
:1076800004A808F0D5FF04A91748F9F775FB04A86A
:1076900008F089FF1448F9F7F3FB0948F9F7DCFC17
:1076A0001349084808F0EEFA064808F0FBFA3B7860
:1076B000013B5BB23B70C3E7650300209E8801007D
:1076C00054040020B4030020B9880100680300209E
:1076D000E09701006C07002030040020C7880100FB
:1076E00084030020029801003C040020D38801009C
:1076F000E68801002DE9F041C0B000211C2214A849
:1077000013910BF02EFC202213A99B48F9F75AF88D
:1077100078B92022994913A80CF0F7FB98499948A9
:1077200008F0B0FA13A9974808F0B5FA954808F0A0
:10773000B9FA914D6A7D2B7C04922A7D0392EA7CF2
:107740000292AA7C01926A7C009240218E4A1BA878
:107750000CF0A2FA8D498B4808F094FA13A98948D5
:1077600008F099FA1BA9874808F095FA854808F0AF
:1077700099FA4FF47A730022CDE90F23844A0E92CE
:107780002BAC08228DF84820ADF84A3013AA5023BC
:107790000EA9204606F004F84FF47A637D497E482E
:1077A0003B9308F06FFA02F091FB0A2201467A48F7
:1077B00008F0DDFA784808F075FA204606F01FF860
:1077C0001BA9204606F042F9744906460AA808F0AB
:1077D0002FFF294607A8F9F78BFA079A0A9920463E
:1077E00006F012F807A808F0DEFE0AA808F0DBFE93
:1077F000204606F028F9002E40F0B780204606F01B
:1078000033F9DFF8DC810646204606F09FFA07468A
:1078100000B3214607A806F09DF941460AA808F0E2
:1078200007FF0AA907A808F0ACFF07460AA808F056
:10783000BAFE07A808F0B7FE002FE5D021460AA837
:1078400006F0A2F90AA92846F9F796FA0AA808F05C
:10785000AAFED9E752494B4808F014FA0A223146E9
:10786000484808F078FA474808F01CFAC82E70D14A
:107870004C4B4D490A9348480C944FF0FF330D93FD
:107880000B9708F0FFF902F021FB0A22014642485B
:10789000464D08F06CFA404808F004FA0120FFF762
:1078A00081FD43493C4808F0EDF93B4808F0FAF9FE
:1078B0003D49394808F0E6F902F008FB0A22014682
:1078C000354808F054FA344808F0ECF90AA9394868
:1078D00006F0F2FD2860204605F086FF2C68C4B94A
:1078E0003549364808F0CEF9354907A808F0A0FE1A
:1078F00007A92148F9F740FA07A808F054FE2646E0
:10790000304B2B933DA808F04EFE304640B0BDE80A
:10791000F0812D49204808F0B5F902F0D7FA0A2283
:1079200001461D4808F023FA1B4808F0BBF9FFF791
:10793000C3F92649134808F0A5F9254B1B78002BFD
:10794000DED00D48F9F74DF90028D9D0FEF792F8AE
:10795000D6E7B6F5987F0CBF1E491F49174808F0B7
:1079600091F9204605F040FFCAE71C49134808F08A
:1079700089F94FF0FF36C3E73C0400207A8F0100FD
:1079800021870100B40300203F8701006E870100BA
:10799000409601008287010068030020988701005B
:1079A000AB870100E0970100F3870100300400205D
:1079B000BE8701006C070020D487010084030020EB
:1079C000029801004C970100EB870100F987010044
:1079D0006403002000880100148801002E88010043
:1079E000A6870100012838B50C4630DD4D682F49C7
:1079F00028460CF0F4F928B901212D48F9F732F99D
:107A0000C82038BD2B4928460CF0E9F9014600286A
:107A1000F3D02949294808F035F92548F9F718F92C
:107A20000A220146254808F096F9244808F03AF958
:107A300061681F48F8F7ECFE6168204808F02BF9F0
:107A40001F491E4808F01EF91C4808F02BF91D4C70
:107A500094F90030012B1FDDFFF74CFEC82802D13E
:107A600004232370CDE7431C10D11749174808F0B1
:107A700009F9164808F016F9154B164800221A7035
:107A80000323237003F07AFEC920BAE7124B1B7858
:107A9000002BE5D10F23E4E71049114808F0F2F874
:107AA0000F4808F0FFF84FF4FA70AAE7738E010050
:107AB0003C0400207C8E010055830100B4030020AB
:107AC00075830100D80300207C8301006803002037
:107AD000660300209C0300206403002097830100BC
:107AE000840300202DE9F3470024324D0094224600
:107AF000214623463048314FDFF800A108F07AF8DC
:107B000028464FF47A762E4B6C60AE6040F8143BFA
:107B10004FF0080808F066F885F820802946294DBE
:107B20000122384607F094FF4FF0010900943B46CC
:107B300029460722244802F011F83B462946CDF891
:107B400000900322214802F009F800943B460622E7
:107B50001F4F20482946204D02F000F84FF4805373
:107B6000C5E901462B611D491D4B2B60381D85F869
:107B7000204008F05DFD3D601A4D1B4952463846D5
:107B800009F052F9C5E90146184C194B19482B6008
:107B9000494685F810806E8201F094FF2946204600
:107BA00007F044FC14495246204602B0BDE8F047B5
:107BB00009F03AB9C00400204C0300209C040020C6
:107BC0009C960100D4070020680300208403002055
:107BD0003C040020B403002054040020029801005B
:107BE000707A01009C030020C3580000E0030020CD
:107BF000409601003404002081EA000000000020CB
:107C00002DE9F0470024C8B03C22214609A8089479
:107C10000BF0A7F97C22214629A828940BF0A1F9A2
:107C200023460122402108A802F0CAF9AF49B04E0C
:107C3000B04F08A80CF0F1F87F22AF4928A80CF04B
:107C400064F9012328AA08A9AC4807F0C0FA234622
:107C50000122402108A802F0B3F9A94908A80CF0B4
:107C6000DCF87F22A74928A80CF04FF9A64928A8DC
:107C70000CF0D3F8012328AA08A9A04807F0A7FA16
:107C800023460122402108A802F09AF99F4908A83A
:107C90000CF0C3F87F229E4928A80CF036F9012386
:107CA00028AA08A9954807F092FA23460122402104
:107CB00008A802F085F9974908A80CF0AEF87F22D1
:107CC000954928A80CF021F9012328AA08A98B4876
:107CD00007F07DFA33783D6801335BB23370002DD5
:107CE00000F03B818D4BDFF86092B3F80080ADF877
:107CF00000801E2221460DF102000BF032F93E22D7
:107D000021460DF16200ADF86080DFF840A2DFF897
:107D100040820BF026F9ED683B68002B00F0AE8046
:107D2000002D00F0AB802B7C03F00F03052B40F0FF
:107D30008E802946404606F088FC002800F08780A7
:107D400028680CF0B4F80134044400222946404667
:107D500006F085FC4369112B12D8DFE803F07C871D
:107D6000877C7C097C7C7C7C11111111111111879D
:107D70001F226B4968460CF0C8F800238DF860306C
:107D800000230122402108A802F01AF93F222968A5
:107D900008A80CF094F8494608A80CF03EF85146A3
:107DA00008A80CF03AF801235E4A544808A907F0E5
:107DB00073FA00230122402108A802F001F93F22B2
:107DC000296808A80CF07BF8494608A80CF025F8AB
:107DD000554908A80CF021F80123544A474808A93E
:107DE00007F05AFA00230122402108A802F0E8F81F
:107DF0003F22296808A80CF062F84D4908A80CF049
:107E00000CF8514608A80CF008F801236A4608A9A6
:107E10003A4807F0DCF99DF86030C3B10023012235
:107E2000402108A802F0CCF83F22296808A80CF0ED
:107E300046F83F4908A80BF0F0FF3B4908A80BF0B3
:107E4000ECFF012318AA08A92C4807F0C0F908F094
:107E50006BFD6D6860E71F22364968460CF055F8E7
:107E600035493F2218A80CF050F889E71F22334902
:107E700068460CF04AF83F223149F3E7002301221B
:107E8000402108A802F09CF82E49DFF8C4901B4D51
:107E900008A80BF0C2FF0123621E08A9174807F0CB
:107EA00010FA3B68DC683B68002B53D0002C51D0A3
:107EB000237C03F00F03052B14D12146484606F01E
:107EC000C4FB78B1D4F8008040460BF0F0FF414687
:107ED0000246284606F0C5FD63681BB12C212846E2
:107EE00006F0B2FD08F020FD6468DCE7EB8F0100CE
:107EF00065030020D4030020E58F0100E00300208B
:107F0000C58F01002490010011900100F28F010043
:107F1000648F0100D78F01005E8F01009281010004
:107F2000D18F0100C08F0100F98F0100868F010001
:107F30004F830100B88F0100748F0100CB8F0100C7
:107F4000B48F0100DE8F0100498301004B8F0100D7
:107F50006C070020044806F06CFE3378013B5BB2EE
:107F6000337048B0BDE8F087E003002070B5A44C42
:107F700094F900300B3392B01A2B2BD8DFE813F0B2
:107F8000F300E3002A002A002A002A002A002A001F
:107F90002A002A002A001B0047004A0053009100D3
:107FA000AE00D3002A002A002A002A002A0003017A
:107FB000100125011F01934B93481B78002B14BF20
:107FC0000921012101F07FFD03F024FA022801D0EC
:107FD000FEF7BEF994F90030012B40F346818B4B3C
:107FE0001B78002B40F0368103F01EFA054603F0A3
:107FF00011FA022800F03081013D042D00F2358194
:10800000DFE815F037013901470149012A01022350
:108010002370DFE77E4D2B781BB9FDF76BFF012343
:108020002B700323F4E7774D77482B78002B14BF90
:108030000B21032101F047FD764B1B78002B40F00C
:108040002C817548F8F704FEE8B1744B1B78C3B96E
:10805000FFF750FBC82801D10423D9E72B783BB1A7
:108060006F49704807F00EFE6E4807F01BFEF3E7FD
:1080700001A803F01DFA029B0BB10F23C8E7F623FA
:10808000C6E76949EDE72B784BB10423674965489A
:10809000237007F0F7FD634807F004FE9AE70F230B
:1080A000F4E7584B58481B78002B14BF0B210321D1
:1080B00001F009FD5E4B196841B95E49594807F066
:1080C000E1FD584807F0EEFD0723A1E75A4806F006
:1080D000BCFA0128F1D9FDF7A5FF7BE7574B1D68D6
:1080E00008F0CCFB002301464FF4FA52284601F079
:1080F000FBFF00283FF46EAF00230322412101A8BB
:1081000001F05EFF4E4901A80BF087FE01A94D4822
:1081100007F03DF9FFF774FD06234B4941482370F2
:1081200007F0B0FD56E7374B37481B78002B14BFDC
:108130000A21022101F0C7FC424806F0EBFD0028AD
:108140007FF448AF88E708F099FB3C4B1860F523B3
:1081500023702C4B2C481B78002B14BF09210121C4
:1081600001F0B1FC36E7354B1D6808F087FB0023B2
:10817000014641F28832284601F0B6FF00283FF45C
:1081800029AF002344E72F4806F0C4FD10B12D4865
:1081900006F08DFD08F072FB284B18600D2337E7C1
:1081A000264B1D6808F06AFB0023014642F210725C
:1081B000284601F099FF00287FF44EAF0AE708F047
:1081C0005DFB1E4B18600E2322E7FFF7E9F9054619
:1081D00000287FF441AF194B1E6808F04FFB2B4677
:1081E000014647F23052304601F07EFF00283FF44E
:1081F000F1AE1649164807F045FD01F065FFE9E6C6
:10820000D803002064030020340400204803002029
:10821000CC030020650300203C04002066030020FE
:10822000978C0100B4030020BE8C0100CE8C0100AD
:10823000DC030020088D01006C070020880400206A
:10824000508C0100E00300201B8D0100328D0100E5
:10825000840300200025CAE61149124807F012FDE8
:10826000104807F01FFDF623237094F9000012B0A8
:1082700070BD0D49F1E70D490D4807F003FD01A858
:1082800003F016F901A801F075FE094807F00AFD90
:10829000EBE70849E1E70849EEE70320E7E700BF1D
:1082A000558D0100840300205E8D0100728D010058
:1082B000B40300208F8D0100A28D010008B518487D
:1082C00001F003FC08F030FB06F09AFBFFF74EFECE
:1082D000022802DD134806F045FE08F025FB124B8C
:1082E0001B7823B1114B1B680BB101F0C7FB104B7E
:1082F0001B6853B10F4B93F90030052B01D0FEF7EB
:108300003FFE08F011FBFEF705FF08F00DFB022011
:10831000FEF7C0FB08F008FBBDE80840FEF752BCC2
:1083200034040020E003002028040020240400205E
:10833000D4030020D803002010B54FF4E1311B48CE
:1083400007F0B8FF1A48F8F743F9044630BB19495B
:10835000164807F0ADFC21462046FDF7F9FB14480E
:10836000F8F7B5FC144B18701148F8F7B8FC134B2C
:108370001870FEF719FBFEF7A1F9FEF7F5FA1420C5
:1083800008F0B0FA0E490F4807F033F84FF4FA70CE
:1083900008F0A8FABDE81040FFF702B90A490B48F7
:1083A00007F070FC094807F07DFCD8E7D4070020EF
:1083B0003C040020C68101000500002006000020CA
:1083C000D95B0000E0030020DB810100680300208E
:1083D00007B5002300931A461946034807F00AFC24
:1083E00003B05DF804FB00BFE404002003207047E5
:1083F0007047000073B56E460546304686E80600B5
:10840000FCF770FC04463046FCF706FA10B1002C6D
:1084100008BF01244FF480416868F9F777FF012C09
:108420001BD0022C04D0FCB91C491D4807F02AFCC3
:108430003046FCF702FA70B36868FAF793F818B997
:108440000124204602B070BD00206C6802F02AF8BA
:1084500001462046FAF79EF8F2E73046FCF78CFB1F
:1084600001280AD0022808D00E490D4807F00AFC5E
:108470000B4807F017FC0024E3E76868FAF772F886
:108480000028DDD000206D6802F00CF80146284677
:10849000FAF780F8D5E70446D3E700BF2E90010035
:1084A000680300204690010010B5044608F07EFAEB
:1084B000204610BD10B504461649174807F002FCC7
:1084C00000216068FAF766F8236820469B6900215E
:1084D000984794F9080002F001F840B10F4910489C
:1084E00007F0D0FB0E4807F0DDFB002010BD94F92B
:1084F000090001F0F3FF0028F0D1A17C94F90800F5
:1085000008F0D2FB94F90900A17C08F0CDFB012012
:10851000ECE700BF6F900100680300207E9001002F
:108520008403002001292DE9FF41044600F08980E1
:108530004FF480414068F9F7D1FE002800F08180B7
:108540004FF400416068F9F7C9FE60B9764D95F9BE
:108550000030002B75D04FF400416068F9F7D6FE6B
:108560002B78013B2B7094F9080001F0B7FF00282D
:1085700067D194F9090001F0B1FF0546002860D1E8
:108580006068F9F7EFFF2A462946074602A8FBF77D
:10859000C5FF4FF40072616802A8FCF7B1FB2946E1
:1085A00002A8FCF77DFA06466068F9F75DFE02282E
:1085B00001D0052800D1002694F90A00A0F10E038D
:1085C000DBB2072B00F29C804FF0FF0808F04EFA58
:1085D000E289218ACDF80080002307F0DAFF051E2A
:1085E000C0F28A80454500F38980002F40F08B80DF
:1085F000751B15F10A0F55DA94F90900A17C08F0F2
:1086000053FB6068F9F7AEFF30B9666801F04AFFC6
:1086100001463046F9F7BEFFA37C6842002B3CD0F0
:1086200000210091FF23192207F0B3FFFF28014624
:10863000A8BFFF21462994F90800B8BF462108F0D9
:10864000B9FA002004B0BDE8F0813849384807F095
:1086500019FB374807F026FB3649354807F032FB4F
:10866000A17C94F9080008F01FFBA17C94F9090093
:1086700008F01AFB00216068F9F78CFF4FF4804185
:108680006068F9F783FE4FF400416068F9F77EFEF9
:10869000254A137801331370D3E7FF22009219465D
:1086A0001922C1E70A2DD7DD94F90800A17C08F052
:1086B000FBFA6068F9F756FF30B9666801F0F2FE20
:1086C00001463046F9F766FFA37C83B10021009193
:1086D000FF233322284607F05CFFFF280146A8BF8E
:1086E000FF214629B8BF462194F90900A7E7FF22D8
:1086F000009219463322EDE7002576E7454674E7F8
:108700007FB14FF0FF3508F0B9F800230146B4F906
:108710000C20384601F0E8FC002896D16B1C7FF451
:1087200067AFA6F17F0564E70400002052900100C6
:108730006803002061900100002110B50446817497
:108740004068F9F73BFE43B2002BBBBF40422072AA
:1087500023720123B8BFA374237A6068013B182BEE
:1087600084BF202323720121F9F728FE43B2002B96
:10877000BBBF4042607263720123B8BFA374637AC7
:108780006068013B182B84BF212363720221F9F733
:1087900015FEC3B2192B8ABF0023A072A372032156
:1087A0006068F9F70BFE80B2431EB3F5806F26BFF9
:1087B0000023E381E08104216068F9F7FFFD80B2C6
:1087C000B0F5806F8ABF4FF4806320822382052139
:1087D0006068F9F7F3FD00B20028D6BF42F21073CB
:1087E000A081A38110BD000038B50446F7F7FDFD58
:1087F0002046FFF7A1FF2549254807F063FA94F9C1
:10880000080001F06BFE40B12249234807F03AFA14
:10881000214807F047FA002038BD94F9090001F01B
:108820005DFE05460028EFD1012194F9080008F00B
:1088300013FA012194F9090008F00EFAA17C94F9C9
:10884000080008F031FAA17C94F9090008F02CFA2C
:10885000294694F90A0008F0FFF929466068F9F7FB
:1088600099FE4FF480416068F9F790FD4FF40041A4
:108870006068F9F78BFD236820469B6902219847C1
:10888000064B02221A700120C6E700BF8B90010040
:10889000680300207E900100840300200400002073
:1088A00007B5002300931A461946034807F0A2F9BA
:1088B00003B05DF804FB00BFEC040020002070470B
:1088C00003207047704700002DE9F0410646F7F796
:1088D0008CFDB468002C41D0E468254F254DDFF8AD
:1088E000A88064B3236843B31B7833B33A46214668
:1088F000284605F0BEFE30B94FF0FF333A46214618
:10890000284605F0FEFE42462146284605F0B1FE07
:1089100030B94FF0FF3342462146284605F0F1FEBC
:10892000154A2146284605F0A4FE30B94FF0FF3322
:10893000114A2146284605F0E4FE6468D1E70F4954
:108940000F4807F09FF90E4807F0ACF9336830463E
:108950009B69022198470120BDE8F0810949084838
:1089600007F090F9064807F09DF92046F4E700BFAC
:10897000799401006C0700205D9001004B9101008B
:10898000680300205A9101004E90010038B5084D4F
:1089900008490446284607F075F9284607F082F989
:1089A000236820469B6900219847012038BD00BFFD
:1089B00068030020399101002DE9F04F91B008AC17
:1089C0000746204684E806000693FCF7D5F80B28F6
:1089D00000F028822046FCF7CFF80A2800F0228217
:1089E0002046FCF77FF983462046FBF715FF20B1B0
:1089F000BBF1000F08BF4FF0010B2046FBF70CFF47
:108A000090B12046FCF76EF907280DD12046FCF7FF
:108A1000B3F811286AD012286AD0102804D1FF2296
:108A200021460EA8FCF7B7F8BB68002B00F0FA81CE
:108A30004FF00008DC68CDF80C80C146C246CDF886
:108A40000880002C00F0DE80A24AA348214605F0F1
:108A500010FEA24A214605469F4805F00AFEA04A9C
:108A6000064621469C4805F004FE0590002D00F0C6
:108A70008B80002E00F088802B7C03F00F03022BEC
:108A800040F08280337C03F00F03022B7CD1954AA7
:108A90009148214605F0EDFD43690493069B002BA8
:108AA0005DD0194620680BF0D4F9002857D108A8EA
:108AB000FBF7B2FE08BBBBF1070F6FD008AA104648
:108AC0000792FBF7BAFE079A00283CD01046002117
:108AD0000792FBF7E5FF6861FDF75CF8079A00284D
:108AE00031D0236800934FF4007328E0802297E789
:108AF0000A212046FBF796FF96E708A8FCF73CF80A
:108B0000706108A8FCF738F801283FD0022843D04C
:108B1000FDF740F858B17369012B08D16B69132B2D
:108B200005DC1E226A6108A90EA8FCF734F8FDF7DF
:108B300031F840B12368009308AA4FF4407306CA85
:108B40007868F9F7D3FF059B4BB10023CDE90033DB
:108B500008AB0CCB4FF0FF31059801F0DFFA7369D9
:108B6000022B0FD001330DD06B69049A0299434553
:108B700002FB03F21144C4BF9846049B0291C4BF98
:108B800091460393049B9A4464685AE76A6908A96A
:108B90000EA8FCF700F8BBE70022F8E708A8FBF7EF
:108BA0004CFE00288AD008A8FBF782FE7369A8B1A2
:108BB000022B01D001330CD14B494C4807F06BF824
:108BC0004A4807F06FF80122726108A90EA8FCF765
:108BD00082F808A8FBF76CFE6861A8E7022B0ED0AC
:108BE00001330CD04249414807F055F83F4807F09F
:108BF00059F80222726108A90EA8FCF76CF800234C
:108C00006B6194E7BAF1000F00F00C8139493748E5
:108C1000029B93FBFAF507F035F80A2251463348D8
:108C200007F099F83449314807F02CF8FF26029BE9
:108C30002E4893FBF6F10A2207F08DF82F492B48B6
:108C400007F020F80A222946284807F084F82C4922
:108C5000264807F017F899FBF6F10A22234807F097
:108C60007AF82849214807F00DF80A2203991F488D
:108C700007F071F824491D4807F004F81B4807F075
:108C800011F8224AB968144805F0F3FC0EAE82468A
:108C9000224621460AA8FBF741FC2A460AA930468B
:108CA000FBF779FF0DF13008002D14BF01220222DD
:108CB00031464046FCF70FF8CDE900444FF0FF3154
:108CC00098E80C00504601F029FA0DBB012011B0C4
:108CD000BDE8F08F799401006C0700204E900100F0
:108CE000DC900100E0900100E290010068030020A8
:108CF000ED900100F9900100029101000D91010039
:108D000014910100229101002991010002980100B3
:108D1000BB68002BDAD0DD68434FDFF828B1002DA7
:108D2000D4D0424A2946384605F0A3FC5A46446945
:108D30002946384605F09DFC3D4A8046294638467E
:108D400005F097FC3B4A82462946384605F091FCDF
:108D5000B8F1000F60D0BAF1000F5DD000285BD0F1
:108D600098F8102002F00F02022A55D19AF810202C
:108D700002F00F02022A4FD1027C02F00F02022AF7
:108D80004AD1002C48D04269022A47D0013245D04E
:108D9000B9F1000F44D0DAF814302968264803FBF3
:108DA00004FA039BCAEB0A2292FBF4F45C4306F03C
:108DB00072FF94FBF9F421491F4806F06CFF0A2268
:108DC000FF211D489AFBF1F106F0C5FF1C491A4826
:108DD00006F058FF0A222146174806F09AFF164867
:108DE00006F060FFD8F81430A34215D000221146D7
:108DF0000AA8FBF793FB22460AA93046FBF7CBFEF5
:108E00000023CDE900334FF0FF3196E80C002846EF
:108E100001F084F9C8F814406D6880E70024E1E7A8
:108E20004C46DFE7002052E76C070020E09001008D
:108E3000799401004E900100680300202D910100FB
:108E4000339101005D90010010B5044607F0AEFDBE
:108E5000204610BD0023836043683BB15B682BB1A3
:108E60001A7C02F00F02062A08BF836070470000D8
:108E700007B5002300931A461946034806F0BAFEC8
:108E800003B05DF804FB00BFF404002043687BB12D
:108E9000B0F90A20042A05D0052A05D0032A05D1F5
:108EA000022070470120704711207047187C7047DE
:108EB000184670477047000038B50446F7F795FA32
:108EC0002849294806F0DEFE0A22B4F9081026488F
:108ED00006F041FF2549244806F0D4FE6368224885
:108EE0001B68196806F0D7FE21491F4806F0CAFE24
:108EF0001D4806F0D7FE606888B3B4F908307BBB24
:108F0000236820469B6B98470128054605D0022818
:108F10000AD00121B4F9080019E003212046F7F72F
:108F200031FB294607F098FE00212046F7F72AFB7F
:108F3000012107F091FE01212046F7F723FB0121D3
:108F400007F08AFE02212046F7F71CFB012107F0FB
:108F500083FE236820469B6902219847012038BD83
:108F60000020FCE7B8910100680300204C7B010061
:108F70002B93010010B504462449254806F082FED3
:108F80000A22B4F90810224806F0E5FE21492048DB
:108F900006F078FE63681E481B68196806F07BFEC1
:108FA0001D491B4806F06EFE194806F07BFE23683B
:108FB00020469B6B9847012805D002280AD0002143
:108FC000B4F9080019E003212046F7F7DBFA002185
:108FD00007F042FE00212046F7F7D4FA002107F0FF
:108FE0003BFE01212046F7F7CDFA002107F034FEC1
:108FF00002212046F7F7C6FA002107F02DFE23686C
:1090000020469B6900219847012010BDB8910100BE
:10901000680300204C7B0100168E01002DE9F0430F
:10902000044689B040689DF840309DF8445002AF36
:1090300087E80600002800F09880B4F90820002A8C
:1090400000F09280002B00F093800021F9F7B6F930
:10905000236881469B6B2046984706B2022E19D0A2
:10906000032E19D0012E0CBF05210121002204A8D6
:10907000FBF754FA4FF0FF33009397E80C0004A974
:1090800006A8FCF741F8012E32D0022E27D1002D80
:1090900043D13DE00421E9E71DB34FEAD9713846D9
:1090A000B4F90850FBF7FCFC80460146284607F05F
:1090B00081FD3049304806F0E5FD0A22B4F9081078
:1090C0002D4806F048FE2D492B4806F0DBFD0A220C
:1090D0004146294806F03FFE274806F0E3FD0120FF
:1090E00043E0B4F9080001F0F9F90028D5D0E0E731
:1090F00003212046F7F746FA06462DB19DF81710D2
:10910000304607F057FDC2E701F0E8F90028F5D036
:10911000B4F9080001F0E2F928B99DF81610B4F985
:10912000080007F047FD01212046F7F72BFA064615
:1091300085B19DF81510304607F03CFD2046022110
:10914000F7F720FA044655B19DF81410204607F0B1
:1091500031FDC4E701F0C2F90028EAD0EEE701F0E2
:10916000BDF90028F0D0BAE7104609B0BDE8F08399
:109170001846FAE7677E0100680300202B7B010098
:1091800010B5044607F012FC204610BD07B50023B9
:1091900000931A461946034806F02CFD03B05DF80B
:1091A00004FB00BFFC040020032070477047000050
:1091B00038B50446F7F719F92149224806F062FD4F
:1091C0000A22B4F908101F4806F0C5FD1E491D48C3
:1091D00006F058FD1B4806F065FDB4F9080001F0E3
:1091E0007DF9054640B11949194806F04BFD18486C
:1091F00006F058FD002038BD0121B4F9080007F041
:109200002BFDB4F90800A17A07F04EFD606810B19B
:109210002946F9F7BFF9236802219B692046984740
:109220006068FAF775FF002807DD0020646801F028
:1092300039F901462046F9F7ADF90120DBE700BF17
:1092400042920100680300202B9301007E900100F0
:109250008403002038B50F4D0F490446284606F018
:1092600011FD0A22B4F90810284606F074FD0B49D6
:10927000284606F007FD284606F014FDB4F908005C
:10928000002107F0E9FC236820469B6900219847EC
:10929000012038BD6803002042920100168E0100B3
:1092A00010B5044607F082FB204610BD002110B522
:1092B000044681724068F0B1F9F780F803B2002BE0
:1092C000BBBF4042208123810123B8BFA372238901
:1092D0006068013B182B84BF202323810121F9F70B
:1092E0008DF808F0F7FF0022054B09F04BF809F064
:1092F00021FB08B1E06010BD41F28833E360FAE77A
:1093000000408F4030B5044687B000232F22CDE9BE
:109310000023ADF80830B0F90800A37A0D4671B308
:1093200083F0010107F0C0FCE368B3F57A7F57D3FF
:109330003149324806F0A6FC0A22B4F908102F4839
:1093400006F009FD2E492D4806F09CFC0A2229460C
:109350002A4806F000FD294806F0A4FC2949684681
:109360000AF05BFD6068F8F77FFF002D3ED01428FF
:1093700007D0152836D00F2836D1234902E01946E8
:10938000D0E7224903A80AF06EFD21491B4806F0E8
:1093900079FC63681968236809685D6A03AA6B46EB
:1093A0002046A8470A220146144806F0D4FC194971
:1093B000124806F067FC636810481B68196806F0DD
:1093C0006AFC69460D4806F066FC13490B4806F036
:1093D00059FC03A9094806F05EFC084806F062FC47
:1093E00007B030BD0D49CDE70D49CBE702280CBFD2
:1093F0000C490D49C6E700BF4E92010068030020EA
:10940000FE7E0100199201000C92010027920100DA
:1094100053920100B27C01005F9201002092010092
:109420002F92010010920100149201000129F7B55A
:10943000044644D04368002B41D0002211466846C0
:10944000FBF76CF84FF4007261686846FBF758FC54
:1094500000216846FBF724FB05466846FBF78CFBBA
:109460006068F9F77FF8064607F008FAE268FF211E
:109470006A430023B2FBF1F20146304600F034FEAD
:109480000746E6B107F0FAF900230146E2683046E4
:1094900000F02AFE064620B30020666801F002F8BC
:1094A00001463046F9F776F84DB1207A01F004F81C
:1094B000A37A834203D101212046FFF723FF002036
:1094C00003B0F0BD9FB131462046FFF71BFF606837
:1094D000FAF71EFE01460028F1D16068F9F75AF844
:1094E000EDE7207A00F0E8FFA37A8342EAD1002D6D
:1094F000E5D0207A00F0E0FFA37A8342DFD1002F8D
:10950000DDD1D8E7F7B56E4686E806000446454942
:1095100045489DF820501F4606F0B4FB3046FBF747
:1095200079FD37B1414938460AF093FC08B900206B
:1095300051E06368002BFAD0B4F9080000F0CEFFC8
:109540000028F4D13046FBF767F9002845D13046B2
:10955000FBF7C8FB012840D010D302280DD00446E9
:109560003349314806F08EFB0A2221462E4806F088
:10957000F2FB2D4806F096FBD9E7D5B10021304625
:10958000FBF78EFA054658B16068F8F7EBFF08BBA9
:10959000646800F087FF01462046F8F7FBFF19E0FA
:1095A00001466068F8F7F6FF29462046FFF7AAFE55
:1095B00010E06068F8F758FE15280BD8012303FA6D
:1095C00000F01C4B184205D029463046FBF768FADC
:1095D0000028D9D1012003B0F0BD3046FBF7CCFA0A
:1095E00015280DD80125144F05FA00F00740CBD1FE
:1095F000430705D539466068F8F7CCFF3946D4E70C
:109600000E49094806F03EFB3046FBF7B5FA0A2240
:109610000146054806F0B8FB034806F043FB012469
:109620009EE700BF379201006803002019920100F5
:10963000BA7901000240380002C03800AD7901005B
:1096400007B5002300931A461946034806F0D2FADC
:1096500003B05DF804FB00BF0405002090B1C368AF
:109660007BB11A7C02F00F02042A01D1586948B973
:10967000D86838B1037C03F00F03042B01D1406993
:10968000704700207047000030B52DED028B054675
:1096900087B008EE101A002851D0324B1B68002BFF
:1096A0004DD0FFF7DBFF30490446304806F0EAFAB8
:1096B00018EE100A08F00EFE0223024600932B4813
:1096C0000B4606F01DFC2A49284806F0DBFA2968FB
:1096D000264806F0E0FA2749244806F0D3FADFEDE1
:1096E000267AB4EE678AF1EE10FA2CD0DFED237AF9
:1096F000B4EE678AF1EE10FA25D0B5EE408AF1EEAD
:1097000010FA20D01CB12146184806F0C4FA1748B8
:1097100006F0C8FA04AC18EE101A02A8FAF70BFF0C
:10972000032202A92046FBF7E1FA0023CDE900332A
:109730004FF0FF3194E80C00284600F0EFFC07B032
:10974000BDEC028B30BD002CF9D00D49074806F066
:1097500099FA2146054806F09EFA044806F0A2FA56
:10976000EDE700BF24040020A89201006803002058
:1097700047940100359401000000FEC20000AA4297
:10978000AD9201002DE9F043284F386889B00028D8
:1097900046D0274E3368002B45D001F049F92549C2
:1097A0002548DFF8A080DFF8A090234C06F06AFA85
:1097B000214806F077FA01A9386801F0CBFA0028B1
:1097C0002DDD03AA082101A800F078FA002303AADE
:1097D00031688DF81C30404604F04BFF4946054681
:1097E000204606F04FFA03A9204606F054FA8DB140
:1097F0002846FFF733FF05460028DCD00F492046F6
:1098000006F040FA2946204606F045FA204606F0C2
:1098100049FAD0E70A49204606F034FAF6E7012073
:1098200009B0BDE8F0831846FAE700BF180500202C
:1098300024040020C9930100B4030020FE7E01002F
:10984000DC9301006C070020A8920100FFF79ABF8B
:109850002DE9F3413E4C2368002B77D13D493E482A
:1098600006F010FA3C4806F01DFA142007F09CF8A8
:10987000054601F097F83948256000F0EDFE2068B4
:1098800001F0AAF800284AD03549364806F010FA07
:10989000206801F0E7F9206801F0AAF8206801F0DB
:1098A00025FA002839D030492B4806F001FA2F4E0E
:1098B0003068002847D02E4D2F687FB91C2007F054
:1098C00073F82168804601F0C9FA4046C5F8008067
:1098D00001F0A4FB3946286801F0DEFB3368DFF8AD
:1098E000A480DC681C4F336883B37CB3694620686E
:1098F00000F01CFA50B34146384606F0C3F921681F
:10990000384606F0C8F9384606F0CCF90C2269460C
:10991000286801F040FB6468E5E71649C4E700F0F9
:10992000DFFD206801F058F8054638B112490D48AE
:1099300006F0A8F90B4806F0B5F9B8E70F4910484A
:1099400006F0B6F9284602B0BDE8F0810120FAE73A
:10995000180500200B9301006803002090050020EB
:1099600031930100B403002050930100240400202F
:109970002005002064930100799301009693010073
:1099800084030020B2930100034B0146186808B11C
:1099900001F018B8704700BF1805002037B52D4CEE
:1099A000206801F011F8022805D0042811D0012800
:1099B00018D129490EE02949294806F063F92848B9
:1099C00006F070F9206801F091F941F2883003B097
:1099D00030BD2449224806F055F9214806F062F9C5
:1099E00000F07EFD204D2B6813B1204B1B683BB966
:1099F0001F491B4806F046F9194806F053F9E4E7F9
:109A00001C4C22683AB91A7C02F00F02062A02D1D5
:109A1000DB6803B123601848FFF7B6FF2368A3B1E2
:109A20006946186800F082F978B19DF80030282B5B
:109A30000BD16946286801F0BFFB01462068FFF79B
:109A400023FE6946286801F05DFB23685B6823609C
:109A5000BBE700BF18050020EB920100BE92010099
:109A600084030020D292010020050020240400205D
:109A7000FD92010014050020916B000038B5094CDF
:109A8000256806F0FBFE0023014641F28832284695
:109A900000F02AFB20B1FFF781FF06F0EFFE206007
:109AA00038BD00BF1C05002007B5002300931A46EF
:109AB0001946034806F09EF803B05DF804FB00BFAA
:109AC0000C050020704770477047704707B50023AA
:109AD00000931A461946034806F08CF803B05DF867
:109AE00004FB00BF24050020174B1B7870B504460B
:109AF0000D469BB1154B027A1B789A420ED8144A38
:109B00000A291368164616D1124A0021D154406919
:109B100010B1217A06F034F800233360E06840B1D8
:109B20000D4B227A1B789A4203D8036829461B689A
:109B30009847012070BD4E2BF0DC0D291FBF591C2A
:109B40001160044AD554E9E778040020060000209B
:109B500084050020340500200500002030B50025D4
:109B600045604361034D9DF80C300560C160027291
:109B7000037430BDEC93010007B5002300931A462F
:109B80001946034806F036F803B05DF804FB00BF41
:109B90002C050020D0E90423D05C70470368DB6803
:109BA0001847704700207047184B70B50E4619686B
:109BB000044679B10B7C03F00F03062B0AD1324621
:109BC000134804F056FD037C03F00F03042B01D16E
:109BD000406970BDB4F924506B1E9BB20C2B13D896
:109BE0000C4930460AF035F970B90B492F2305EBC3
:109BF000850584F826300622294404F127000AF05E
:109C000084F904F12600E4E70020E2E7980400204C
:109C10006C07002009950100BC9401002DE9F0417A
:109C2000056A044625B1002303622846BDE8F08199
:109C3000D0E90432995C242934D1991849787B29D8
:109C400030D1023213442E461A4613F8017B4FB32B
:109C50007D2F0FD00136F7E7A26122693AB163691F
:109C6000D25C12B10133636125E02261DDE74FF080
:109C7000FF35DAE7B6B14FF0000882F8008061697D
:109C80002269236802319B69114420469847D4E930
:109C9000043233441344C4E906089F7063690333F4
:109CA0001E446661A269002AD7D0E369D25C002A0B
:109CB000D2D00133E3611546B7E7000070B5D0B1EB
:109CC000CAB14D1E0C4E441E13462844844203F173
:109CD00002030CD014F8015F2D11755D03F8025CCE
:109CE000257805F00F05755D03F8015CEEE709B214
:109CF000002302F8113070BDA2940100A0F16103AD
:109D0000052B02D85738C0B27047A0F14103052B8C
:109D100001D83738F7E73038C0B2092805D919B16A
:109D200001230B70002070470846704737B50023A9
:109D30008DF80730F9B1E0B1851C4C1E00F112021C
:109D400015F8020C0DF10701FFF7D8FF000104F828
:109D5000010F0DF1070115F8010CFFF7CFFF237874
:109D60000235184395422070EAD19DF8070080F033
:109D7000010003B030BD0846FBE738B50546D8B151
:109D80000468ACB124789CB1286803783BB12D2BD2
:109D900005D0303B092B02D901302860F4E708F0E8
:109DA0005EFE2C21044628680AF046F810B92860A7
:109DB000204638BD0130FAE70446F9E72DE9F743BC
:109DC0000E46002206210746FAF7A8FB002E55D0C2
:109DD0003368002B52D01B78002B4FD0D6F8008070
:109DE00098F800404CB32D2C6CD0303C092C03D992
:109DF00008F101033360F1E74146002400220FFA25
:109E000082F9013211F80930303B092BF7D92E21A4
:109E100040460AF011F818B3002211B2431801327B
:109E20005B78303B092BF8D94378A3F13002092A3B
:109E300001D82F2B03D8002204E0A146E7E7392BF5
:109E400088BF09220A2555438278A2F13003092BE5
:109E500005D82F2A16D9392A88BF09231D4499B954
:109E6000404608F0FCFD394602466846FAF7A7FE70
:109E70002C21306809F0E0FF10BB3060384603B099
:109E8000BDE8F0830023E9E7022940460EDCB9F182
:109E9000070F0BDC08F0E3FD6422424304B16D427E
:109EA0002A4439466846FAF7B0FEE1E708F0D0FDEB
:109EB00008F060FD394602466846FAF78CFED7E79F
:109EC0000130DAE708F10101012497E708B5002025
:109ED0000AF0FAFFADEB000008BD704730B5441E34
:109EE000224612F8013F002BFBD11A460A2514F82E
:109EF000010F70B1032A14DC2E2806D1FF2B10DCD1
:109F00008818013203710023F1E7303805FB0303A1
:109F1000EDE7FF2B04DC032A02DC114401200B7166
:109F200030BD0020FCE700002DE9F3410024DFF8FC
:109F300040800C700D461746061D0A2201A916F82E
:109F4000010B08F0A5FF3A4601A9284609F0B7FF22
:109F5000032C04D03A464146284609F0B0FF0134AC
:109F6000A3B2042B1CB2E8D1284602B0BDE8F081B0
:109F7000F48D01002DE9F0410E4D0F4FDFF83C80CC
:109F800006460024032C0ED033190A2219792846DC
:109F900005F0BFFE41462846013405F073FE042C4F
:109FA000F0D1BDE8F081F1790A22284605F0B1FE32
:109FB0003946F0E7B40300204C7B0100F48D01002A
:109FC0002DE9F047DFF8F0A0DAF8005004460E461D
:109FD00017469946002D49D02B7C03F00F03062B22
:109FE00043D12C4A2C48294604F043FB022F8046DB
:109FF00037D0032F37D1294ADAF80010264804F069
:10A0000038FB0546B8F1000F30D098F8103003F057
:10A010000F03042B2AD1D8F814103246204609F039
:10A0200074FF32461E49204609F049FF0DB32B7CD0
:10A0300003F00F03042B1CD169693246204609F056
:10A040003EFF32461649204609F039FFB9F1000FAC
:10A0500004D032464946204609F031FF2046BDE88B
:10A06000F087104AC8E70025CCE7002532460E49A4
:10A07000D4E7022F0AD0032F05D0012FE1D10B4BDB
:10A0800032461968DAE732460949D7E732460949C4
:10A09000D4E700BF989401006C0700205D90010098
:10A0A000808701009D94010002950100800300203B
:10A0B000B6940100B3940100980400200B460A22D4
:10A0C0000146184606F031BC10B5054C054920463E
:10A0D00005F0E1FD2046BDE8104005F0E3BD00BFFE
:10A0E000680300206394010010B54AB102441BB11B
:10A0F000B2FBF3F403FB14228A4208D288420AD945
:10A10000012010BD884294BF00200120F9E782425F
:10A11000F8D80020F5E78242F5E700002DE9F04F7E
:10A12000A5B002AF0C4687E80C00DDE92EAB064671
:10A13000002800F0DF80037C03F00F03062B1CD8FF
:10A14000DFE813F0D3001B001B001B00CF0007004B
:10A150001D00894BC5681A7801321A701E464DB130
:10A16000CDE900AB284697E80C002146FFF7D6FF63
:10A170006D68F4E73378013B337000200EE0014650
:10A180007E4A7F4804F075FA054650B10023CDE9B8
:10A190000033214697E80C00FFF7C0FF25B0BDE86B
:10A1A000F08F784A7648314604F063FA764A814661
:10A1B0003146734804F05DFA80461CB1012C74D01E
:10A1C0002C460CE0714A6E48314604F052FA0546BE
:10A1D0006F4A6B48314604F04CFA044605B93546DF
:10A1E000002C08BF3446B9F1000F00F08180B8F1AF
:10A1F000000F08BFD84635B12B7C03F00F03042BAA
:10A200000CBF6D690025002C77D0237C03F00F0371
:10A21000042B72D1D4F814A00026B9F1000F00F07D
:10A22000C980002D00F088805A495B4805F02AFD5E
:10A23000D9F81410584805F02EFD5849564805F035
:10A2400021FD2946544805F026FD534805F02AFD16
:10A250003846FAF7DFFEB8F1000F40F00D8199F8AB
:10A26000103003F00F03042B40F00481D9F81410D0
:10A2700014A8F8F77FFA14A8F8F7BAF988B1FFF72D
:10A2800025FEB0F5966F044664DA4549454805F069
:10A29000F9FC0A222146434805F05DFD414805F0DE
:10A2A00001FD14A8F7F7D6FFE4E03F4A34483146F1
:10A2B00004F0DFF93D4A05463146314804F0D9F94A
:10A2C0000446002D40F0DC80304A2D48314604F031
:10A2D000D0F90546002C3FF47BAF002808BF354677
:10A2E00081E70024A046A14679E700242546A04640
:10A2F000D1467CE7D846D14605461022002300937C
:10A300000DEB02014FF440733846FAF76FFD8246B9
:10A310003846FAF7E7FC06B2002E7FF47EAF3846E7
:10A32000FAF77AFA30B93846FAF787FA002818BFF0
:10A33000022672E7012670E71D49174805F0A2FCC6
:10A34000D9F81410144805F0A6FC1449124805F079
:10A3500099FC7DE72DB10022294614A8F9F7E2FC0B
:10A360009FE70123009301952B4697E8060014A868
:10A37000F8F764FE95E700BF65030020FF7A01004F
:10A380006C070020F67A0100387B01001894010068
:10A390001D9401002C9401006803002033940100F7
:10A3A0004A940100840300202294010027940100B4
:10A3B00038940100B8F1000F5CD0BAF1000F59D009
:10A3C00098F8103003F00F03042B4FD1D8F8143055
:10A3D000ADF8446000244FF47A72CDE909422A4A6C
:10A3E0000892CDE90C3414AA4023214608A8CDE9EF
:10A3F0000E44109405F02AFF24AB1844234900F8BA
:10A40000404C234805F03EFCD8F81410204805F0D5
:10A4100042FC20491E4805F03EFC14A91C4805F0EA
:10A420003AFC1D491A4805F02DFC5146184805F024
:10A4300032FC174805F036FC184804F06BFCA8B154
:10A44000174B93F900308BB92F2114A809F0F4FCB5
:10A4500030B9D8F814300322402114A8FFF7B0FD1A
:10A460000123524614A90D4804F0B1FEB9F1000FC2
:10A470007FF4F5AE012091E6BAF1000FA0D1EEE62F
:10A4800000287FF4B0AEA3E6FC93010042940100E3
:10A49000680300203594010033940100E00300209C
:10A4A000B003002010B5044606F0E8F9E040431E72
:10A4B000033388BF012010BD054B1A68054B53F8C4
:10A4C000201001238B40134214BF0120002070474D
:10A4D000080500503C98010001207047002070479B
:10A4E00038B52149214805F0E3FB0121204800F05F
:10A4F0007CF91F4800F006F90121172006F0ACFB9B
:10A500000021162006F0A8FB142400252946172058
:10A5100006F0CAFB0A2006F0E5F9013C85F00105CA
:10A52000F4D11420134C06F0DDF9114800F094F832
:10A530002068A0B100F050FA88B1206800F092FBCA
:10A540000D490A4805F0B4FB206800F051FA206874
:10A5500000F0CCFB28B10949044805F0A9FB012013
:10A5600038BD0749F8E700BF739401006803002075
:10A5700090050020180500207D94010050930100F3
:10A580006493010007B5002300931A461946034857
:10A5900005F030FB03B05DF804FB00BF8805002028
:10A5A0002DE9F84380460D46174601EB02090C469B
:10A5B0004C45A4EB05060BD0D8F8003014F8011B6D
:10A5C0001B68404698470028F2D13046BDE8F88322
:10A5D0003E46FAE77047203005F0BDBC203005F05C
:10A5E000ACBC203005F0BDBC38B5437F0D460BB97F
:10A5F000002038BD00F16804204605F0BAFC0028B0
:10A60000F6D12046294605F089FC0120F1E700003B
:10A610002DE9F0411E4600254FF47A73C0E901533D
:10A620000C4B044640F8203B8846174605F06DFC6D
:10A6300004F1680005F069FC9DF8183063769DF818
:10A640001C302676C4E90487A37665772046BDE8EA
:10A65000F08100BF18950100817E284A0123C3764E
:10A6600070B552F82140417E52F821104FF0A045BC
:10A6700004F5E07401F5E07140F20C6645F82460E1
:10A6800045F8216001694FF0CC74C1F82445016997
:10A690000624C1F80045847E016952F82440C1F8BF
:10A6A0000845447E016952F82420C1F80C2590F930
:10A6B0001820510902F01F0293406031104A42F8FD
:10A6C000213090F91830002BBDBF03F00F0302F6C4
:10A6D000FC32D2189B18B5BF40234022137683F872
:10A6E000002390F918300122590903F01F0302FAE0
:10A6F00003F3034A42F8213070BD00BF3C980100CB
:10A7000000E100E0C37E23B103690022C3F8002505
:10A7100070474269C2F8003570472DE9F0410446A0
:10A7200088461F461546002A50D000F120063046C4
:10A7300005F0FFFB2369C3F88885236901221A62AB
:10A740002369C3F834652369C3F8385523691A604F
:10A750002269D2F84C311BB9D2F82431002BF8D041
:10A760000023C2F84C312269D2F85C311BB9D2F80F
:10A770002431002BF8D00023C2F85C3122696FB974
:10A78000D2F8243153B90123D3612369D3F8482186
:10A79000002AFBD00022C3F8482109E001235361BD
:10A7A0002369D3F80421002AFBD00022C3F8042136
:10A7B0002369D3F8242112B10022C3F8242123698C
:10A7C000D3F83C052066C0B2BDE8F0811046FBE737
:10A7D0000123FFF7A2BF10B5044680F8B01068301F
:10A7E00005F0A7FB0123637710BDF8B5002343777D
:10A7F000036990F8B020C3F88825036901261E621A
:10A80000036900F168050446C3F8445528460F461D
:10A8100005F0A1FB2369C3F8480523699E602369FD
:10A82000D3F850211AB9D3F82421002AF8D00022F5
:10A83000C3F85021284605F08EFB236930B1D3F8C8
:10A8400060211AB9D3F82421002AF8D00022C3F8D5
:10A85000602123696FB9D3F8242152B90122DA614A
:10A860002369D3F84821002AFBD00022C3F84821ED
:10A8700009E001225A612369D3F80421002AFBD0A0
:10A880000022C3F804212369D3F8240168B100220F
:10A89000C3F824212369D3F8C404C3F8C4040228EC
:10A8A00003D004280CBF03200420F8BD0121FFF7CA
:10A8B0009CBF70B54369D3F86421044692B100226D
:10A8C000012500F12006C3F864210577304605F024
:10A8D00030FB6369C3F8346563694022C3F83825E7
:10A8E00063691D636369D3F86821DAB10025C3F891
:10A8F000685104F16806012363772577304605F037
:10A9000018FBD4F8B43003B19847636965773046D3
:10A91000C3F8446505F01FFB6369C3F84805636924
:10A9200001225A636369D3F8042162B10022C3F89B
:10A930000421237F3BB16369D3F83C05D4F8B830D8
:10A94000206603B198476369D3F8242152B10022ED
:10A95000C3F824216369D3F8D024C3F8D0246369F1
:10A9600001225A6170BD00000148FFF7A2BF00BF7D
:10A970009005002007B516231722CDE900324FF0CD
:10A980004022042311460348FFF742FE03B05DF85E
:10A9900004FB00BF900500200148FFF787BF00BF00
:10A9A0009005002010B54FF4C053038000230446E7
:10A9B000837003610248FFF74FFE204610BD00BFC1
:10A9C0009005002001617047807870474178014808
:10A9D000FFF701BF9005002008B5FFF7F7FF034818
:10A9E000FFF764FFB0FA80F0400908BD9005002031
:10A9F000012303707047FF23C37200230373C370E6
:10AA0000037143718371C371037243728372704720
:10AA100010B5064A01440023884204D010F8014BC7
:10AA20006340D35CF8E7184610BD00BF30950100C5
:10AA3000FFF7E1BF38B5084C0D46FFF7C7FFE1212E
:10AA40002046FFF7D1FD29462046FFF7CDFDBDE8A2
:10AA50003840FFF7A1BF00BF9005002010B5054C9E
:10AA6000417801222046FFF7B3FE2046FFF7B6FDEE
:10AA7000C0B210BD9005002010B5F0210446FFF7CC
:10AA8000D9FF2046BDE81040FFF7E8BF70B5044687
:10AA900005F0F4FE0025064605F0F0FE801BB0F53B
:10AAA0007A7F4DD2236903B198472046FFF7E4FF30
:10AAB00010F00103054605D1A278012A00D1A37048
:10AAC000284670BD1420013800BF00BF00BF00BF82
:10AAD00000BF00BF00BF00BF00BF00BF00BF00BF7E
:10AAE00000BF00BF00BF00BF00BF00BF00BF00BF6E
:10AAF00000BF00BF00BF00BF00BF00BF00BF00BF5E
:10AB000000BF00BF00BF00BF00BF00BF00BF00BF4D
:10AB100000BF00BF00BF00BF00BF00BF00BF00BF3D
:10AB200000BF00BF00BF00BF00BF00BF00BF00BF2D
:10AB300000BF00BF00BF00BF00BF00BFC3D1ABE775
:10AB40000123BCE710B5E1210446FFF773FF20465F
:10AB5000BDE81040FFF782BF10B50446FFF796FF2F
:10AB60002046FFF733FF96210648FFF73DFDFFF72C
:10AB700013FF2046FFF78AFF2046BDE81040FFF78D
:10AB8000E1BF00BF90050020FFF7E6BF10B5C3216D
:10AB90000446FFF74FFF2046BDE81040FFF75EBFB9
:10ABA00038B504460D46FFF771FF2046FFF70EFF4C
:10ABB000D2210C48FFF718FDE94345EA0111C9B25B
:10ABC0000848FFF711FDFFF7E7FE2046FFF746FFB5
:10ABD000A84202D00423A37038BDA378042BFBD174
:10ABE0000023F8E79005002010B50446FFF7CEFFDC
:10ABF00040F00401C9B22046BDE81040FFF7D0BFC5
:10AC000070B5164604460D46FFF740FF16B12046C4
:10AC1000FFF7EAFF2046FFF7D9FEA5210548FFF719
:10AC2000E3FC29460348FFF7DFFCBDE87040FFF76F
:10AC3000B3BE00BF9005002070B500220C46552120
:10AC40000646FFF7DDFF651E073415F8011F0022D9
:10AC50003046FFF7D5FFA542F7D170BDFFF7ECBF37
:10AC6000FFF7CEBF10B50446FFF7B0FE2046002226
:10AC7000F021FFF7C5FFBDE81040FFF78DBE0000D3
:10AC800070B5164605460C46FFF700FF16B128467C
:10AC9000FFF7AAFF2846FFF799FE87210648FFF72E
:10ACA000A3FC002C0CBF214680210348FFF79CFC2D
:10ACB000BDE87040FFF770BE9005002010B500227F
:10ACC00004460121FFF7DCFF2046FFF7DFFEC0F35B
:10ACD000401010BDFFF7F2BF10B50446FFF756FF56
:10ACE00020460021BDE81040FFF75ABF38B50446A2
:10ACF000FFF7CCFEC30729D42046FFF7EDFF20461F
:10AD0000FFF7C4FE2046FFF761FEB4211048FFF7AD
:10AD10006BFCFFF741FE2046FFF7B8FE10F004037E
:10AD2000054602D00223A37002E0A278022AFAD0DC
:10AD3000237843B12046FFF729FF40F00101C9B253
:10AD40002046FFF72DFFC5F3400038BD0020FCE78B
:10AD5000900500202DE9F74F057B04460F46002D96
:10AD60006BD1FFF7C3FF002869D02046FFF78EFEA6
:10AD70002A46F0212046FFF743FFDFF8C8804FF056
:10AD8000FF394FF0010A94F90B30EEB24FEAD60BBF
:10AD90009D4206F007060AFA06F623DA04EB0B03D7
:10ADA000DB78334020460193FFF770FE2046FFF723
:10ADB0000DFE78214046FFF717FC019B002B0CBFCE
:10ADC000194680214046FFF70FFCFFF7E5FD2046BE
:10ADD000FFF75CFE820600F0400307D55BB16FF021
:10ADE000010027E00CBF01230023DBE71BB90306AA
:10ADF00058BF4FFA85F904EB0B03010693F90320C2
:10AE000076B205F101054CBF3243B243402DDA70F2
:10AE1000B9D1B9F1FF3F04BF0123237384F80B902C
:10AE2000E31C013F0B3413F8012B07F8012FA34259
:10AE3000F9D1012003B0BDE8F08F0020FAE74FF010
:10AE4000FF30F7E79005002008B5FFF783FF20EA01
:10AE5000E070C0B208BDFFF749BF7047054A826184
:10AE60000022027102700922427001228160827008
:10AE7000C27070475BAE000010B50C46204607213B
:10AE8000FFF7C6FDE3791B1A5842584110BD70B553
:10AE9000044680680E461546FFF7DDFFB8B131461F
:10AEA000A068FFF7DBFE0022BE21A068FFF7D8FEF6
:10AEB0006E1E0835A068FFF767FE06F8010FAE4268
:10AEC000F8D1A068FFF7C7FF431E5842584170BD34
:10AED00010B51446FFF7DBFF38B108212046FFF715
:10AEE00097FD237A1B1A5842584110BD70B504468D
:10AEF0000D4680681646FFF7AEFF2946A068FFF7AB
:10AF0000ADFE00224E21A068FFF7AAFE0022B17814
:10AF1000A068FFF7A5FE0022F178A068FFF7A0FE69
:10AF20002B78102B04D000223179A068FFF798FE0F
:10AF3000A068FFF790FF2946A068FFF78FFE2278F0
:10AF4000A0684821FFF78CFE142005F0CBFC237885
:10AF500013B10A2005F0C6FCA068BDE87040FFF7F9
:10AF60007ABF38B504460D468068FFF774FF29465E
:10AF7000A068FFF773FE0022B421A068FFF770FEFF
:10AF8000A068FFF7A7FE0546A068FFF764FFB5FAC3
:10AF900085F0400938BDF0B585B0144601AA0746D2
:10AFA0000E46FFF795FF054690B13378102B0FD072
:10AFB0000B2C10D00C2C03D00A2C0ED13F2300E018
:10AFC0007F2301AA314638468DF80830FFF78EFFFF
:10AFD000284605B0F0BD5F23F3E71F23F1E71FB557
:10AFE0000B78102B10D001AAFFF772FF78B19DF8F3
:10AFF00008303F2B0ED003D81F2B0DD0002006E0C9
:10B000005F2B03D07F2BF9D10C2000E00B2005B083
:10B010005DF804FB0A20FAE70920F8E7F0B587B0ED
:10B02000044605F02BFC00F51C55A068FFF700FD59
:10B03000002310352371012601A9A068FFF704FF42
:10B0400040B305F01BFCA84224D201A92046FFF71B
:10B0500013FF0028F0D023782BB901A92046FFF771
:10B0600080FF00B1267003AA01A92046FFF70FFF59
:10B0700001A920466778FFF7B2FF874205D96078BB
:10B080002379607001332371D6E701A92046FFF7C9
:10B09000A6FFF5E707B0F0BD817070471FB501AAA4
:10B0A000FFF7F5FE9DF80400003018BF012005B041
:10B0B0005DF804FB0939C9B20229F8B598BF104BF5
:10B0C0000546164694BF33F9114040F2EE248AB18A
:10B0D000C3787BB103786BB905F0D0FB07463146E6
:10B0E0002846FFF7DBFF20B905F0C8FB001BB8427C
:10B0F000F5D3F8BD2046BDE8F84005F0F3BB00BF2E
:10B1000030960100F8B504460F46FFF768FF064683
:10B1100010B900252846F8BDA068FFF79CFE00285E
:10B12000F7D03946A068FFF799FD2278A06844213E
:10B13000FFF796FDA5782DB13A4631462046FFF738
:10B14000B9FFE7E70125E5E710785378C00040EA4A
:10B15000C3200B78102B00B20BD1D1799379C000AA
:10B16000CB1ADB0120F07F0093FBF1F3103B184476
:10B1700000B2704730B585B001AA04460D46FFF70E
:10B18000A7FE30B101AA29462046FFF7DDFF05B032
:10B1900030BD0148FBE700BF80E4FFFF10F5DC5F36
:10B1A000CABF07EE900ADFED037AFAEEEC7A17EEEB
:10B1B000900A70470000FEC208B5FFF7DBFFBDE84C
:10B1C0000840FFF7EBBF01460422012001F0AABAB4
:10B1D00001460422052001F0A5BA014606220920F5
:10B1E00001F0A0BA014604220F2001F09BBA000032
:10B1F0002DE9F04F3D4E3E4C336813F0010387B00C
:10B2000082468B4615460ED1E3644FF47A7323656C
:10B21000384BA36404F15C0004F0E4FC082384F8D8
:10B22000683001233360344E346001F04DFC002758
:10B23000002859D04FF000494FF00208CDF80C908B
:10B2400005978DF8108003AC94E80E002B4805F0AC
:10B25000B5FD5046FFF7C1FF3B463A4639460097D9
:10B26000204604F0C7FC04A8FFF7BCFF234805F004
:10B27000B1FD2B465A465146306801F08FFF012838
:10B2800005462DD1CDF80C9005978DF8108094E8E7
:10B290000E001A4805F092FD3168204601F0E5FCE9
:10B2A00004A8FFF79FFF3168204601F0ECFC04A8DA
:10B2B000FFF789FF3168204601F0DEFC04A8FFF7A4
:10B2C00087FF0E4805F086FD3168204601F0E2FC5C
:10B2D0000B4B049A5A6005F0EBFA80B200F08EFD39
:10B2E000284607B0BDE8F08F0546F9E74C06002078
:10B2F000640600209C960100600600204C08002097
:10B3000058060020F0B585B007460E4614461D4687
:10B3100001F0DAFB00B34FF00043019300230393E5
:10B3200002238DF8083004AB13E90E000B4805F03A
:10B3300045FD3846FFF751FF301DFFF753FF281D2D
:10B34000FFF741FF0A980430FFF742FF034805F07A
:10B3500041FD034B62685A6005B0F0BD4C08002007
:10B3600058060020F0B58DB01D4600230F4600930F
:10B37000FF230446164619461A4602A804F03AFC72
:10B380000B4B7A680493CDE905237268CDE9072356
:10B390006A68CDE90923039B0B930AAB009306AAC5
:10B3A00008AB04A92046FFF7ADFF0DB0F0BD00BF0C
:10B3B000AC98010000B50B4B4968526889B0CDE9E3
:10B3C0000231CDE905230493012301918DF8073063
:10B3D000019B079304AA06AB02A9FFF7C3FF09B0BC
:10B3E0005DF804FBAC9801007FB5094B4A680493F3
:10B3F000CDE90232012301928DF80730019B0593BC
:10B4000004AA02A9FFF7D6FF07B05DF804FB00BF4E
:10B41000AC98010008B501F0BDFB012803D002285B
:10B420000CBF0220002008BD7FB51E4E30680028EA
:10B4300036D001F0CBFE0228044601D004282CD1DE
:10B440004FF00043019300230393022301AD8DF8D5
:10B45000083095E80E00144805F0B0FC3168284625
:10B4600001F003FC02A8FFF7BDFE3168284601F099
:10B470000AFC02A8FFF7A7FE3168284601F0FCFB92
:10B4800002A8FFF7A5FE084805F0A4FC316828468D
:10B4900001F000FC054B029A5A60204604B070BDD2
:10B4A0000446FAE7600600204C08002058060020F9
:10B4B00030B585B0044604F095FB4FF0004301938E
:10B4C000002303930A4D02238DF8083004AB13E9DF
:10B4D0000E00284605F072FC0422A1180F2001F08E
:10B4E000D9F9284605F076FC204605B030BD00BFEE
:10B4F0004C08002030B585B0044604F073FB4FF0D3
:10B5000000430193002303930A4D02238DF8083072
:10B5100004AB13E90E00284605F050FC0422A118E4
:10B52000052001F0B7F9284605F054FC204605B087
:10B5300030BD00BF4C08002030B585B0044604F093
:10B5400051FB4FF000430193002303930A4D022364
:10B550008DF8083004AB13E90E00284605F02EFCE8
:10B560000422A118012001F095F9284605F032FCCB
:10B57000204605B030BD00BF4C08002007B50023B1
:10B5800000931A461946044804F034FB034803B0FC
:10B590005DF804EB04F026BB50060020580600209E
:10B5A000007C07288CBF00200120704781F001003B
:10B5B00070470846704708B50368DB6B984780F012
:10B5C0000100C0B208BD4182704713B502AB0268EA
:10B5D00003F8011D546819460122A04702B010BDAE
:10B5E000037C087C984204D107288CBF00200120EE
:10B5F000704700207047000010B50446007C072803
:10B6000016D800F0A1FD182806D80A4B23FA00F03E
:10B61000C04300F0010010BD1C2807D1236820465C
:10B620009B689847003018BF0120F4E70120F2E73B
:10B630000020F0E701001001F0B591B0044604A825
:10B640000F46164604F0CEFA00224FF47A73CDE985
:10B6500008230CA8184B079304F0C4FA0823684683
:10B660008DF83C3004F0BEFA207C072807D800F0A3
:10B670006BFD10B1207C00F0CBFD082323740F4B31
:10B680000F4D5B68039302A904A8029501F0DDFD4C
:10B6900041F288336A46394604A801F05FFF40B1A1
:10B6A0002368019A9B6903920295324602A92046BB
:10B6B000984711B0F0BD00BF9C96010058060020CD
:10B6C000AC98010008B5007C072802D800F02EFFD6
:10B6D00008BD0020FCE710B50446207C07280BD8E5
:10B6E00000F032FD172801D01C2805D1207C00F085
:10B6F0001DFFB0F5006FF0D310BD38B50546007CD6
:10B700000728144605D892B200F092FE10B9012322
:10B710006B600024204638BD08B5007C072802D89D
:10B7200000F02EFE08BD0020FCE7007C072802D8B0
:10B7300012B200F08BBD0020704707B501220DF159
:10B740000701007C00F082FD0028CCBF9DF80700B7
:10B750004FF0FF3003B05DF804FB10B5037C072BFE
:10B76000044602D94FF0FF3010BD03689B6898472C
:10B770000028F7D0207C00F02FFEF5E738B504460E
:10B78000007C07280AD800F043FD05F077F805464D
:10B79000207C00F0D9FC10B90823237438BDFBF7D6
:10B7A000FBF9012005F09EF805F068F8638A401B5C
:10B7B0009842EDD3207C00F0E5FCEDE77FB5044630
:10B7C000007C07280D46164607D800F0BDFC10B1D6
:10B7D000207C00F01DFD082323740021684604F03E
:10B7E00015FA6A68019B9A4202D1002004B070BD2C
:10B7F0004FF0FF3102A804F009FA6A68039B9A42ED
:10B80000F3D00021212000F003FB07282074ECD89E
:10B81000291D324600F0D4FC05F030F80546207CA6
:10B8200000F092FC172815D01C2813D00028DCD07B
:10B8300005F024F8638A401B984205D8FBF7ACF961
:10B84000012005F04FF8EAE7207C00F09BFC08237C
:10B850002374CAE70120C9E710B41446064A1278D7
:10B8600001EB022101EB00201A46214680B25DF86F
:10B87000044B01F00FB800BF300700207FB5037CF8
:10B88000072B05464FF000041BD84FF0004302265B
:10B890000394019301AC8DF8086094E80E000A4807
:10B8A00005F08CFA334622460421287CFFF7D4FFAA
:10B8B0009DF804309DF80540034844EA032405F050
:10B8C00089FA204604B070BD4C0800207FB50B7C7F
:10B8D000072B05460E4605D9002104F097F92846A6
:10B8E00004B070BD4FF00043019300230393022383
:10B8F00001AC8DF8083094E80E00084805F05EFAB7
:10B90000042322460C21307CFFF7A6FF034805F0F4
:10B9100061FA2146284604F07FF9E0E74C08002050
:10B920007FB5037C072B05464FF000041BD84FF072
:10B93000004302260394019301AC8DF8086094E85B
:10B940000E000A4805F03AFA334622461021287CB8
:10B95000FFF782FF9DF804309DF80540034844EA54
:10B96000032405F037FA204604B070BD4C080020CF
:10B9700007B5002300931A461946034804F03AF924
:10B9800003B05DF804FB00BFD006002003681B6B0A
:10B9900018470000024A02608A694260704700BF8F
:10B9A000AC980100808B7047008A7047408C7047CC
:10B9B00013B502AB026803F8011D54681946012251
:10B9C000A04702B010BD704710B5044690F82000A3
:10B9D000072804D800F0D6FB082384F8203010BDD7
:10B9E00038B5044690F8200007280D4601D800F02D
:10B9F000C9FB2946022000F00BFA072884F8200032
:10BA00004FF000009EBF60842582012038BD0000F9
:10BA1000F0B591B0044604A80F46164604F0E2F8CB
:10BA200000224FF47A73CDE908230CA8134B079337
:10BA300004F0D8F8082368468DF83C3004F0D2F8BA
:10BA40000F4B104D5B68039302A904A8029501F007
:10BA5000FCFB41F288336A46394604A801F07EFDBA
:10BA6000012808D12368019A1B6A03920295324685
:10BA700002A92046984711B0F0BD00BF9C96010076
:10BA800058060020AC98010008B50023C383043198
:10BA900090F8200000F09CFD08BD08B590F820004B
:10BAA00000F0C4FD08BD10B593B204460A46C18B30
:10BAB00090F8200000F060FDE38B0344E38310BDA9
:10BAC00013B5438C04461BB94FF0FF3002B010BDD4
:10BAD00001220DF1070190F8200000F0B7FB0028CB
:10BAE000F2DD638C9DF80700013B6384EEE710B53F
:10BAF000438C044613B94FF0FF3010BD934294BFFE
:10BB00001AB212B290F8200000F0A0FB0028F2DD7B
:10BB1000638C1B1A6384F0E708B590F82030072B7C
:10BB200005D8428C1AB1184600F056FC08BD4FF0FB
:10BB3000FF30FBE773B5044690F8200007280E4657
:10BB4000154601D800F01EFB094B00932A46736886
:10BB500001936946822000F017FA072884F8200034
:10BB60004FF000009EBF60840120258202B070BDAE
:10BB7000AC98010013B50446628C2AB123680021F9
:10BB80001B6B20469847F7E794F8200000F0F8FB7D
:10BB9000D8B10822694694F8200000F057FB00282D
:10BBA00013DD694604F1140004F03EF89DF804200A
:10BBB0009DF805309DF8070003EB0223A3839DF851
:10BBC000063000EB032080B2608402B010BD00009C
:10BBD00007B5002300931A461946034804F00AF8F3
:10BBE00003B05DF804FB00BFD806002007B5084B82
:10BBF0001B7801EB032101EB002001220DF107016D
:10BC000080B200F047FE9DF8070003B05DF804FB2A
:10BC10003007002007B5084B1B7801EB032101EB2F
:10BC2000002002A980B201F8012D012200F07AFD66
:10BC3000C0B203B05DF804FB3007002010B4144616
:10BC4000064A127801EB022101EB00201A46214638
:10BC500080B25DF8044B00F065BD00BF30070020E6
:10BC60002DE9F7430C4617461E4601AA022324215C
:10BC70000546FFF7F1FD9DF804209DF8053043EAE5
:10BC80000223224A1C441378332B0CBF05F1080011
:10BC900005F11000A4B2C002C4F30A0980B24844FE
:10BCA000372B904680B22DD009EB0603B3F5006F19
:10BCB00028DDC9F500691FFA89F94A46394600F0BE
:10BCC00031FD98F80030332B0CBF05F1080005F169
:10BCD0001000C002A6EB090280B292B207EB090184
:10BCE0003444A4B200F01EFD23128DF8043001AAE2
:10BCF0000223242128468DF80540FFF79FFF03B05B
:10BD0000BDE8F08332463946EAE700BF310700203C
:10BD100008B50321FFF76AFF08BD07B50B128DF8C0
:10BD200004308DF80510022301AA0421FFF786FFD5
:10BD300003B05DF804FB08B50A4604230C21FFF7A5
:10BD40007DFF08BD07B50B128DF804308DF8051086
:10BD5000022301AA1021FFF771FF03B05DF804FB75
:10BD600007B5022301AA2021FFF776FD9DF8040004
:10BD70009DF8053043EA002003B05DF804FB0000A5
:10BD800038B50546FFF7ECFF04462846FFF7E8FF05
:10BD90008442034604D1034B03EBC5039C8038BDAA
:10BDA0001C46F2E7E806002007B5022301AA262177
:10BDB000FFF752FD9DF804009DF8053043EA00208E
:10BDC00003B05DF804FB07B5022301AA2821FFF7A1
:10BDD00043FD9DF804009DF8053043EA002003B0C0
:10BDE0005DF804FB044B1B78332B0CBF0C30183070
:10BDF000C00280B2704700BF31070020034B1A8891
:10BE0000C0F30D0050401880704700BF08000020AC
:10BE10002DE9F043574B1B7885B081460F468BB315
:10BE2000332B4FF0004301934FF000054FF0020316
:10BE300003958DF8083001AE96E80E004E4814BF09
:10BE40004FF008084FF0040804F0B8FFECB22046A9
:10BE5000FFF75EFF7055D8B10135EBB29845F5D8C4
:10BE600000234FF03451F25C1D2ADCB203D821FAD2
:10BE700002F2D20708D40133DAB24245F3D33E4886
:10BE800004F0A8FF082465E01021204600F0C6FE5B
:10BE90003A4B002123F81410FA20013800BF00BFEC
:10BEA00000BF00BF00BF00BF00BF00BF00BF00BF9A
:10BEB00000BF00BF00BF00BF00BF00BF00BF00BF8A
:10BEC00000BF00BF00BF00BF00BF00BF00BF00BF7A
:10BED00000BF00BF00BF00BF00BF00BF00BF00BF6A
:10BEE00000BF00BF00BF00BF00BF00BF00BF00BF5A
:10BEF00000BF00BF00BF00BF00BF00BF00BF00BF4A
:10BF000000BF00BF00BF00BF00BF00BF00BF00BF39
:10BF1000C3D14A462046FFF77DFEFF22022120467C
:10BF2000FFF778FED7B139462046154DFFF7F5FEED
:10BF300000260121204600F071FE25F834602046DD
:10BF4000FFF741FF05EBC40358809E719E800A48AD
:10BF500004F040FF204605B0BDE8F083094B1A8885
:10BF6000013292B2B2F5404F38BF4FF440421A80CE
:10BF70001988D9E7310700204C0800204C07002021
:10BF8000E8060020080000202DE9F047694B1B78E7
:10BF900086B082460E461746A3B3332B4FF00043BC
:10BFA00003934FF000054FF0020305958DF8103014
:10BFB0000DF10C0898E80E005F4814BF4FF0080917
:10BFC0004FF0040904F0FAFEECB22046FFF7A0FEA1
:10BFD00008F80500E0B10135EBB29945F4D800232B
:10BFE0004FF0345118F803201D2ADCB203D821FA8F
:10BFF00002F2D20708D40133DAB24A45F2D34E48EE
:10C0000004F0E8FE082485E01021204600F006FE3A
:10C010004A4B002123F81410FA20013800BF00BF5A
:10C0200000BF00BF00BF00BF00BF00BF00BF00BF18
:10C0300000BF00BF00BF00BF00BF00BF00BF00BF08
:10C0400000BF00BF00BF00BF00BF00BF00BF00BFF8
:10C0500000BF00BF00BF00BF00BF00BF00BF00BFE8
:10C0600000BF00BF00BF00BF00BF00BF00BF00BFD8
:10C0700000BF00BF00BF00BF00BF00BF00BF00BFC8
:10C0800000BF00BF00BF00BF00BF00BF00BF00BFB8
:10C09000C3D152462046FFF7BDFDFF2202212046B4
:10C0A000FFF7B8FD002F39D039462046FFF735FE9F
:10C0B0005E238DF80630737903F07F038DF8073027
:10C0C000B3798DF808300125F3798DF80930311DE9
:10C0D0002046ADF80450FFF72EFE39462046FFF704
:10C0E00031FE0623194601AA2046FFF7A7FD29467F
:10C0F000134D0026204600F091FD25F834602046BF
:10C10000FFF761FE05EBC40358809E719E800A48CC
:10C1100004F060FE204606B0BDE8F087094B1A889F
:10C12000013292B2B2F5404F38BF4FF440421A800C
:10C130001988BAE7310700204C0800204C0700207E
:10C14000E80600200800002030B585B04FF000431D
:10C150000193002303930A4C02238DF8083004ABAB
:10C1600013E90E000546204604F028FE2846FFF796
:10C17000CFFD0546204604F02DFE284605B030BD13
:10C180004C08002030B585B04FF0004301930023E8
:10C1900003930A4C02238DF8083004AB13E90E0018
:10C1A0000546204604F00AFE2846102100F036FD20
:10C1B000204605B0BDE8304004F00CBE4C0800201D
:10C1C000F0B585B04FF000430193002303930F4D6A
:10C1D00002238DF8083004AB04460F461646284665
:10C1E00013E90E0004F0EAFD39462046FFF7A3FDEF
:10C1F00031462046FFF7A6FD2046042100F00EFD43
:10C20000284605B0BDE8F04004F0E4BD4C0800202D
:10C2100030B585B04FF000430193002303930A4CDF
:10C2200002238DF8083004AB13E90E0005462046C2
:10C2300004F0C4FD2846082100F0F0FC204605B0BB
:10C24000BDE8304004F0C6BD4C0800202DE9F04F99
:10C2500085B04FF000430193464E00230393022321
:10C2600036F830408DF8083001AB17460546894650
:10C2700041480ECB04F0A2FDA7420EDD2846FFF791
:10C2800093FD04462846FFF78FFDA042F9D106EB47
:10C29000C5039B79E41A26F835408CB92846FFF788
:10C2A00037FD142805D020B1B0F11C0418BF4FF0A1
:10C2B000FF34314804F08EFD204605B0BDE8F08F14
:10C2C0004FEAC50BBC4206EB0B03A8BF3C46B3F8D4
:10C2D0000280A7B2B9F1000F21D02846FFF782FDF6
:10C2E000264A1278C8F30A0A5044372A80B23DD051
:10C2F0001AFA84F2B2F5006F38DDCAF500631FFA4E
:10C3000083FA5246494600F0C5FA2846FFF76AFD0F
:10C31000A7EB0A02D14492B2494600F0BBFA06EB01
:10C320000B0236F835309179B844DB1B0F44BFB2AD
:10C330001FFA88F89BB2F92FA2F8028026F8353050
:10C3400000D8ABB95E440023B3714FEA28238DF8BF
:10C35000043001AA0223282128468DF80580FFF722
:10C360006DFC4021284600F059FCA2E73A46D3E78D
:10C3700097719EE7E80600204C0800203107002056
:10C380007FB5134D064635F83000F8B94FF000433D
:10C390000193022303908DF8083004AB0D4813E994
:10C3A0000E0004F00BFD3046FFF7FEFC044630465D
:10C3B000FFF7FAFCA042F9D1064804F00BFD05EBAB
:10C3C000C6039879201A80B225F8360004B070BDF3
:10C3D000E80600204C0800207FB54FF00043019391
:10C3E00000230393104D02238DF8083001AC94E82C
:10C3F0000E000646284604F0E1FC3046FFF7F2FC4A
:10C400000A4B03EBC60301225B88C3F30A031844FB
:10C41000214680B200F03EFA284604F0DBFC9DF88D
:10C42000040004B070BD00BF4C080020E8060020E6
:10C430002DE9F04FB2F5006F87B028BF4FF40062CE
:10C44000DFF8E49005468A46164603AC02234FF017
:10C4500000474FF000080397CDF814808DF8103096
:10C4600094E80E00484604F0A9FC2846FFF788FC33
:10C4700083462846FFF74CFC0190484604F0AAFC8E
:10C48000019B172B01D01C2B32D104F04DFAB34580
:10C49000DCD303974FF000080227CDF814808DF805
:10C4A000107094E80E00204804F088FC41463346A2
:10C4B00052462846FFF7D4FB2021284600F0AEFB69
:10C4C000DFF864804FF0004B02212846FFF78EFB17
:10C4D00010F0100A1FD12846FFF71AFC814648B910
:10C4E000114804F077FC4E46304607B0BDE8F08FA7
:10C4F0004646CEE7404604F06DFC04F015FACDF850
:10C500000CB0CDF814A08DF8107094E80E004046E1
:10C5100004F054FCD8E7102202212846FFF77AFBEA
:10C52000014804F057FCDFE74C08002030B585B027
:10C530004FF0004301930023039302238DF808304A
:10C5400004AB054613E90E000A4804F037FC284600
:10C55000FFF716FC04462846FFF7DAFB05460548B8
:10C5600004F038FC172D02D01C2D18BF00242046E3
:10C5700005B030BD4C0800202DE9FF411C464FF0AE
:10C580000043019300230393104D02238DF80830DC
:10C5900004AB06460F469046284613E90E0004F009
:10C5A0000DFC3046FFF7ECFB844228BF0446A4B2E2
:10C5B0002346424639463046FFF752FB284604F0F0
:10C5C00009FC204604B0BDE8F08100BF4C08002003
:10C5D0007FB50B7806460D4614462BB94B781BB930
:10C5E0008B780BB9C878D0B1DCB14FF00043019320
:10C5F0000023039302238DF8083004AB13E90E00E7
:10C60000094804F0DBFB29463046FFF794FB21463E
:10C610003046FFF797FB044804F0DCFB012004B030
:10C6200070BD2046FBE700BF4C0800202DE9FF4706
:10C6300000234FF000480227CDF8048003938DF8C3
:10C64000087001AC94E80E0005461F48DFF87890AA
:10C6500004F0B4FB2021284600F0E0FA022128462D
:10C66000FFF7C4FA10F0100623D102212846FFF785
:10C67000BDFA10F0080A0BD0182202212846FFF755
:10C68000C9FA114804F0A6FB304604B0BDE8F087B3
:10C69000484604F09FFB04F047F9CDF80480CDF83C
:10C6A0000CA08DF8087094E80E00484604F086FB54
:10C6B000D4E7102202212846FFF7ACFA024804F022
:10C6C00089FB0120E1E700BF4C08002007B50023EB
:10C6D00000931A461946034803F08CFA03B05DF83C
:10C6E00004FB00BFE006002070B505460C468E181E
:10C6F000B44206D02178284604F06DFB04F8010B03
:10C70000F6E770BD024B0021187804F0CDBA00BFE7
:10C710000A000020024B0121187804F0C5BA00BFBE
:10C720000A0000202DE9F3414F4B1B78332B0446C0
:10C730000D4616461FD100EB02084C4F4D1E1FFA46
:10C7400088F8A0457AD0FFF7DDFFF021384604F0E5
:10C7500042FB210A384604F03EFBE1B2384604F0C1
:10C760003AFB013415F8011F3846A4B204F033FB3C
:10C77000FFF7D0FFE5E7342BC7B21DD1FFF7C2FFAB
:10C78000330A241263F07F030422694637488DF888
:10C7900000408DF801708DF802308DF80360FFF7CE
:10C7A000A3FF013D314CAF19AF4245D015F8011F31
:10C7B000204604F010FBF7E7FFF7A4FFFF2C08D892
:10C7C00000238DF800308DF8017004238DF80230BD
:10C7D0000DE0230419D4E41024F01F04002344F0D6
:10C7E0000C048DF800308DF801708DF80240052E94
:10C7F00028D82A46531BDBB2B34218DA02A80344F6
:10C8000012F8011B03F8051CF4E744F3871323F027
:10C810001F03B4F5404F4FEA14228DF800208DF825
:10C82000017034BF43F0140343F01C03CEE7F21C45
:10C8300069460E48FFF758FFFFF76CFF304602B01D
:10C84000BDE8F081032269460848084FFFF74CFF16
:10C85000731E6C1E15FA83F514F8011F384604F098
:10C86000BAFAA542F8D1E7E7310700204C080020CA
:10C8700007B502AB012203F8011D1946FFF752FF6D
:10C88000C0B203B05DF804FB08B501460020FFF715
:10C89000EFFF08BD2DE9F3413E4B1B78332B0446D7
:10C8A0000E46154620D100EB02083B4F4E1E1FFAE4
:10C8B00088F8A0453AD0FFF725FF0F21384604F04D
:10C8C0008AFA210A384604F086FAE1B2384604F0C2
:10C8D00082FA0021384604F07EFA013406F8010F8E
:10C8E000A4B2FFF717FFE4E7342BC7B222D1FFF75A
:10C8F00009FF2412C5F3062304228DF804408DF8A5
:10C9000005708DF806308DF807500DEB02012248B6
:10C91000FFF7EAFE2A460021304606F022FB2A46AF
:10C9200031461D48FFF7E0FEFFF7F4FE284602B04F
:10C93000BDE8F081FFF7E6FEFF2C07D800238DF855
:10C9400004308DF805708DF806300DE023040ED408
:10C95000E41024F01F04002344F008048DF8043090
:10C960008DF805708DF80640032201A9CFE744F346
:10C97000871323F01F03B4F5404F4FEA14228DF8BC
:10C9800004208DF8057034BF43F0100343F0180302
:10C99000D9E700BF310700204C08002007B501226D
:10C9A0000DF10701FFF776FF9DF8070003B05DF872
:10C9B00004FB08B50020FFF7F1FF08BD10B580208B
:10C9C000FFF762FF1424FFF7F4FF40B1013C0120A0
:10C9D000A4B203F087FF002CF5D1204610BD012042
:10C9E000FCE7000008B50F4B33221A70FFF7E6FF93
:10C9F00008B9002008BD1020FFF746FFFFF7D9FF58
:10CA00001028F6D11220FFF73FFFFFF7D2FF1228C0
:10CA1000EFD10020FFF738FFFFF7CBFFB0FA80F02F
:10CA20004009E7E73107002008B5124B34221A709D
:10CA3000FFF7C4FF08B9002008BD0820FFF724FF56
:10CA4000FFF7B7FF0828F6D11020FFF71DFFFFF70B
:10CA5000B0FF1028EFD10020FFF716FFFFF7A9FF66
:10CA60000028E8D11F20FFF799FFC31E5842584104
:10CA7000E2E700BF3107002008B5124B37221A70D9
:10CA8000FFF79CFF08B9002008BD0820FFF7FCFE57
:10CA9000FFF78FFF0828F6D11020FFF7F5FEFFF70C
:10CAA00088FF1028EFD10020FFF7EEFEFFF781FF8F
:10CAB0000028E8D13920FFF771FF031F5842584181
:10CAC000E2E700BF310700207FB52D4E3478002CFF
:10CAD00053D14FF40C7003F005FF2A4804F058F9C5
:10CAE000294B0121187804F0B7F8FFF713FE4FF037
:10CAF0000043019302238DF80830039404AB13E93B
:10CB00000E00204804F05AF9FFF78EFFB0B11F4B1A
:10CB100040221A70E5B202221E212846FFF77AF859
:10CB2000013402221F212846FFF774F8082CF1D1A6
:10CB30001448012404F04EF934701BE0FFF79CFF09
:10CB400018B1124B10221A70F2E7FFF74BFF0446A0
:10CB500058B10E4B042255211B201A70FFF788FE96
:10CB600055211A20FFF784FEE2E7094B18700548AB
:10CB700004F030F9204604B070BD0124FAE700BF8C
:10CB8000320700204C0800200A0000203007002057
:10CB9000310700201FB5FFF797FF38B11D4B1B78F9
:10CBA000342B4FF0000003D0372B1BD004B010BD46
:10CBB0004FF000430193022303908DF8083004AB3B
:10CBC00013E90E00144804F0F9F83520FFF7E6FEEB
:10CBD0000446114804F0FEF814F0200F14BF0120A1
:10CBE0000220E3E74FF000430193022303908DF806
:10CBF000083004AB13E90E00074804F0DFF82E20DC
:10CC0000FFF7CCFE0446044804F0E4F814F0010FEA
:10CC1000E4E700BF310700204C08002038B50A4681
:10CC200001210446FEF7F6FF054D2402287804EBA7
:10CC30000020013080B2FFF7B1FE0028F6D138BDE8
:10CC40003007002007B5002300931A461946034811
:10CC500002F0D0FF03B05DF804FB00BF28070020FE
:10CC600014220021103006F07CB910B510310446B2
:10CC700002F0D2FF204610BD10B51431044602F078
:10CC8000CBFF204610BD10B51831044602F0C4FF9A
:10CC9000204610BD10B52031044602F0BDFF2046ED
:10CCA00010BD30204B1C0870110902F00F02092A38
:10CCB00094BF3032373203F801290A460029F3D1F4
:10CCC0007047000007B5002300931A461946034831
:10CCD00002F090FF03B05DF804FB00BF34070020B2
:10CCE0002DE9F0418EB004468846164600212022E8
:10CCF00006A806F036F9FF231A461946009302A843
:10CD000002F078FF04F14805554B04934322039B3E
:10CD1000059304A92846FEF7B7FE013000F09D8078
:10CD2000504B069363688DF821601BBA0793330A52
:10CD30008DF820301C22802306A926462846ADF80F
:10CD40002230FEF7B0FE1A2200210DF11E0006F07F
:10CD500008F956F8080F0690B388ADF81C30102279
:10CD600006A92846FEF79FFE2022002106A806F00D
:10CD7000F8F80627202206A92846FEF794FE013F70
:10CD8000F8D1394B069340F23513ADF81C303D23F2
:10CD90008DF81F3007238DF8203001238DF82130C6
:10CDA0003368CDF82230B388ADF826302F498DF89E
:10CDB0001E8040F60C430DF12A00ADF8283007F034
:10CDC00052F8E27A0CA92046FFF76BFF227B0DF1A7
:10CDD00032012046FFF765FF627B0DA92046FFF771
:10CDE00060FF1E2206A92846FEF75DFEB8F1030F7C
:10CDF00024D140F23243ADF81830237C8DF81A303C
:10CE0000637C8DF81B30A37C8DF81C30E37C8DF89F
:10CE10001D3040F23643ADF81E30237F8DF82030B0
:10CE2000637F8DF82130A37F8DF822300C22E37FC1
:10CE30008DF8233006A92846FEF735FE0C4A0D4B27
:10CE400006A9CDE906232846FF2309228DF82030C4
:10CE5000FEF729FE2846FEF720FE0EB0BDE8F08161
:10CE6000AC9801000101060063825363E49601005F
:10CE700037060103060F3A3B2DE9F04391B0054612
:10CE80008846164603F0FAFC05F14804074620469A
:10CE9000FEF770FE00280BDC03F0F0FCC01B4045E1
:10CEA00000F2D280F9F778FE012003F01BFDEEE7D7
:10CEB000242207A92046FEF71AFE9DF81C30022BFB
:10CEC00040F0BD80B5F86430432B40F0B880089F37
:10CED0003FBA3760062205F108010EA806F00EF8E9
:10CEE000064628B92B689F4202D36B689F4207D938
:10CEF0002046FEF768FD0026304611B0BDE8F083FD
:10CF00000B9B2B610146CC222046FEF7F0FD05F17C
:10CF100024072046FEF74AFD002840F39180204672
:10CF2000FEF7CEFD33287DD015DC012844D006DC89
:10CF30000028EED02046FEF7C3FDC2B253E003281E
:10CF400044D00628F6D12046FEF7BAFD04228046DA
:10CF500005F1200141E03A284AD020DC352823D0D1
:10CF60003628E7D12046FEF7ABFD05F11C08414607
:10CF7000814601A802F050FE002103A802F046FEFF
:10CF8000029A049B9A4230D0414605A802F044FE22
:10CF90002A6E069B9A4228D05FFA89F223E03B284A
:10CFA00033D0FF28B5D0C5E72046FEF789FD2046DF
:10CFB000FEF786FDC6B2ACE72046FEF781FD0422EF
:10CFC00005F114012046FEF792FDA2E72046FEF788
:10CFD00077FD0422804605F118012046FEF787FD03
:10CFE0005FFA88F2043A0021ECE704224146E9E7BF
:10CFF0002046FEF765FD042205F128012046FEF7D4
:10D0000076FDAB6A1BBAAB6283E72046FEF758FD9C
:10D01000042205F12C012046FEF769FDEB6A1BBADC
:10D02000EB6276E72046FEF74BFD042239462046A8
:10D03000FEF75DFD6B6A1BBA6B622B6369E7002626
:10D040002046FEF7C0FC57E7FF2655E72DE9F347DA
:10D0500004464FF4FA61012003F091FA274660601C
:10D0600047F8480B3846FEF7AFFC44213846FEF738
:10D07000B7FC002800F0908003F000FC4FF000099E
:10D08000804600254FF0030A94F84430032B1CD04F
:10D0900043BB63680133636003F0F0FB4FF47A72C3
:10D0A000A0EB08000121B0FBF2F2204692B2FFF79C
:10D0B00017FE012384F84430002DE5D103F0DEFB98
:10D0C000A36BA0EB08009842DBD93846FEF77CFC46
:10D0D00063680133636003F0D1FB2064284602B02B
:10D0E000BDE8F087042B11D163680133636003F05E
:10D0F000C5FB4FF47A72A0EB08000321B0FBF2F2FB
:10D10000204692B2FFF7ECFD0223D3E7012B19D1A1
:10D1100001AAE16B2046FFF7AFFE0228064638D190
:10D12000019B636003F0AAFB4FF47A72A0EB080046
:10D130000321B0FBF2F2204692B2FFF7D1FD84F852
:10D140004460B9E7022BB7D101AAE16B2046FFF793
:10D1500093FE0528064617D1636A84F844A013B9E4
:10D160004FF461736362A36A13B9636A5B08A362D5
:10D17000E36A1BB9636AA3EBD303E362A36A236385
:10D18000E36A636301257FE7062802D184F84490AF
:10D1900092E7FF2EFAD08FE705469FE7F8B5002506
:10D1A0000F460446C0E90955C562C0E90E238560F3
:10D1B0008581FFF755FD3B68A360BB88A38184F898
:10D1C00044502046BDE8F840FFF740BF10B5044684
:10D1D00003F054FB236CC31AB3F57A7F14D34FF4D6
:10D1E0007A71B3FBF1F201FB1233C01A236B206496
:10D1F00051008B4234BF00239B1A2363636B994217
:10D200008CBF00239B1A6363206BE0B994F8443011
:10D21000032B06D1042384F844302046FFF716FF81
:10D220000130636B73B994F84430032B00D04BB9D1
:10D23000002384F844302046FFF712FD2046FFF714
:10D2400005FF033010BD0020EBE74B68436000236F
:10D250000381704770B500240139234611F8010F8E
:10D26000B8B1A0F13005EEB2092E08D803EB830364
:10D2700005EB43039BB2FF2BF0D900200DE02E28D5
:10D28000FBD1032CF9D0601C14442371C4B20023D9
:10D29000E4E7032C01D1D371012070BD07B5002351
:10D2A00000931A461946034802F0A4FC03B05DF847
:10D2B00004FB00BF3C0700202DE9F74305460E465E
:10D2C00003F0DCFA05F10C04288105F108010222C3
:10D2D00002AD2046FEF7E7FB012325F8023D0222BE
:10D2E00029462046FEF7DFFB4FF4807302222946D1
:10D2F0002046ADF80630FEF7D6FB00230222294671
:10D300002046ADF80630FEF7CEFB02222946204625
:10D31000FEF7C9FB022229462046FEF7C4FB37462A
:10D320003378E3B13E46B04618F8013B0BB12E2BE3
:10D3300013D1A6EB0709B9F1000F0CDD01220DF1A5
:10D34000050120468DF80590FEF7ADFB4A463946AB
:10D350002046FEF7A8FB4746E2E74646E3E702A978
:10D36000012201F8033D2046FEF79DFB4FF4807635
:10D37000294602222046ADF80660FEF794FB022201
:10D3800029462046ADF80660FEF78DFB012003B06C
:10D39000BDE8F0832DE9F04387B006460F4690467E
:10D3A00003F06CFA06F10C0405462046FEF7E2FB9A
:10D3B000002808DC03F062FA401BB84200F2C48087
:10D3C000F9F7EAFBF1E7726A73689A4240F0BF80AE
:10D3D000338D352B40F0BB802046FEF7E7FA0B2853
:10D3E00040F3B8800C220DEB02012046FEF77FFBD4
:10D3F000BDF80E203189130A43EA0223BDF80C2040
:10D400001BB29DB29142ADF8065001D1002B07DB53
:10D410002046FEF7D8FA4FF6FC7007B0BDE8F0835F
:10D4200040F20F231D4005D02046FEF7CCFA4FF600
:10D43000FB70F2E7BDF812301F0A47EA0327BFB2BC
:10D440002FB92046FEF7BFFA4FF6FA70E5E7BDF8B0
:10D4500010305BBAAAB29BB29A4216DA01220DF1E1
:10D460000A012046FEF743FB9DF80A201AB100216D
:10D470002046FEF73CFB9DF80A100029EED104225D
:10D480002046FEF734FB0135E1E70026B1460122D4
:10D490000DF105012046FEF72AFB9DF8052012F04C
:10D4A000C00134D112B12046FEF721FB9DF8055092
:10D4B000002DECD1022202A92046FEF718FB022221
:10D4C0000DF10A012046FEF712FB042229462046F0
:10D4D000FEF70DFB02220DF106012046FEF707FBC9
:10D4E000BDF80830BDF80620B3F5807F52BA92B27D
:10D4F0001CD1BDF80A0040BA85B2012D16D1042A0C
:10D500000DD02046FEF75FFA4FF6F77085E701224F
:10D5100000212046FEF7EBFA8DF80590C6E708F1EA
:10D5200004012046FEF7E3FA284676E7013600219B
:10D530002046B6B2FEF7DBFAB742A8D12046FEF786
:10D5400042FA4FF6F67068E74FF6FF7065E74FF660
:10D55000FE7062E74FF6FD705FE700002DE9F347CC
:10D5600005468A4691469846FFF774FE0446B8BBC6
:10D570001E4B6A685B689A4234D003F07FF905F16C
:10D580000C0600F00F0101F580613046FEF728FA25
:10D590000128074620D1164B009335226B68019372
:10D5A00069463046FEF770FA98B151462846FFF7B3
:10D5B00083FE70B13046FEF770FA50B14A464146DC
:10D5C0002846FFF7E7FE0446F9F7E6FA384603F087
:10D5D00089F93046FEF7F8F9204602B0BDE8F08739
:10D5E0000124F9E76FF00104F6E700BF3C070020D3
:10D5F000AC98010007B5002300931A46194603486A
:10D6000002F0F8FA03B05DF804FB00BF4407002005
:10D61000006903681B691847006903685B6918475C
:10D6200013B5006949680368034C01919B69009434
:10D630006946984702B010BDAC98010000690368C4
:10D64000DB691847006903689B6A18470069003066
:10D6500018BF01207047006C70470164704710B517
:10D6600090F83830044633B920690368DB6898477E
:10D67000002808DA10BD03689B6898470028F3D19A
:10D680004FF0FF30F6E794F82220A2F10803022BB6
:10D69000F0D8A36A002BC2BFE36A0133E3620A2A0F
:10D6A000E8D1E36B013BE363002BE3D1092384F86A
:10D6B0002230DFE710B50446006903681B6A98470B
:10D6C00094F82230083B022B07D8A36A002B04DD14
:10D6D0000028A2BFE36A1B18E36210BD73B590F87F
:10D6E0002230092B04460ED10026206903689B686E
:10D6F000984740B120690368DB689847C5B20A2D96
:10D700001CD184F8225094F822300A2B04D1E36B08
:10D7100013B9092384F8223094F82230092B22D03F
:10D72000206903689B68984794F822300A2B03D13C
:10D73000E36B9842A8BF184602B070BD0D2DD4D03F
:10D74000284605F084FB0028CFD0E06BADF80460DC
:10D7500010228DF804500021050101A807F012FBEA
:10D760002844E063C1E70020E6E7000000234FF013
:10D77000FF32C0E90A23084A80F8223012680263A7
:10D78000064A4362126880F83830C36347F2305368
:10D7900042630364704700BF1000002014000020A3
:10D7A00038B504461D4600204FF47A73C4E90103DE
:10D7B0000B4B2360C4E9041204F1180002F012FAC2
:10D7C0000123258484F8443084F84530054904F168
:10D7D000480002F02DFF2046FFF7C8FF38BD00BF0C
:10D7E0004C9701000298010010B5044600690368D7
:10D7F0005B6A98472046BDE81040FFF7B7BF01239A
:10D8000080F822307047000038B50446006915469C
:10D8100002F041FA0449206902F03DFA29462069E4
:10D82000BDE8384002F04EBA217A010038B504460E
:10D830000D460069114602F02EFA1D49206902F0DA
:10D840002AFA2946206902F026FA1A49206902F0CC
:10D8500039FA94F84530F3B16369B3B116492069D8
:10D8600002F019FAD4E9040102F015FA238C502BC6
:10D8700008D01249206902F00EFA0A22218C206990
:10D8800002F069FA206902F00DFA0D4B0D491A6891
:10D890002046FFF7B9FF94F8443023B10A4A0B49F8
:10D8A0002046FFF7B1FF012384F82230002038BD65
:10D8B0004C7B0100119701001B970100B27C010015
:10D8C0000C000020229701002D97010033970100E2
:10D8D00038B504460069154602F0DDF905492069AE
:10D8E00002F0D9F9294620690A22BDE8384002F041
:10D8F00034BA00BF217A010010B50446006902F075
:10D90000D1F9022384F8223010BD70B590F822308E
:10D91000012B04460D46164601D8FFF7EDFF20699E
:10D920000368324629465B68BDE87040184770B509
:10D9300090F82230012B04460D4601D8FFF7DCFF9A
:10D940002069036829461B68BDE87040184710B578
:10D950000446206903689B68984720B120690368E2
:10D96000DB689847F5E710BD2DE9F347994690F835
:10D970002230083B022B04460E469246DDE90A7827
:10D9800004D8FFF7E4FF2046FFF7F0FE94F822509A
:10D99000012D45D894F844305BB1D4E90401228CC0
:10D9A0000368B9B921490091E16901919B69694610
:10D9B00011E0206903689B6A98470028EDD0314642
:10D9C00052462046FFF732FF064650B1304602B0BD
:10D9D000BDE8F087DB6998470028F0DC4FF0FF36A0
:10D9E000F4E7B9F1000F04D04A4611492046FFF789
:10D9F0000BFF002F17DD3A460E492046FFF768FF60
:10DA0000B8F1000F0FD001252046FFF775FF002D5C
:10DA1000DCD023683A465B68414620469847D5E704
:10DA20006FF00106D2E7002DD0D1EDE7AC980100F0
:10DA3000EB960100F896010090F82230012B01D8F6
:10DA4000FFF75ABF7047FFF7F7BF000007B5002385
:10DA50004FF0FF32CDE90023024AFFF785FF03B004
:10DA60005DF804FB3E9701002DE9F04790F8223065
:10DA7000012B044651D9DFF8D88000250327002365
:10DA80006362022384F8223002F0F8FE46468246A2
:10DA90004FF00A090A2D46D002F0F0FE236CA0EBED
:10DAA0000A00984245D2236820469B68984748B3AD
:10DAB00023682046DB689847431C0546ECD094F861
:10DAC0002230022B05D0032B0FD002F0D7FE824666
:10DAD000E0E733782A2B01D083421AD17278731C85
:10DAE0000AB984F822701E46EFE7A0F13002092A35
:10DAF00095BF636A042309FB032384F8223098BF8F
:10DB00006362E2E74FF47A7002F0ECFEC2E70A2D9E
:10DB100006D16FF00300BDE8F0876FF00100FAE76F
:10DB20006FF00200F7E7636AC72B02DC652B18BFB2
:10DB3000002594F82230042BE9D1606AC72801DC63
:10DB400065289CD10A2D18BF6FF00200E3E700BFE3
:10DB50000797010038B501F1480504463A212846E7
:10DB600002F046FE421C034605D10649204602F05B
:10DB70005FFD204638BD00222946204602F056FEB1
:10DB8000F7E700BF02980100F8B501F14806054625
:10DB90000F4630463A2102F02BFE441C013005D1DD
:10DBA0000C49284602F044FD2846F8BD3B6DA342CF
:10DBB00009DD2146304602F0FFFD007805F03EF910
:10DBC00008B10134F2E73B6D22463146284602F0A7
:10DBD0002DFEE9E70298010010B503680446DB68F2
:10DBE000984794F82230A3F10802022AC0B232D931
:10DBF000052B31D0072B39D0042B54D1226B13784D
:10DC000083420BD1531C2363537823B9C4E90A33ED
:10DC1000052284F822200A281DD136E0636B19788A
:10DC200081420BD15A1C62635B78002BF3D1012334
:10DC300084F83830062384F82230ECE71B49096861
:10DC40008A42F7D11A4A12689342F3D10D28F1D1D2
:10DC5000072384F8223010BDA0F13002092AE9D848
:10DC6000A36A0A2101FB0323A362D4E70A28F2D1A5
:10DC700094F838309BB1092384F822300023E36301
:10DC800094F82230083B022BE5D9042384F8223093
:10DC9000064B1B682363064B1B686363DBE70823A3
:10DCA00084F82230ECE70A28D5D1E9E710000020FB
:10DCB0001400002038B5044602F0E0FD054694F853
:10DCC0002230083B022B13D902F0D8FD236C401BF5
:10DCD00098420DD2236820469B68984718B1204689
:10DCE000FFF77AFFE8E74FF47A7002F0FBFDE6E712
:10DCF00094F82230083B022B94BF00206FF0020002
:10DD000038BD10B590F82230083B022B044601D9EB
:10DD1000FFF7D0FFA06A10BD38B590F82230083B5D
:10DD2000022B054601D9002038BDFFF7EAFF01307C
:10DD3000F9D02846EC6AFFF7E4FF8442B4BF002024
:10DD40000120F1E7FFF7E8BFFFF7E6BF38B500F1C4
:10DD5000480504460E49284602F0C7FC94F82230D4
:10DD6000083B022B09D92046FFF736FF0D2801D0CA
:10DD70000A2807D1236D002BF0D0206D003018BF8A
:10DD8000012038BDC1B2284602F0D0FCE6E700BF52
:10DD90000298010007B5002300931A46194603486C
:10DDA00001F028FF03B05DF804FB00BF5C07002012
:10DDB00080687047C1607047036810B59B690C4666
:10DDC0009847036821461B68BDE8104018472DE9B5
:10DDD000F84380460D46174601EB02090C46A14563
:10DDE000A4EB050609D0D8F800304046DB68984718
:10DDF000431C03D004F8010BF1E73E463046BDE872
:10DE0000F883C368013310B5044612D12368204655
:10DE10009B69984703689B68984758B123682046D8
:10DE2000DB6898472028F1DD2368C1B25B69204692
:10DE30009847012010BD70B50446C068431C18D136
:10DE400002F01CFD00F5FA75236820469B6998478F
:10DE500003689B68984718B902F010FD8542F3D813
:10DE6000236820469B6998470368BDE87040DB68DB
:10DE700018474FF0FF33E36070BD10B5182005F070
:10DE80001BF8044618B11822002105F06AF8204654
:10DE900010BD70B506460C46D4B1237C65681B07DF
:10DEA00004D4E16811B13046FFF7F3FF237C03F09F
:10DEB0000F03042B03D1606908B100F0CFFC206888
:10DEC00008B100F0CBFC204604F0FEFF2C46E3E74F
:10DED00070BD00002DE9F04F036885B0DB68054692
:10DEE0000E469847421C044604D14FF0FF3005B05F
:10DEF000BDE8F08F2D282FD12B682846DB68984786
:10DF0000431C0446F1D04FF0FF330093A4F13003DB
:10DF1000092B4FF000070DD84FF00A082B68284650
:10DF2000DB689847A0F13003303C092B08FB07471A
:10DF30000446F3D92E2C11D024F02003452B0DD00C
:10DF4000009B7B437361022333742B6828465B6913
:10DF5000E1B298470020CAE70123D6E7384604F02B
:10DF6000A7F92E2C8046894639D12B68DFF814B1E9
:10DF7000DB6828469847002704464FF0000A5246BF
:10DF80005B464046494604F0FDF980468946A4F1C7
:10DF9000300004F08DF942464B4604F03DF82B6802
:10DFA0008046DB68284689469847A0F13003092B54
:10DFB00007F1FF370446E2D924F02003452B2AD18C
:10DFC0002B682846DB6898472B28044609D12B6824
:10DFD0002846DB68984704464FF0010A0AE000270C
:10DFE000EAE72D28F8D12B682846DB6898474FF0E0
:10DFF000FF0A04464FF0000B0A22A4F13003092B5C
:10E000000DD802FB0B3B2B680392DB682846984730
:10E01000039A0446F1E74FF0010A4FF0000B009815
:10E0200004F046F942464B4604F0ACF9CDE9000154
:10E03000584604F03DF980465046894604F028F9D8
:10E0400002460B464046494604F09CF98046384655
:10E05000894604F02DF902460B464046494603F036
:10E06000DBFF02460B460020064902F0F5FE0B4698
:10E070000246DDE9000104F085F904F07BFC03238E
:10E08000706161E70000244019B10A22496901F07A
:10E0900040BE084670470000F8B506462DED028BDD
:10E0A000D1B391ED058A18EE100A04F013F9B5EE1C
:10E0B000C08AF1EE10FA04460D4606D51A493046DC
:10E0C00001F0E9FD05F100431D462946204604F014
:10E0D00031FC0A2201460746304601F048FE13494A
:10E0E000304601F0D8FD384604F0D2F802460B461F
:10E0F0002046294603F08EFF09A3D3E9002303F04D
:10E100008BFF00220A4B04F03DF904F013FC0A22B5
:10E110000146304601F03AFEBDEC028B0020F8BD0E
:10E120009A9999999999A93F439D0100F48D01000D
:10E1300000002440F8B50368DB6806460F469847A0
:10E14000222803D04FF0FF342046F8BD04233B744F
:10E1500000F0F4FA05460028F4D033683046DB6856
:10E160009847431C044611D0222C36D01F2C34DD96
:10E170005C2C04D02946E0B200F0F6FAEDE73368F3
:10E180003046DB689847421C044603D1284600F01D
:10E19000F7FAD9E7622817D007DC2F2803D05C28CC
:10E1A00001D02228D9D12946E6E76E280FD004DC19
:10E1B0006628D2D129460C20DEE772280AD07428BE
:10E1C000CBD129460920D7E729460820D4E729469C
:10E1D0000A20D1E729460D20CEE7284600F012FBA1
:10E1E00000247861B0E7000038B50D461D490446AB
:10E1F00001F051FD7DB3013D15F8011F59B31F29F1
:10E2000007D9222905D05C2903D0204601F047FD1B
:10E21000F2E75C21204601F042FD29780C2914D058
:10E2200007D8092915D00A2911D00829E4D162217B
:10E23000EBE72229E9D003D80D29DDD17221E4E7EB
:10E240002F29E2D05C29E0D0D6E76621DDE76E21F8
:10E25000DBE77421D9E72221204601F020FD0020D0
:10E2600038BD00BF247A01004969FFF7BDBF38B54A
:10E270000368DB68044698474FF48075411C0FD053
:10E2800020280EDC013D6A1C236803D0DB68204691
:10E290009847F3E72368C1B25B692046984700209E
:10E2A00038BD002DF6D14FF0FF30F9E703682DE9B6
:10E2B000F047DB6804468846914698477B2803D0A0
:10E2C0004FF0FF30BDE8F087062388F81030204675
:10E2D000FFF7CDFF23682046DB6898477D2843D0B1
:10E2E0002368C1B25B6920469847FF264FF0000AB9
:10E2F000FFF7C3FD05460028E2D096B3C8F80C002E
:10E300002046FFF7B4FF29462046FFF713FF0130F0
:10E31000D6D02046FFF7ABFF6B692B602368C5F8AA
:10E3200014A0DB68204698473A28C9D12046FFF759
:10E330009EFF4A462946204600F018F80130BFD01B
:10E340002046FFF794FF23682046DB6898472C2877
:10E350002F464FF00006CBD07D3818BF4FF0FF306E
:10E36000B0E778608760CBE70020ABE7F7B50446FD
:10E370000E461746FFF77BFF013002D14FF0FF300A
:10E3800011E023682046DB689847431C0546F5D01A
:10E390002368C1B25B6920469847222D05D13146DA
:10E3A0002046FFF7C7FE03B0F0BD2D2D03D0A5F129
:10E3B0003003092B04D831462046FFF78BFDF2E7E6
:10E3C0005B2D05D13A463146204600F078F8EAE761
:10E3D0007B2D05D13A4631462046FFF767FFE2E73D
:10E3E0006E2D15D102AD002345F8083D23680422A7
:10E3F0001B6929462046984704280246BED11D497C
:10E40000284605F070FD0028B8D100233374CAE710
:10E41000662D16D1002300938DF804302368052261
:10E420001B696946204698470528A7D1052212494D
:10E43000684605F058FD0028A0D1012333743075DB
:10E44000B1E7742D9AD102AD002345F8083D236849
:10E4500004221B69294620469847042802468DD18C
:10E460000649284605F03FFD002887D10123337473
:10E47000337598E7C6970100CB970100D19701004B
:10E48000F8B5064617460D4611B900242046F8BDDA
:10E49000FFF7F3FC04460028F7D02846FFF7E7FE15
:10E4A0003A4621462846FFF761FF0130EED121466A
:10E4B0003046FFF7EEFCE8E70022FFF7E1BF2DE969
:10E4C000F8430368DB6804468846914698475B2812
:10E4D00003D04FF0FF30BDE8F883052388F81030F3
:10E4E0002046FFF7C4FE23682046DB6898475D2876
:10E4F0002AD02368C1B25B6920469847FF26FFF700
:10E50000BCFC05460028E4D0DEB1C8F80C0020466B
:10E51000FFF7ADFE4A4629462046FFF727FF06468D
:10E520000028D6D12046FFF7A2FE23682046DB68EC
:10E5300098472C282F46E2D05D3818BF4FF0FF30A7
:10E54000C9E778608760E2E70020C4E738B5054690
:10E5500051B3CC687B2101F0A2FB013002D14FF016
:10E56000FF3038BDB4B121682846FFF73DFE0130C9
:10E57000F5D03A21284601F092FB0130EFD0214638
:10E58000284600F013F80130E9D0646814B12C215A
:10E590002846E0E77D21284601F081FB01304FF05D
:10E5A000FF3018BF0020DCE70846DAE7E9B10B7C52
:10E5B00003F00F03062B18D8DFE803F004070D0F54
:10E5C000111315000A4901F066BB0B7D0BB1094917
:10E5D000F9E70949F7E7FFF757BDFFF75DBDFFF71B
:10E5E00043BE00F00EB8FFF7B1BF0020704700BF78
:10E5F000C6970100D1970100CB9701001046FFF7A5
:10E60000D5BF38B50546F1B1CC685B2101F047FBB9
:10E61000013002D14FF0FF3038BD54B121462846B9
:10E62000FFF7C4FF0130F5D0646814B12C212846EF
:10E63000ECE75D21284601F032FB01304FF0FF305E
:10E6400018BF0020E8E70846E6E731B1CB680022B2
:10E65000D0B2013213B15B68FAE70846704731B1B6
:10E66000C96821B11AB1013AD2B24968F9E708463E
:10E67000704738B515460C4641B1CC6834B12946CF
:10E68000206805F0ACFB08B16468F7E7204638BDA8
:10E6900051B14AB1CB6813B9CA6070470B4659688B
:10E6A0000029FBD15A6093607047F8B505460E46C5
:10E6B00017461C4673B1186808B100F0CFF8384609
:10E6C00000F076F82246206031462846BDE8F84042
:10E6D000FFF7DEBFF8BD08B5FFF7CFFB18B1037C2D
:10E6E0006FF303030374037C6FF30713037408BD14
:10E6F00010B50C46FFF7C1FB10B10223037444614F
:10E7000010BD70B50D46194604461646FFF7F0FFDA
:10E710003246034629462046BDE87040FFF7C5BF94
:10E7200007B5002300931A461946034801F062FA20
:10E7300003B05DF804FB00BF6407002038B50C206F
:10E7400004F0BAFB044650B1064820604FF48075CF
:10E750002A46002104F005FC00236560A3602046E2
:10E7600038BD00BF78080020D1E90132013B9A4250
:10E7700004D20B6898548B6801338B60002070477B
:10E7800008B104F0A1BB704738B5054658B1074C35
:10E79000216819B1284605F05CFB10B1A468002C73
:10E7A000F6D1204638BD0446FBE700BF70070020C5
:10E7B000F8B50746FFF7E8FF20B10379013303718D
:10E7C0000068F8BD0E4D2B6843B9384605F054FB80
:10E7D000012328602B71F4E73546F4E7AE68002E7C
:10E7E000FAD10C2004F068FB04460028E9D0A860A8
:10E7F000384605F041FB012320602371A660E0E765
:10E8000070070020826838B5044622B103681344BB
:10E8100013F8013C1BB121460020FFF7A5FF054876
:10E82000FFF7C6FF054610B1204604F04DFB284611
:10E8300038BD00BF7808002010B5074CA06800B9AB
:10E8400010BD0268836822B9A36004F03DFBA36891
:10E85000204604461846F2E77007002038B5FFF757
:10E8600093FF054660B10479013CE4B204713CB900
:10E87000006804F029FB2C60BDE83840FFF7DCBFDE
:10E8800038BD000008B5064B1B7843B9054801F0B8
:10E8900009FA05490348BDE8084001F0F3B908BD8D
:10E8A000C1070020D4070020FC970100F0B50478D0
:10E8B0009FB005464CB31C4B1C4F1B68986804F076
:10E8C000ABF92846194906F07BF91EAD012445F83D
:10E8D000780D3946002006F073F91E2C264645F8BF
:10E8E000240002D001340028F3D1114B009F1C6892
:10E8F00084B12168384605F0ACFA48B96368294606
:10E90000304698470446FFF7BDFF20461FB0F0BDD4
:10E91000A468EDE7074B1B78002BF6D106490748A2
:10E9200001F0C6F9EFE700BF380000204C7B010082
:10E93000BC070020C107002003980100D407002075
:10E94000F8B505460C200F4604F0B6FA0C4B044609
:10E950001860284605F0ABFA013004F0ADFA2946FC
:10E96000064605F080FA284605F0A1FA0023335444
:10E97000044B1A68A260C4E900671C60F8BD00BFC0
:10E98000BC0700207C070020184B1B7870B5FBB932
:10E990001748184D01F0D4FCC4B20A2C0CD00D2C31
:10E9A0000AD0082C15D12146114801F078F92B78AE
:10E9B00073B1013B2B700BE02B780F4E0F490C48C5
:10E9C0000024F45401F067F93046FFF76FFF2C7014
:10E9D00070BD2146064801F062F92B783A2B9FBFA3
:10E9E0005A1C2A70044AD454F2E700BFC107002021
:10E9F000D4070020C00700208007002000980100F5
:10EA0000064B1B7810B53BB9054C204601F092FC33
:10EA100010B1FFF7B9FFF8E710BD00BFC107002034
:10EA2000D4070020054A00231370054A01461360ED
:10EA300010B1044801F03EBC704700BFC007002081
:10EA40007C070020D407002070B504460D4601F075
:10EA500015FFA061A068036829461B68BDE87040E7
:10EA6000184770B504460D46164601F007FFA06131
:10EA7000A0680368324629465B68BDE870401847C5
:10EA800010B50446C06804F01FFA204610BD2DE9F9
:10EA9000F04105460E4601F0F1FE4FF47A778046CC
:10EAA000A86803689B689847044658B901F03CFF82
:10EAB00001F0E4FEAB8AA0EB08007B439842EFD361
:10EAC000204605E0A8680368DB689847307001209D
:10EAD000BDE8F08138B5148821441546FFF7D7FF0B
:10EAE00008B101342C8038BD2DE9F74F02AD002666
:10EAF00025F8026D8A462A46C1680446FFF7EAFFF8
:10EB000018B9002003B0BDE8F08FE3680DF10809E3
:10EB100093F8008009F8036D0127BDF80630052B36
:10EB200007D14FF0FF33A068E36303685B6A98473F
:10EB3000E7E749462046FFF7AAFF0028E1D0BDF8E5
:10EB40000630E268591CADF806109DF80510D15446
:10EB50009DF8053003F07F0207FB02661A064FEAB4
:10EB6000C717DAD49DF8063008F0F008013BB8F179
:10EB7000300F8AF800301DD12A46E1682046FFF7A1
:10EB8000A9FF0028BDD02A46E1682046FFF7A2FF72
:10EB90000028B6D0E2689AF80030134459789D787E
:10EBA000137805EB01259B07ADB201D50235ADB257
:10EBB000022701E000273D46BDF806B0A7EB0B0792
:10EBC00007EB0B0296422AD949462046FFF75FFF22
:10EBD000002896D0A06B88B1B8F1300F0ED19AF80A
:10EBE0000020C2F1FF2202F57F02FE325A44AA42FF
:10EBF00004D902689DF8051012689047BDF80620F8
:10EC0000218A914208D9E1689DF805008854BDF831
:10EC100006200132ADF806200BF1010BD0E7A26B04
:10EC200022B9218A594538BFADF80620BDF8060043
:10EC300068E70120704773B50025DC1103F07F06FB
:10EC4000A3B20CB146F080060DF1080C681C6544B7
:10EC5000C0B205F8046C0546002CEED1C0F10405E5
:10EC6000515501ADA04205DD231A1344615D597170
:10EC70000134F7E7013002B070BDF8B5064617461B
:10EC80001C46FFF7D8FFB368C0B21A680444C0F14D
:10EC900005015568394422461846A847054601F043
:10ECA000EDFDB061A8B2031B58425841F8BD10B544
:10ECB000C368E0221A70C36800225A700446806854
:10ECC000E168036802225B689847A0684FF0FF3351
:10ECD000E36303685B699847A06803685B6A9847C9
:10ECE00001F0CCFDC4E9060010BD023330B598B286
:10ECF0000C46631A14F8015B9BB21DB1431C1554FA
:10ED000098B2F6E7C11A0A44191202F8021C02F876
:10ED1000013C30BD38B50546806808B9002038BDD3
:10ED200003689B6A9847EC6B68B9002CF6D1A86819
:10ED30006FF00203EB6303685B699847A868036898
:10ED40005B6A9847EAE7B4FA84F04009E7E7000015
:10ED50002DE9FF470C9D9DF840A0044689461746C3
:10ED60001E46FFF7D7FF8046002840F0DF80A068EE
:10ED700003689B6A9847002840D00123E3826E4BCA
:10ED8000029345F25443ADF80C3004238DF80E3055
:10ED9000052302A91944E26811F8051CD154013376
:10EDA0000C2BF6D1002D3DD09DF838309DF8342045
:10EDB0005B0143F0040343EAC203DBB2BAF1000F84
:10EDC00001D043F002031FB1002E2DD143F0800388
:10EDD000E2681373638AE2681B125373E368628A02
:10EDE0009A73218A484605F0A5F8238A1130984283
:10EDF0001DD9A06803685B6A984797E0A068216BFB
:10EE00000368A28E39B1DB6998470128B5D06FF04D
:10EE10000103E3638AE049499B690291E16A039136
:10EE200002A9F1E72B46C9E743F0C003D0E7494602
:10EE30000F23E2682046FFF758FF814605B3218A79
:10EE4000284605F077F809F102031844238A98420E
:10EE5000CFD84B462946E2682046FFF746FF218A75
:10EE600005460F9805F066F8238A02302844984238
:10EE7000BFD82B46E2680F992046FFF736FF814640
:10EE800017B3218A384605F055F809F102031844F2
:10EE9000238A9842ADD84B46E26839462046FFF7B0
:10EEA00024FF814686B1218A304605F043F809F1F6
:10EEB00002031844238A98429BD84B46E2683146A5
:10EEC0002046FFF712FF8146A9F105039BB2E268D5
:10EED00010212046FFF7D1FE01F0D0FCC4E9060066
:10EEE0004FF47A75A06803689B68984758B901F099
:10EEF000C5FCE369C01AA38A6B439842F2D36FF052
:10EF00000303E36375E70DF107012046FFF7ECFD0E
:10EF100004287FF46EAFE368DD785DB901F0AEFCE4
:10EF20004FF00108E06184F82050E563404604B0EA
:10EF3000BDE8F087E5635CE700044D51AC98010043
:10EF400010B586B0012404940B9C03949DF82840CE
:10EF500002949DF824400194089C0094FFF7F8FE69
:10EF600006B010BD2DE9F3470446FFF7D3FE8046F7
:10EF7000D0B101F083FC628A4FF47A735343E269A3
:10EF8000821A9A42074603D8A269821A93421FD274
:10EF900094F8203063B16FF00303A068E363036863
:10EFA0005B6A98474FF00008404602B0BDE8F08722
:10EFB000E268C0211170E2685370A068E1680368DC
:10EFC00002225B689847C4E90677012384F8203061
:10EFD000A06803689B6898470028E5D00DF10701F9
:10EFE0002046FFF781FD83B20646002B73D0E3680D
:10EFF000E7611A7802F0F002302A57D1626A002ADB
:10F00000D2D09DF807209918901C49781D5C05EB1B
:10F010000125ADB2D11C19442A46184403F088FFDB
:10F02000E3689DF807202B44134400229A70E1689E
:10F030009DF807C091F8009009F00609B2B20CF1F2
:10F040000200B9F1020F0844666A0CF10303A2EB57
:10F050000C0225D12B440CF1050C11F803E00B44F4
:10F06000521B93F801A06544053A29440AEB0E2A85
:10F07000B047E36840221A70E36883F80190E368C0
:10F080001FFA8AFA4FEA2A229A70E36883F803A0EB
:10F09000A068E168036804225B689847A76183E77A
:10F0A0002B44033A521B1944B0477DE7C02A0BD1C9
:10F0B000D0221A70E36800225A70A068E1680368E1
:10F0C00002225B6898476FE7D02A7FF46DAF002378
:10F0D00084F8203068E72046FFF71CFE002808BFB0
:10F0E0004FF0000860E770B590B005460E46FFF798
:10F0F00011FEE0B1304604F0DAFE3123C4B28DF8DF
:10F100000030A31C8DF801303B220023314601A8BA
:10F110008DF802308DF8034004F0F7FE2B68221DB5
:10F120005B68694628469847003018BF012010B038
:10F1300070BD2DE9F0470446884617461D469DF8E8
:10F140002060FFF7E7FD50B3B4F810904046494601
:10F1500004F0F0FEEB1D1844814520D34146052301
:10F16000E2682046FFF7C1FD00211FFA81FC431829
:10F17000AC459BB2E26801F1010104D217F80CC062
:10F1800002F803C0F1E7002EA3F1050320469BB26D
:10F1900014BF31213021BDE8F047FFF76EBD0020DC
:10F1A000BDE8F08773B505460E4614466AB1018A7C
:10F1B000104604F0BFFE034600220092314622466C
:10F1C0002846FFF7B6FF02B070BD1346F4E7F7B567
:10F1D00005460E461F46144662B1018A104604F0E9
:10F1E000A9FE03460097224631462846FFF7A1FFB5
:10F1F00003B0F0BD1046F4E72DE9F0470446884619
:10F2000092461E46FFF786FD002843D0218A4046DD
:10F2100004F090FE9DF82030002BE3680CBF3022F4
:10F22000312287B21A70B21C3A44012002F07F01E9
:10F23000E568D20918BF41F08001431C29545FFAE8
:10F2400080F9D2B941469BB2E2682046FFF74DFDF6
:10F25000A368E1681A68D2F8048002461846C047DD
:10F2600055468046B244AA4509D0A06815F8011B4E
:10F2700003681B6898478044F5E71846D6E701F015
:10F28000FDFAA06109F1030038443044A0EB080303
:10F2900058425841BDE8F087F7B505460E461F466F
:10F2A000144662B1018A104604F044FE03460097FA
:10F2B000224631462846FFF79FFF03B0F0BD1046B7
:10F2C000F4E7F8B505460E4614461F46FFF722FD43
:10F2D00028B331460523EA682846FFF706FD631F79
:10F2E000002F03440CBF3021312106469BB2EA684F
:10F2F0002846FFF7A0FC0146A868EC680368053EB5
:10F300000E44C1F105015B6821443246984704462A
:10F3100001F0B4FAA861A0B2831B58425841F8BD6D
:10F3200070B50D460446018A2846164604F002FED2
:10F3300045B3012E26D8238A0930834222D32046A2
:10F34000FFF7E8FCF0B1E38A01339BB2C3B1E3827B
:10F35000E38AE2681B125371E368E28A9A71E268F9
:10F36000294607232046FFF7C0FCE3681E54031F0D
:10F37000E26820469BB28221BDE87040FFF77DBC69
:10F380000123E4E7002070BD0022FFF7C9BF70B57C
:10F390000D460446018A284604F0CCFD25B3238A95
:10F3A0000930834220D32046FFF7B4FCE0B1E38A62
:10F3B00001339BB2B3B1E382E38AE2681B1253715B
:10F3C000E368E28A9A71E268294607232046FFF73C
:10F3D0008CFC431FE26820469BB2A221BDE870402E
:10F3E000FFF74BBC0123E6E7002070BD0163828676
:10F3F000704741627047C06B704738B504460D4690
:10F4000009B9002038BD038A4BB9084603F054FD02
:10F41000E060E0682582003018BF0120F2E7C06894
:10F4200004F022FC0028F3D1EBE7000070B50C4B90
:10F4300000250446456040F8283B0E4600F0D2FB0C
:10F440004FF0FF33E363A660A56325824FF480711C
:10F450002046FFF7D2FF0F236382A382204670BDB0
:10F460001C98010007B5002300931A46194603486B
:10F4700000F0C0FB03B05DF804FB00BFC407002030
:10F480008271054A417112680449B2FBF1F14FF4EF
:10F490007A724A43C26070471800002040420F0051
:10F4A00038B504460D464079022101F0D5FB01F044
:10F4B000E5F9A0F5FA60A060657438BD70B5054641
:10F4C0000E460024687901F001FCB042A3B206D1D7
:10F4D000EA689A4204F10104F4D84FF0FF33184669
:10F4E00070BD30B50D46D1B0044601F0C7F93DB945
:10F4F000A368C31AB3F5FA6F02D2207C51B030BDB5
:10F5000000250221A06025606079257101F0A4FB2F
:10F51000012001F0E7F90121607901F09DFB294606
:10F52000607901F0C1FBA379153B012B00F28C80BF
:10F5300040F24C40013800BF00BF00BF00BF00BF19
:10F5400000BF00BF00BF00BF00BF00BF00BF00BFC3
:10F5500000BF00BF00BF00BF00BF00BF00BF00BFB3
:10F5600000BF00BF00BF00BF00BF00BF00BF00BFA3
:10F5700000BF00BF00BF00BF00BF00BF00BF00BF93
:10F5800000BF00BF00BF00BF00BF00BF00BF00BF83
:10F5900000BF00BF00BF00BF00BF00BF00BF00BF73
:10F5A00000BF00BF00BF00BF00BFC3D16079022110
:10F5B00001F052FB607C00283BD0013800BF00BF47
:10F5C00000BF00BF00BF00BF00BF00BF00BF00BF43
:10F5D00000BF00BF00BF00BF00BF00BF00BF00BF33
:10F5E00000BF00BF00BF00BF00BF00BF00BF00BF23
:10F5F00000BF00BF00BF00BF00BF00BF00BF00BF13
:10F6000000BF00BF00BF00BF00BF00BF00BF00BF02
:10F6100000BF00BF00BF00BF00BF00BF00BF00BFF2
:10F6200000BF00BF00BF00BF00BF00BF00BF00BFE2
:10F63000C3D172B600212046FFF740FF013007D149
:10F640000020207462B659E7142001F04BF9ADE7B1
:10F6500001212046FFF732FF0130F1D000250021C3
:10F660002046FFF72BFF01214DF805002046FFF74C
:10F6700025FF0DEB05030835B5F5A07F5860EED1E9
:10F6800062B600225DF832500DEBC203691C586867
:10F6900001D0431C02D1002020742FE7D1108542F5
:10F6A000635C4FEA4303DBB202F1010238BF43F06F
:10F6B0000103282A6354E5D16178237822790B4429
:10F6C000A1780B44E1780B44DBB29A42E3D10120EC
:10F6D000E2E70000000000002DE9F8430D462DEDA3
:10F6E000028B11460446FFF7FCFE00287ED0A3796A
:10F6F0000B3B0B2B7AD8DFE803F0063F7979797959
:10F70000797979796565A378E07808EE103A010691
:10F71000B8EE488A48BFFFEE007A00F00F0048BFFD
:10F7200037EEC88A02F0C4FD31A3D3E9002302F00A
:10F7300029FE064618EE100A0F4602F0CBFD0B46D6
:10F7400002463946304602F067FC03F013F90346DF
:10F750006DB102F0BFFD2AA3D3E9002302F012FE2F
:10F76000254B002202F058FC03F004F90346BDECDF
:10F77000028B1846BDE8F883E078A67800F00F0009
:10F7800002F096FD1AA3D3E9002302F0FBFD07EE79
:10F79000906AF8EE677A804617EE900A894602F082
:10F7A00099FD02460B464046494602F035FC03F0FF
:10F7B000E1F83206034648BF80F00043002DD6D062
:10F7C0001846C6E7A678E378300200F4FE401843F6
:10F7D00007EE900AF8EEE77A17EE900A02F07AFD4B
:10F7E00003A3D3E9002302F0CDFDE0E7034BBEE71E
:10F7F0009A9999999999B93F000040400000C07FBB
:10F80000CDCCCCCCCCCCFC3FD0B50446FFF769FEC8
:10F8100090B3A3790B3B0B2B2ED8DFE803F0060641
:10F820002D2D2D2D2D2D2D2D1C1C607802F040FD31
:10F8300014A3D3E9002302F0A5FD064620780F4665
:10F8400002F036FD02460B463046394602F0E4FB34
:10F8500003F090F8D0BD208840BA80B207EE900A3D
:10F86000F8EEE77A17EE900A02F034FD05A3D3E92B
:10F87000002302F087FDEBE70148EBE7AFF30080E0
:10F880000000C07F9A9999999999B93F00B55DF8A0
:10F8900004FB0020704700B501205DF804FB10B5A3
:10F8A0000446C06803F010FBB4F90600002802DB30
:10F8B000002101F0D1F9204610BD70B50546C068A1
:10F8C0000E4603F001FBEC7C2A7C94420CBF03241F
:10F8D000042414FB06F4A4B2AC80204603F0ECFA36
:10F8E000E86028B12246002103F03BFB6E8070BD2A
:10F8F000A8806880FBE7F0B4FF29C1F38107C1F35A
:10F900008112C1F30115477401F003078CBF002178
:10F9100001210170C168C47C067CC27405748774BF
:10F9200061B1A41B6142A2EB050561416A426A41D3
:10F93000914203D04188F0BCFFF7BFBFF0BC7047D5
:10F9400038B5437804460D4633B1B0F906000028B7
:10F9500002DB002101F080F96378E5804BB1284695
:10F96000012101F079F928460021BDE8384001F075
:10F970009BB938BD70B50E46002104464170017236
:10F98000C160416119461546FFF7B5FF3146204673
:10F99000FFF793FF20462946FFF7D2FF204670BDB0
:10F9A00070B540F2FA5404FB00F303F500431B1456
:10F9B000B3F5FF7F98B222DAFE2BD8B242DDC0F158
:10F9C000FE00C5B20023FF204E1CC943C9B27043DC
:10F9D000013201EB2020504300F47F4406FB03F08A
:10F9E00006FB05F301EB202001EB232150434A43A2
:10F9F000120244EA102002F47F02104370BDB3F5F6
:10FA00007F7F0DDAB0F53F7FDBB28BBFC3F1FC0324
:10FA10000233D8B2DBB294BFFF20FF230025D3E727
:10FA2000A04211D040F2FA44A042DBB204D8043321
:10FA3000DDB20020FF23C7E7C3F1FA03DBB20020E9
:10FA4000FF25C1E70023FBE700231846F8E7000085
:10FA500070B50446083015460E4600F0C3F8FF2383
:10FA6000064A84F822300023266025712361A38290
:10FA7000C4E906222384204670BD00BF439D0100D7
:10FA80000161828270470000024B002908BF1946BD
:10FA900081617047439D0100024B002908BF194650
:10FAA000C1617047439D01000184704773B50D46E5
:10FAB00001690446164639B92B4BC2685B689A4205
:10FAC00002D1002002B070BDA28A002AF9D094F8B9
:10FAD000223005F007000341DB0738D515F47E7F9F
:10FAE00008BF238C206804BF03F47E731D430368A2
:10FAF00000292ED05B6A98470128E2D13C2120687A
:10FB000000F0CDF80A222946206800F024F9237974
:10FB100033BB1649206800F0B5F8A169206800F0F1
:10FB2000BAF82021206800F0BAF8E169206800F0F6
:10FB3000B2F82379B3B90E49206800F0A3F8314632
:10FB4000206800F0A8F8206803689B6A98470120A5
:10FB5000B8E708490091E16801911B6A6946CAE764
:10FB60000549D7E70549E7E7CC07002024980100BD
:10FB70002A980100AC980100AB7A01003598010089
:10FB800008B5FFF793FF08BD07B5002300931A4699
:10FB90001946034800F02EF803B05DF804FB00BFDF
:10FBA000CC0700202DE9F84306460D46071D00F15D
:10FBB0000709002417F8011B0A22284600F0E4F880
:10FBC0002E218046284600F06AF84F454044044400
:10FBD000F0D10A22F179284600F0D6F82044BDE899
:10FBE000F8830000024A026000224260704700BFB2
:10FBF000AC98010030B58371034D9DF80C30056061
:10FC000001714271C37130BDAC980100014AC0E975
:10FC100000217047AC980100024A02600A68426005
:10FC2000704700BFAC9801000B68436070474160AB
:10FC300070472DE9F04106460D4601EB02080C46DF
:10FC40004445A4EB050707D0336814F8011B1B6873
:10FC5000304698470028F3D13846BDE8F08170B5AA
:10FC6000044608460D4604F022F923680246294658
:10FC700020465B68BDE87040184709B1FFF7EFBF49
:10FC80000846704708B5FFF7F8FF08BD03688A68A3
:10FC90005B680968184708B5FFF7EFFF08BD036800
:10FCA0001B6818470149FFF7DABF00BF0098010041
:10FCB00038B50546FFF7E1FF04462846FFF7F2FF97
:10FCC000204438BD38B50546FFF7D7FF044628461F
:10FCD000FFF7E8FF204438BD70B58AB00D460AA989
:10FCE000002301F8043D012A98BF0A22B5FBF2F473
:10FCF00002FB1456F3B2092E94BF30333733DBB214
:10FD0000254601F8013D002CF0D1FFF7B6FF0AB0FF
:10FD100070BD2DE9F04107460E4615462AB9036825
:10FD2000C9B21B68BDE8F04118470A2A05D100296D
:10FD300005DBBDE8F041FFF7CFBFD2B2F9E72D21D7
:10FD4000FFF7ADFF2A46044671423846FFF7C4FF6D
:10FD50002044BDE8F081FFF7DCBF38B50546FFF76A
:10FD6000D8FF04462846FFF79DFF204438BD10B455
:10FD70002AB903685DF8044B1B68C9B21847D2B2B0
:10FD80005DF8044BFFF7A8BFFFF7F1BFFFF7EFBF28
:10FD90002DE9F84F19460646104614461D469DF8B3
:10FDA000287002F089FD28B14C493046BDE8F84F73
:10FDB000FFF755BF25F000494FF0FF32484B204672
:10FDC000494602F079FD48B94FF0FF32444B2046D6
:10FDD000494602F053FD08B94249E6E74FF0604258
:10FDE000414B2046294602F05DFD08B13F49DCE762
:10FDF0004FF060423E4B2046294602F035FD002878
:10FE0000F4D1002200232046294602F02DFDD0B176
:10FE10002D213046FFF743FF05F1004382461D4682
:10FE20003449DFF8D8904FF0000B00204FF0000865
:10FE30005FFA8BF39F4208D942464B4602F0CCFB57
:10FE40000BF1010BF4E78246EAE722462B4602F06B
:10FE5000E3F80D46044602F06DFD0A220146804695
:10FE60003046FFF739FF8244A7B3404602F010FA4C
:10FE700002460B462046294602F0CCF804460D46C1
:10FE800030461D49DFF87490FFF7E9FE4FF0000897
:10FE90008244013FFFB2FF2F1CD04B464246204612
:10FEA000294602F06FFA0D46044602F01BFD0A22B5
:10FEB000014683463046FFF72CFF8244584602F045
:10FEC000F7F902460B462046294602F0A3F80446FD
:10FED0000D46DEE75046BDE8F88F00BFB098010040
:10FEE000FFFFEF7FB4980100FFFFEF41B8980100DA
:10FEF000FFFFEFC10000E03FF48D0100000024404F
:10FF00009DF800100091FFF743BF08B54022002183
:10FF100003F027F80022C0E9102208BD026C10B5DA
:10FF2000531C446C03F03F039C421CBF8154036488
:10FF300010BD0023C0E910337047D0E9102393426D
:10FF40001FBFC25C013303F03F03436414BF10467C
:10FF50004FF0FF307047D0E91030181A48BF4030DA
:10FF60007047D0E91023934214BFC05C4FF0FF30BC
:10FF70007047036C406C013303F03F031B1A584277
:10FF8000584170470649074A074B9B1A03DD043B5B
:10FF9000C858D050FBDC00F037F8F0F751F90000FA
:10FFA000549D010000000020A0020020FEE7FEE7B3
:10FFB000FEE7FEE7FEE7FEE7FEE7FEE7FEE7FEE719
:10FFC000044B1868421C04BF034B1878831F584227
:10FFD0005841704730010010E00F00F0074B1B78CC
:10FFE000062B09D1064B1B68C3F30313033B032BFA
:10FFF00002D8044AD05C704700207047E00F00F040
:020000021000EC
:10000000E80F00F0C098010008B5FFF7D9FF28B14C
:10001000654B664A1B68C3F304231360FFF7DEFFDA
:1000200010B1634B634A1A60FFF7CAFF28B1624BF5
:10003000624A1B68C3F342331360FFF7CFFF20B15E
:100040005F4AD36823F08073D360FFF7B9FF40B1F4
:100050004FF080430022C3F80C21C3F81021C3F8ED
:100060003825FFF7BBFF10B1564B03221A60FFF78C
:10007000B5FF40B1544B05221A6001229A67002255
:100080009A603F225A60514B1A68511C0BBF504B6B
:10009000504B1A781B6802BF08331B68C3F3031365
:1000A000062A4DD1033B032B03D84B4AD35C002BCC
:1000B00046D04FF08052494BD2F80414C3F82015B3
:1000C000D2F80814C3F82415D2F80C14C3F8281574
:1000D000D2F81014C3F82C15D2F81414C3F8301544
:1000E000D2F81814C3F83415D2F81C14C3F840150C
:1000F000D2F82014C3F84415D2F82414C3F84815D4
:10010000D2F82814C3F84C15D2F82C14C3F85015A3
:10011000D2F83014C3F85415D2F83414C3F860156B
:10012000D2F83814C3F86415D2F83C14C3F8681533
:10013000D2F84014C3F86C15D2F84424C3F87025E3
:10014000FFF73EFF28B1264B264A1B6803F04F03FA
:100150001360FFF735FF48B14FF08043D3F8002418
:10016000D20744BF6FF00102C3F80024174B1B688D
:10017000062B09D1174B1B68033B022B81BF1A4A80
:10018000136843F480631360184AD2F8883043F44C
:100190007003C2F88830BFF34F8FBFF36F8F144BDB
:1001A000144A1A6008BD00BF240300104035014006
:1001B00074C007400DF0ADBA440200103C05004089
:1001C000F0ED00E0A00500401056004030010010A6
:1001D000E00F00F034010010BC98010000C00040A6
:1001E00058020010E40E00403C17004000ED00E013
:1001F000180000200090D00310B5044600F03EFB2C
:10020000E06023682046DB689847002808DA00F0A1
:1002100035FBE368C01AA3689842F2D34FF0FF3071
:1002200010BD2DE9F04180460D468F180C46BC42AA
:10023000A4EB050607D04046FFF7DEFF002802DBEF
:1002400004F8010BF3E73046BDE8F0812DE9F843EF
:100250008046894616461C467BB1D7181546BD42D6
:10026000A5EB060409D04046FFF7C6FF002804DBD3
:10027000814502D005F8010BF1E72046BDE8F8837F
:1002800070B50D4609490446164600F0D1F92846D6
:10029000FFF7B2FF002806DB864204D0C1B2204639
:1002A00000F044FAF3E7204670BD00BF0298010059
:1002B0000120704703681322DB6918477047036900
:1002C000C3F81C150369D3F81C21002AFBD00022B7
:1002D000C3F81C210120704710B490F95C30144C15
:1002E00059090122203103F01F0302FA03F344F8F5
:1002F000213003695DF8044B0421C3F80813036936
:100300005A600369DA6003690022C3F800250269B4
:100310004FF0FF33C2F80C350269C2F81435026998
:10032000C2F8083502691430C2F81035FFF701BE73
:1003300000E100E01430FFF70EBE1430FFF711BEED
:100340001430FFF7FABD0000036990F85E2010B585
:10035000C3F80C25036990F85D20C3F8142590F8C4
:1003600061200369012A01BF90F85F40C3F810457E
:10037000036990F8604006BFC3F80845036900228E
:10038000B1F5966FC3F86C2569D9B1F5166F69D9C7
:10039000B1F5965F69D9B1F5165F68D9B1F5615FBE
:1003A00067D9B1F5964F66D9B1F5E14F65D9B1F589
:1003B000164F64D9B1F5614F64D9B1F5963F64D950
:1003C000B1F5E13F63D9B1F5613F63D9364B99424D
:1003D00063D9B1F5E12F63D9B1F5612F94BF4FF027
:1003E00070634FF080530269C2F824350369042218
:1003F000C3F8002501690023C1F808310169C1F87B
:100400001C31016901230B6001698B600169C1F82E
:10041000042390F95C20510902F01F0293406031DF
:10042000224A42F8213090F95C30002BBDBF03F026
:100430000F0302F6FC32D2189B18B5BF602360226E
:10044000137683F8002390F95C300122590903F0F8
:100450001F0302FA03F3154A42F8213010BD4FF48E
:100460009E23C0E74FF41D23BDE7114BBBE7114BA3
:10047000B9E7114BB7E7114BB5E7114BB3E74FF4B1
:100480001D03B0E74FF46B03ADE70E4BABE74FF046
:10049000EB73A8E74FF06C73A5E74FF08063A2E71A
:1004A0004FF0E8639FE700BF90D0030000E100E059
:1004B00000B013000050270000F03A0000A04E00EA
:1004C00000C0750000903A012DE9F0411E4600255C
:1004D0004FF47A73C0E901530D4B044640F8143BC6
:1004E00017468846FFF711FD0A4AC4F8108084F8C1
:1004F0005C7052F8263084F85D309DF8183052F860
:10050000233084F85E3084F861502046BDE8F081E5
:10051000CC9801003C98010010B50369D3F808217C
:1005200004464AB1D3F818151430C9B2FFF7F6FCE7
:1005300023690022C3F8082110BD00000148FFF71D
:10054000EBBF00BFD407002007B519230093022298
:10055000182303490348FFF7B7FF03B05DF804FB16
:1005600000200040D407002010B5044628B103F055
:1005700047FB90FBF4F303FB1404204610BD8842B4
:1005800010B5044603DA081AFFF7EEFF04442046CC
:1005900010BD10B5029C401AE41A6043521A90FB39
:1005A000F2F0184410BD10B50446006802F08CFC4F
:1005B000204610BD10B50446006808B102F084FC66
:1005C00000232360C4E9013310BD38B504460D464D
:1005D0000068013103F048FB10B1C4E900050120B7
:1005E00038BD036810B5044623B143688B4201D37C
:1005F000012010BD2046FFF7E8FF0028F9D0A368CE
:10060000002BF5D122681370F2E770B50E46114643
:1006100004461546FFF7E5FF20B92046FFF7CAFF5D
:10062000204670BDA5603146206803F01CFCF7E74A
:1006300038B500230446C0E9003383600D4639B164
:10064000084603F034FC294602462046FFF7DDFF4A
:10065000204638BD38B5054608460C4603F027FC51
:10066000214602462846BDE83840FFF7CEBF38B5E0
:10067000054600680C4668B16A688B689A4207D3E1
:10068000096803F0F0FBA368AB600023A36038BDEA
:1006900002F01AFC23682B6063686B60A368AB6090
:1006A0000023C4E90033F1E7884210B50B46044645
:1006B00004D0096821B19A68FFF7A7FF204610BD52
:1006C000FFF778FFFAE710B500230446C0E90033CE
:1006D0008360FFF7E9FF204610BD884210B504464D
:1006E00001D0FFF7C4FF204610BD10B5044619B174
:1006F000FFF7B0FF204610BDFFF75CFFFAE770B5CB
:1007000005460E4609B9002070BD6AB184681444DC
:100710002146FFF766FF0028F5D02868AB68314610
:10072000184403F0A0FBAC600120EDE707B50023FF
:100730008DF80410012201A98DF80530FFF7DFFFC5
:1007400003B05DF804FB10B58A6809680446FFF73A
:10075000D6FF10B92046FFF72DFF204610BD826856
:1007600008B53AB921B10878B0FA80F0400900E044
:10077000012008BD006809B90078F5E703F069FBBE
:10078000F2E7884270B515D083688A6893420FD12A
:1007900083B104680D68013C14F8010F50B104F0F6
:1007A0009BFB064615F8010B04F096FB8642F3D03E
:1007B000002070BD0120FCE783688B4201D90068EE
:1007C00018B903480023037070470844704700BFFE
:1007D000380800208368934210B506D90468A01831
:1007E00003F02AFB08B1001B10BD4FF0FF30FBE700
:1007F0000022FFF7EFBFF8B583689342054602D8A1
:100800004FF0FF30F8BD0368541C00221F5D1A55DD
:100810000668304603F09AFB37550028F0D02B6865
:10082000C01AEFE78268013AFFF7E5BF2DE9F04112
:100830009A420E461F460F4988BF1346154680460A
:1008400084BF3D461F46FFF7F3FEB468AC420DD9A6
:10085000BC4228BF3C46336800221F5D1A553168F0
:1008600040462944FFF741FF33681F554046BDE825
:10087000F08100BF02980100FEE700000A4B1968F2
:100880000A4B30B5D3F804050C060D0A44EA000201
:100890004FF47A712B46A2FB014501FB0355E00B97
:1008A00040EA454030BD00BF3C0800200010014038
:1008B000094B1968094B30B5D3F804050D0A0C062D
:1008C000074944EA00022B46A2FB014501FB035500
:1008D000E00B40EA454030BD3C08002000100140DC
:1008E00040420F0038B5044648B1FFF7C7FF054640
:1008F00000F01AF8FFF7C2FF401BA042F8D338BD42
:10090000074B0022C3F8042182B0D3F80431054A12
:100910000193019B13680133DBB2136002B070478F
:10092000001001403C080020704770B58AB061B1EA
:10093000931E222B20D801AB1D4648B9AB4207D0ED
:100940000A46AB4213D80023137008460AB070BDA4
:10095000B0FBF2F402FB1406092E204603F101035A
:10096000F4B294BF3034573403F8014CE5E713F880
:10097000010D02F8010BE4E70021E6E770470000F3
:1009800008B500F015F8FFF7F9FF0120FFF7AAFFFF
:10099000F4F754FF034CF4F753FF002CFBD0AFF3F4
:1009A0000080F8E70000000002F086BA02F08CBA7E
:1009B0002A4BE02283F811234FF40032C3F8802140
:1009C0001A604FF080430122C3F818259A6003F59E
:1009D00088330021C3F808150221C3F80413C3F8B3
:1009E00044131A604FF01023D3F80022002A03DBCF
:1009F000D3F80432002B2FDA194B0122C3F8042557
:100A0000D3F80024002AFBD04FF010221521C2F8A1
:100A10000012D3F80024002AFBD04FF01023152237
:100A2000C3F804220E4B1A46D3F800140029FBD059
:100A30000021C3F80415D2F80034002BFBD0BFF31B
:100A40004F8F0849084BCA6802F4E0621343CB6039
:100A5000BFF34F8F00BFFDE7704700BF00E100E02C
:100A600000E0014000ED00E00400FA05192837B568
:100A70000CD84B4B53F82030052B00F0828007D860
:100A8000032B12D07BD8022B00F08180002074E071
:100A90001D2B78D003D81C2BF8D1052206E01E2B85
:100AA00073D01F2BF2D1082200E002223D4B1968BF
:100AB00008296EDD0A296FDD0D29B5BF0C240E242F
:100AC000022303233848C0F8F0350123C0F800356D
:100AD00000200546030103F1804303F5E0430130A4
:100AE0000828C3F81455C3F81055F3D12F4B1868D4
:100AF0002F4B1B6800021B0303F4805300F4E060DB
:100B00001843294BC3F81805C3F81425C3F810255A
:100B10000DF10602C3F82C260122C3F830261A6014
:100B2000D3F80021002AFBD00022C3F800210122C3
:100B30005A601D4B1A46D3F804010028FBD0002050
:100B4000C3F8040101209860D2F81431002BFBD0C7
:100B50000023C2F81431BDF906209A42124AB8BFE8
:100B6000ADF80630A142C2F80035BDF9060004D048
:100B700035BF611A091BC840884003B030BD03224D
:100B800094E7042292E7062290E707228EE70122EB
:100B90008CE70824002395E70A24012392E700BF8D
:100BA0003C98010028000020007000402C0000202C
:100BB00048080020192830B53CD8224B53F82000B3
:100BC000214B00221D4653F82240B4F1FF3F32D1A1
:100BD0001E4C45F822006FEA41411D4D1D4B246813
:100BE00053F822306FEA514125F81210012101FA21
:100BF00004F4C3F86005013CC3F8640505EB420248
:100C0000C3F86805C3F86C050020C3F80015C3F8E5
:100C10000C05C3F80405C3F80845C3F81405C3F868
:100C20001005C3F82025C3F82415C3F82815C3F808
:100C30002C05996030BD8442CAD00132032AC2D14A
:100C4000F8E700BF3C9801001C00002030000020A5
:100C500040080020F498010019280FD8114B53F8D0
:100C6000203003290AD8DFE801F002160A1003F544
:100C7000E0734FF0A042002142F82310704703F5C3
:100C8000E0734FF0A0420C21F6E703F5E0734FF05C
:100C9000A0420421F0E703F5E0734FF0A0420321E6
:100CA000EAE700BF3C98010019280CD8064B53F81E
:100CB0002020012393404FF0A04211B9C2F80C3517
:100CC0007047C2F8083570473C98010019289FBF4B
:100CD0004FF0A043054AD3F8103552F820009ABFD0
:100CE00023FA00F000F00100002070473C9801005A
:100CF00038B50025057329B90B4B0C4A0C48252142
:100D000001F088FE01600B4951F82220027151F870
:100D1000233083719DF8103051F823304371022342
:100D2000C371856038BD00BF00990100639901005F
:100D30000E9901003C980100037B23B94373837330
:100D4000036101230373704784B00DF1100C0CE9AB
:100D50000E009DF80810026800230129C2F8003532
:100D6000039B12D00BD303290CD0C2F85435019B3E
:100D7000C2F824350123C2F8003504B0704743F0AF
:100D80000203F2E743F00403EFE743F00603ECE766
:100D900010B5FFF7D1FF03688279C3F808254279BF
:100DA000C3F80C250279C3F81025034BBDE81040A9
:100DB0000ECBFFF7C9BF00BF6008002010B485B09C
:100DC00001AC84E80E0094E80E0005B05DF8044B19
:100DD000FFF7BABF70470368C3F81C15D3F80821A2
:100DE000002AFBD0D3F818050022C3F80821C0B2AE
:100DF0007047000007B5094B09490A484FF0804287
:100E00001A6000229A6002221A710B2300930C22AE
:100E10000D23FFF76DFF03B05DF804FB60080020B1
:100E2000003002404C0800200B460146184601F0F5
:100E30001BBE0000C0F3C7537F3B162B024605DCE8
:100E4000002B04DB0348184122EA0000704700F041
:100E500000407047FFFF7F002DE9F04FDFF82C9333
:100E60008DB006460F4614461D4600F095F999F9D7
:100E70000080B8F1FF3FCDE9000136D022462B4675
:100E80002046294601F018FD834670BB32463B469A
:100E90003046394601F010FD8246002840F0A2801D
:100EA000304639460022002301F0D4FC10B3002262
:100EB00000232046294601F0CDFC8346002867D058
:100EC0009FEDA77B0122AC4BCDF828A00292CDE983
:100ED0000467CDE906458DED087B0393B8F1000F5B
:100EE00041D09FEDA17B8DED007BDDE900010DB0D0
:100EF000BDE8F08FDDE9000100F066FF80460028C4
:100F000000F08D804FF0000A4FF0000BDDE900018A
:100F100052465B4601F09EFC0028E6D0304639463A
:100F200000F052FF0028E0D02046294600F04CFF98
:100F30000028DAD099F900308F4A03920421002268
:100F4000022BCDE90467CDE90645CDE908AB029156
:100F50000A9203D002A800F03DFF50B901F092FDC3
:100F60002223036005E002A800F034FF002800F00F
:100F70009B800A9B1BB101F085FD0A9B03609DEDE0
:100F8000087B8DED007BDDE900010DB0BDE8F08F41
:100F90002046294600F018FF0028A6D00022002392
:100FA0002046294601F060FC00289ED0724A99F93B
:100FB0000030CDF828B00121CDE90467CDE9064520
:100FC000CDE90212002B74D06C490020022BCDE930
:100FD000080172D101F056FD212303600A9B002B0A
:100FE000CDD0C8E7002200232046294601F032FC7C
:100FF00000283FF47AAF624B5F49CDF828B0002259
:101000000120B8F1020FCDE904670290CDE9064551
:10101000CDE908230391A6D1CDE9002365E7304649
:10102000394600F0D1FE00283FF46CAF2046294637
:1010300000F0CAFE00283FF465AFDDE9002310464A
:10104000194601F039FC99F900A000286BD103235F
:10105000DFF824C10A902946204602930022494B1A
:10106000CDF80CC0CDE90645CDE9046701F08AF959
:1010700004460D46BAF1000F25D1DFF814B14FF048
:10108000604A0022002330463946CDE908AB01F022
:10109000EBFB38BB02A800F09DFE00289ED101F0BA
:1010A000F1FC2223036099E701F0ECFC21230360AB
:1010B0005FE79FED2B7B8DED087B02A800F08AFE99
:1010C00000288BD186E79FED2A7B00220023304643
:1010D00039468DED087B01F0C7FBA0B9BAF1020FCC
:1010E000DDD0D7E72046294600F07CFE22462B467D
:1010F00001F0B0FBA0B9244B99F900A04FF0604279
:10110000CDE90823EAE72046294600F06BFE224697
:101110002B4601F09FFB18B9184B0022CDE908239C
:1011200099F900A0DAE70122134BCDF8288002924A
:10113000CDE90467CDE906450393BAF1000FB8D0B5
:10114000002200231046194601F046FABAF1020FB8
:10115000CDE908013FF43EAFAFE700BFAFF3008039
:101160000000000000000000000000000000F03F50
:10117000000000000000F07FA09901000000F0FFD7
:101180000000F03F0000E03FFFFFEFC73400002009
:10119000FFFFEF47000000002DE9F04F23F000456E
:1011A00055EA020493B00DD06B4E21F00044B442D6
:1011B0000F4682460BDD04F1404404F5801454EAE6
:1011C0000A0350D16549002013B0BDE8F08F9B465B
:1011D000944647D0B542EEDC5F4EB5425DD0002F5D
:1011E00080468946CDE900235BDB0026BCF1000F79
:1011F0000ED1594B9D423FD0584B9D4200F0888004
:10120000BBF1804F00F09C80554B9B4500F0B883AC
:101210004046494600F0D4FDBAF1000F06D1002C3B
:1012200059D04E4B27F040429A4254D0FF0F013F15
:1012300056EA070373D04B4B9D4240F39B8003F16A
:1012400004739D4240F33E84474B9C4272DDBBF1E8
:10125000000F72DD3EA3D3E900231046194601F0CA
:1012600091F8B1E728B1414813B0BDE8F04F00F064
:10127000B3BDA542F7DCAFE704F1404303F58013AB
:1012800053EA0A039ED0384B9C4240F38383BBF160
:10129000000F52DBDDE9000196E7BCF1000F9ED0A4
:1012A00089E7334B9D4231DCA3F154739D429CDDB1
:1012B0002B15A3F2FF33142B40F3A583C3F13403A2
:1012C0002CFA03F202FA03F363458ED102F0010215
:1012D000C2F102068AE7BBF1000F05DA02460B46AF
:1012E00000201E4901F078F9002FBFF66DAF04F120
:1012F000404404F5801454EA060300F03F84012EB4
:101300007FF462AF01F1004319465DE702266DE705
:10131000BBF1000FC0F248834046494654E74246BD
:101320004B461046194600F075FE02460B4601F08A
:1013300053F949E7BBF1000F8CDB0020002143E7A4
:1013400042464B464046494601F01CF83CE700BF88
:101350009C7500883CE4377E0000F07F0000F03F81
:101360000000E03F0000E041FFFFEF3FA4990100D3
:10137000FFFF3F43B4F5801F80F261830022D24B10
:1013800001F000F86FF0340C0C462315CF4DC4F378
:101390001302A3F2FF3342F07F546344AA420B933B
:1013A00044F4401440F33F83C94B9A4240F3048411
:1013B0009FEDAF7B8DED087B8DED107B9FEDAE7BC0
:1013C0000B9B8DED067B01330B93A4F58014002558
:1013D000DDE906232146824600F01CFEA346DDE936
:1013E00006238046894650462146CDE90CAB00F0E5
:1013F00013FE02460B460020B64901F0EDF80A46FE
:101400000146CDE90E12134649460246404600F019
:10141000B9FF631043F0005382468B4603F5002367
:101420008C46CDE904AB5919D3460023CDE902BC63
:101430000293DDE902AB002004460D4602460B464E
:101440005046594600F09EFF02460B46404649462C
:1014500000F0E0FDDDE90623804689462046294666
:1014600000F0D8FD02460B46DDE90C0100F0D2FD8C
:1014700052465B4600F086FF02460B464046494610
:1014800000F0C8FDDDE90E2300F07CFFDDE9044536
:10149000CDE9060122462B462046294600F072FF80
:1014A00077A3D3E9002304460D4600F06BFF76A333
:1014B000D3E9002300F0B0FD22462B4600F062FF86
:1014C00073A3D3E9002300F0A7FD22462B4600F0CA
:1014D00059FF71A3D3E9002300F09EFD22462B465D
:1014E00000F050FF6EA3D3E9002300F095FD2246E3
:1014F0002B4600F047FF6CA3D3E9002300F08CFDDE
:101500002246804689462B462046294600F03AFF6F
:1015100002460B464046494600F034FF5246044618
:101520000D465B46DDE9040100F076FDDDE90623AA
:1015300000F028FF22462B4600F06EFD5246804602
:1015400089465B465046594600F01CFF0022624B1C
:10155000CDE90C0100F060FD42464B4600F05CFD19
:1015600002980D46044622462B465046594600F046
:1015700009FF002282468B46574B2046294600F041
:1015800049FDDDE90C2300F045FD02460B464046CF
:10159000494600F03FFDDDE9042300F0F3FE22465A
:1015A000804689462B46DDE9060100F0EBFE024647
:1015B0000B464046494600F02FFD804689460246CC
:1015C0000B465046594600F027FD029838A3D3E950
:1015D000002304460D4600F0D5FE5246CDE9040135
:1015E0005B462046294600F015FD02460B46404664
:1015F000494600F00FFD30A3D3E9002300F0C2FEFE
:101600002FA3D3E90023804689462046294600F0CF
:10161000B9FE02460B464046494600F0FDFCDDE9B6
:10162000102300F0F9FC80460B98894600F040FE3C
:10163000424682468B464B46DDE9040100F0ECFC55
:10164000DDE9082300F0E8FC52465B4600F0E4FCCC
:10165000029852465B4604460D4600F0DBFCDDE98D
:10166000082300F0D7FCDDE9042337E0AFF3008066
:101670000000000000000000000000000000F03F3B
:10168000EF4E454A287ECA3F65DBC9934A86CD3F67
:1016900001411DA96074D13F4D268F515555D53F4D
:1016A000FFAB6FDBB66DDB3F033333333333E33FE5
:1016B000000000E009C7EE3FFD033ADC09C7EE3F3A
:1016C000F5015B14E02F3EBE000040438E980300FE
:1016D00079B60B000000F03F0000084000F09AFCD3
:1016E0000B4602464946404600F094FC013E56EA4D
:1016F000070382468B4600F05E819FEDD37B8DED24
:10170000047BDDE9001200230E461746CDE902678F
:101710000293DDE9026708463B461146324600F077
:1017200079FC22462B4600F02DFEDDE900238046A1
:1017300089465046594600F025FE02460B46404673
:10174000494600F069FC3246804689463B462046C1
:101750002946CDE9008900F015FE0B4602460646F3
:101760000F464046494600F057FCD14B994204468B
:101770000D468A4640F3248101F13F4303F5E0031F
:10178000034340F0FF81B2A3D3E90023DDE9000168
:1017900000F042FC3246804689463B4620462946B8
:1017A00000F038FC02460B464046494601F07AF804
:1017B000002840F0E781A8464FEA2853A3F2FE3202
:1017C0004FF4801313415344C3F30A52B94DA2F2AC
:1017D000FF321541C3F3130423EA05010020C2F1CF
:1017E000140B44F48014BAF1000F02460B4644FA7D
:1017F0000BFB30463946B8BFCBF1000B00F00AFCBA
:1018000006460F463246DDE900013B4600F004FC87
:101810004FEA0B5A0D4600248FA3D3E9002320463C
:10182000294600F0AFFD3246804689463B462046B9
:10183000294600F0EFFB02460B46DDE9000100F00F
:10184000E9FB87A3D3E9002300F09CFD86A3D3E93D
:10185000002306460F462046294600F093FD024627
:101860000B463046394600F0D7FB06460F46024687
:101870000B464046494600F0CFFB42464B460446E5
:101880000D4600F0C7FB02460B463046394600F0D5
:10189000C1FB2246804689462B462046294600F059
:1018A00071FD73A3D3E9002306460F4600F06AFDDD
:1018B00071A3D3E9002300F0ADFB32463B4600F0B4
:1018C00061FD6FA3D3E9002300F0A6FB32463B463F
:1018D00000F058FD6CA3D3E9002300F09BFB3246D7
:1018E0003B4600F04FFD6AA3D3E9002300F094FBD0
:1018F00032463B4600F046FD02460B46204629464E
:1019000000F088FB06460F4602460B462046294655
:1019100000F038FD0022CDE900014FF08043304651
:10192000394600F077FB02460B46DDE9000100F086
:1019300053FE424606460F464B462046294600F0D7
:1019400021FD42464B4600F067FB02460B463046FF
:10195000394600F05FFB22462B4600F05BFB024657
:101960000B460020544900F055FB8A44BAF5801F0D
:10197000C0F232815146DDE9042300F003FD23E487
:10198000002FFFF645AC4046494613B0BDE8F04F86
:1019900000F056B9BBF1000FBFF6CFACDDE9003463
:1019A000184604F100410FE442464B4600204249EC
:1019B00000F012FE08E49FED387B8DED047BA0E67D
:1019C0003E4B21F00048984540F3EA803C4B0B44E5
:1019D00003430AD132463B4600F01CFBDDE90023FD
:1019E00000F056FF00283FF4E7AEDDE904012CA328
:1019F000D3E9002300F0C6FC29A3D3E9002300F0BB
:101A0000C1FCFFF7E1BBBCF1000F40F0D280C3F195
:101A1000140345FA03F202FA03F3AB4200F0E0804C
:101A20006646FFF7E9BB9FED207B8DED087B8DEDD2
:101A3000107B9FED057B00258DED067BC8E44FF004
:101A4000000CA2E4AFF30080000000000000F03FB3
:101A5000FE822B654715973C00000000432EE63FB1
:101A6000EF39FAFE422EE63F396CA80C615C20BECD
:101A7000D0A4BE726937663EF16BD2C541BDBB3E94
:101A80002CDE25AF6A56113F93BDBE166CC1663F72
:101A90003E5555555555C53F000000000000F0BFAC
:101AA00059F3F8C21F6EA5010000000000000000FD
:101AB000FFFF8F40FFFF0F000000F03FFFCB904083
:101AC00000346F3F5A4B9C427FF734AC594B9C42D9
:101AD0003FF7BDAB0022574B00F09CFA44A3D3E97B
:101AE000002304460D4600F04DFC43A3D3E9002338
:101AF00082468B462046294600F044FC0022CDE970
:101B000002014D4B2046294600F03CFC02460B46A4
:101B10003BA1D1E9000100F07DFA22462B4600F0FE
:101B200031FC02460B460020444900F073FA22467D
:101B3000804689462B462046294600F023FC024673
:101B40000B464046494600F01DFC2FA3D3E9002375
:101B500000F018FC02460B46DDE9020100F05AFADB
:101B600002460B46804689465046594600F054FAD4
:101B7000002004460D4652465B46AFE502460B4642
:101B8000FFF7CFBBDDE9040121A3D3E9002300F077
:101B9000F9FB1FA3D3E9002300F0F4FBFFF714BB0C
:101BA000264B98453FF708AEDDE90223924693465F
:101BB00031E60026FFF72CBB9FED177B8DED087BF0
:101BC0009FED177B8DED107B9FED177B4FF48025EC
:101BD0008DED067BFFF7FCBB5A4600F091F9CAE693
:101BE00002F00102C2F10206FFF706BBAFF300806C
:101BF000000000604715F73F44DF5DF80BAE543E30
:101C0000555555555555D53FFE822B654715F73F20
